:100000000C94C30F0C94F40F0C94F40F0C94F40F95
:100010000C94F40F0C94F40F0C94F40F0C94F40F54
:100020000C94F40F0C94F40F0C94F40F0C94F40F44
:100030000C94F40F0C94F40F0C94F40F0C94F40F34
:100040000C94F40F0C94FB920C94F40F0C94F40F9A
:100050000C94F40F0C94F40F0C942EA50C949BC7E5
:100060000C94F40F0C949F210C94F40F0C94F40F47
:100070000C94F40F0C94F40F0C94F40F0C94F40FF4
:100080000C94F40F0C94F40F0C94F40F0C94F40FE4
:100090000C94F40F0C94F40F0C94F40F0C94B2C461
:1000A0000C94F40F0C94F40F0C94F40F0C94F40FC4
:1000B0000C94F40F0C94F40F0C94F40F0C94F40FB4
:1000C0000C94F40F0C94F40F0C94F40F0C94F40FA4
:1000D0000C94F40F0C94F40F0C94F40F0C94F40F94
:1000E0000C94F40F88A597A5B6A5C5A5E0A5E4A531
:1000F000E7A5EBA5EEA5F2A5F5A5F9A503A6C9C848
:10010000CEC8D3C8DDC8E7C860C9F1C8F9C801C9FD
:100110000BC915C91FC92EC938C960C942C94CC904
:1001200056C981C984C973C977C97DC9BBC988C982
:100130008CC992C996C99AC9A0C9A4C9A8C9BBC982
:10014000AEC9B2C9B6C9084AD73B3BCE016E84BC22
:10015000BFFDC12F3D6C74319ABD56833DDA3D0021
:10016000C77F11BED9E4BB4C3E916BAAAABE00006A
:1001700000803F05A84CCDB2D44EB93836A9020C48
:1001800050B9918688083CA6AAAA2ABE0000008021
:100190003F004D383420582059205A2045004361F3
:1001A0006E6E6F7420656E7465722073756264691B
:1001B000723A20004D3234004D32332025730061F5
:1001C00075746F25692E67006572726F7220777281
:1001D0006974696E6720746F2066696C65004E6F84
:1001E00074205344207072696E74696E67005344C2
:1001F000207072696E74696E672062797465200080
:1002000044656C6574696F6E206661696C65642C09
:100210002046696C653A200046696C652064656C0F
:10022000657465643A006F70656E206661696C651F
:10023000642C2046696C653A200057726974696EB7
:100240006720746F2066696C653A20002E0A006F83
:1002500070656E206661696C65642C2046696C650A
:100260003A20002E0A006F70656E206661696C6529
:10027000642C2046696C653A200046696C652073E1
:10028000656C6563746564002053697A653A200083
:1002900046696C65206F70656E65643A20006F700A
:1002A000656E206661696C65642C2046696C653AF0
:1002B00020004E6F772066726573682066696C65F2
:1002C0003A20004E6F7720646F696E672066696C14
:1002D000653A20002220706F7300222070617265E1
:1002E0006E743A2200535542524F5554494E4520A0
:1002F00043414C4C207461726765743A22004B494B
:100300004C4C45442E2000747279696E6720746FDE
:100310002063616C6C207375622D67636F64652068
:1003200066696C6573207769746820746F6F206DDF
:10033000616E79206C6576656C732E204D41582076
:100340006C6576656C2069733A0053442063617272
:1003500064206F6B006F70656E526F6F7420666102
:10036000696C656400766F6C756D652E696E697475
:10037000206661696C656400534420696E6974206D
:100380006661696C0020204D383531205A005A2DA5
:1003900050726F6265204F666673657420286D6DBC
:1003A000293A0020204D3230302044300020204DAA
:1003B0003230302044002044697361626C6564000F
:1003C00046696C616D656E742073657474696E67DF
:1003D000733A00204C0020430020440020490020B4
:1003E000204D3330312050005049442073657474DF
:1003F000696E67733A0020460020420020204D318C
:100400003435204D31204800204600204200202075
:100410004D313435204D302048004D61746572698E
:10042000616C2068656174757020706172616D65C2
:10043000746572733A00205A0020590020204D3212
:100440003036205800486F6D65206F66667365749E
:1004500020286D6D293A00204500205A00205800C0
:1004600020420020540020204D32303520530041DE
:100470006476616E636564207661726961626C6541
:10048000733A20533D4D696E2066656564726174F0
:100490006520286D6D2F73292C20543D4D696E20E9
:1004A00074726176656C206665656472617465203E
:1004B000286D6D2F73292C20423D6D696E696D7515
:1004C0006D207365676D656E742074696D65202895
:1004D0006D73292C20583D6D6178696D756D2058BC
:1004E00059206A65726B20286D6D2F73292C20208E
:1004F0005A3D6D6178696D756D205A206A65726B21
:1005000020286D6D2F73292C2020453D6D61786961
:100510006D756D2045206A65726B20286D6D2F7397
:10052000290020540020520020204D323034205029
:1005300000416363656C65726174696F6E733A2024
:10054000503D7072696E74696E672C20523D726501
:10055000747261637420616E6420543D74726176BC
:10056000656C00204500205A0020590020204D32A3
:1005700030312058004D6178696D756D204163639D
:10058000656C65726174696F6E20286D6D2F7332B2
:10059000293A00204500205A0020590020204D32E1
:1005A00030332058004D6178696D756D2066656542
:1005B00064726174657320286D6D2F73293A002071
:1005C0004500205A0020590020204D393220580083
:1005D00053746570732070657220756E69743A008B
:1005E00048617264636F6465642044656661756C1C
:1005F000742053657474696E6773204C6F61646511
:10060000640020496E76616C696420657874727547
:1006100064657220005072696E7465722068616C46
:100620007465642E206B696C6C28292063616C6C86
:10063000656421004B494C4C45442E20004B494CED
:100640004C45442E200020746F6F206C6F6E672025
:10065000657874727573696F6E2070726576656EF9
:100660007465640020636F6C6420657874727573C0
:10067000696F6E2070726576656E746564006F6B6D
:1006800000526573656E643A20003A20007A5F6D0F
:1006900061783A20007A5F6D696E3A20006F6B00D6
:1006A0005A204F6666736574004D333030205336E0
:1006B000353920503230300A4D33303020533639FE
:1006C000382050323030004F666673657420617098
:1006D000706C6965642E004D333030205334302007
:1006E00050323030004572723A20546F6F2066618C
:1006F000722100546F6F206661722066726F6D20E8
:100700007265666572656E636520706F696E7400F0
:1007100053657474696E672054726176656C20410C
:100720006363656C65726174696F6E3A200053652E
:100730007474696E672052657472616374204163DA
:1007400063656C65726174696F6E3A2000536574FD
:1007500074696E67205072696E7420416363656CC2
:1007600065726174696F6E3A200053657474696EC6
:1007700067205072696E7420616E642054726176D5
:10078000656C20416363656C65726174696F6E3A74
:1007900020004D31343520533C696E6465783E202D
:1007A0006F7574206F662072616E67652028302D2A
:1007B0003129007A5F6D61783A20007A5F6D696E49
:1007C0003A2000795F6D61783A2000795F6D696E3B
:1007D0003A2000785F6D696E3A2000205A3A002076
:1007E000593A0020436F756E7420583A2000204516
:1007F0003A00205A3A0020593A00583A00464952E5
:100800004D574152455F4E414D453A4D61726C69BD
:100810006E20312E312E302046726F6D2041726372
:100820006869766520534F555243455F434F4445B1
:100830005F55524C3A687474703A2F2F202E2E2E2A
:100840002050524F544F434F4C5F56455253494FDF
:100850004E3A312E30204D414348494E455F545960
:1008600050453A454E444552203344204558545251
:10087000554445525F434F554E543A3120555549E2
:10088000443A30303030303030302D303030302D50
:10089000303030302D303030302D3030303030305E
:1008A0003030303030300A00454E44455220334419
:1008B000204F66662E00454E444552203344207238
:1008C000656164792E0042656420646F6E652E0058
:1008D00020423A0020453A00543A004265642048DC
:1008E000656174696E672E0048656174696E672082
:1008F000646F6E652E003F0020573A0020453A0095
:10090000543A0048656174696E672E2E2E002042AD
:10091000403A0020403A00202F00205400202F00B1
:1009200020423A00202F0020543A006F6B004B49C0
:100930004C4C45442E2000444542554720445259D2
:1009400052554E20454E41424C4544004445425587
:1009500047204543484F20454E41424C45440053B3
:1009600074616E6461726420446576696174696F54
:100970006E3A20004D65616E3A2000202020736998
:10098000676D613A2000206D65616E3A200020207D
:10099000207A3A2000206F662000793A2000783AC9
:1009A0002000506F736974696F6E696E6720746898
:1009B000652070726F62652E2E2E0A003F4E756D97
:1009C000626572206F66206C65677320696E206DAA
:1009D0006F76656D656E74206E6F7420706C6175D6
:1009E0007369626C652028302D3135292E0A005933
:1009F0000058003F53616D706C652073697A652003
:100A00006E6F7420706C61757369626C6520283438
:100A10002D3530292E0A004D3438205A2D50726F52
:100A20006265205265706561746162696C69747990
:100A300020746573740A003F566572626F73652097
:100A40004C6576656C206E6F7420706C617573698F
:100A5000626C652028302D34292E0A002569206D0E
:100A6000696E2C2025692073656300456E642066DD
:100A7000696C65206C69737400426567696E2066F5
:100A8000696C65206C697374004E6F206D6F7665BC
:100A90002E00454E444552203344207265616479EE
:100AA0002E00526573756D696E67207072696E7481
:100AB000005761697420666F7220757365722E2EFF
:100AC0002E00205A3A200020593A20004265642026
:100AD000583A2000205A3A200020593A2000426516
:100AE0006420583A2000202B00200A436F72726560
:100AF0006374656420426564204865696768742092
:100B000076732E2042656420546F706F6C6F677926
:100B10003A200A00202B002B2D2D2D2D2D2D2D2D93
:100B20002D2D2D2B0A007C2E2E2E46726F6E742ECC
:100B30002E2E7C0A007C4C6566742E2E52696768E6
:100B4000747C0A007C2E2E2E4261636B2E2E2E2E7C
:100B50007C0A002B2D2D2D2D2D2D2D2D2D2D2D2BCA
:100B60000A00200A42656420486569676874205459
:100B70006F706F6772617068793A200A004D656125
:100B80006E206F662073616D706C656420706F6994
:100B90006E74733A200020643A200020623A2000EC
:100BA00045716E20636F656666696369656E74730F
:100BB0003A20613A200028422961636B00284629C7
:100BC000726F6E74002852296967687400284C2976
:100BD000656674003F4E756D626572206F662070A9
:100BE000726F626564202850296F696E7473206982
:100BF0007320696D706C61757369626C6520283251
:100C0000206D696E696D756D292E0A0052756E6EC4
:100C1000696E6720696E204452592D52554E206DE1
:100C20006F646500473239204175746F20426564F6
:100C3000204C6576656C696E670A003F2856296509
:100C400072626F7365204C6576656C2069732069EC
:100C50006D706C61757369626C652028302D342964
:100C60002E00486F6D6520582F59206265666F729F
:100C700065205A00486F6D6520582F5920626566BF
:100C80006F7265205A005761726E696E673A20482C
:100C90006F6D696E672042756D7020446976697367
:100CA0006F72203C203100486F6D6520582F59200D
:100CB0006265666F7265205A00486F6D6520582F17
:100CC00059206265666F7265205A005A2070726FF3
:100CD0006265206F75742E20626564005A20707200
:100CE0006F6265206F75742E2062656400536C65B9
:100CF00065702E2E2E0020706F736974696F6E20E0
:100D00006F7574206F662072616E67652E003F50AC
:100D1000726F62652000220A00556E6B6E6F776EEF
:100D200020636F6D6D616E643A2022002569206832
:100D30006F757273202569206D696E757465730017
:100D4000446F6E65207072696E74696E67206669A3
:100D50006C65004B494C4C45442E200053544F5079
:100D60005045442E20005072696E74657220737471
:100D70006F707065642064756520746F2065727291
:100D80006F72732E204669782074686520657272D0
:100D90006F7220616E6420757365204D393939207A
:100DA000746F20726573746172742E202854656D9F
:100DB0007065726174757265206973207265736500
:100DC000742E2053657420697420616674657220E6
:100DD00072657374617274696E6729004E6F204C7E
:100DE000696E65204E756D62657220776974682042
:100DF000636865636B73756D2C204C617374204C54
:100E0000696E653A20004E6F20436865636B7375A9
:100E10006D2077697468206C696E65206E756D62EF
:100E200065722C204C617374204C696E653A200009
:100E3000636865636B73756D206D69736D61746351
:100E4000682C204C617374204C696E653A20004C0C
:100E5000696E65204E756D626572206973206E6FD4
:100E600074204C617374204C696E65204E756D6200
:100E700065722B312C204C617374204C696E653A7D
:100E800020004D313130006F6B00446F6E65207370
:100E90006176696E672066696C652E004D32390097
:100EA0002020506C616E6E65724275666665724296
:100EB000797465733A20002046726565204D656D32
:100EC0006F72793A20004A756C203130203230310F
:100ED0003700436F6D70696C65643A2000286E6F4F
:100EE0006E652C2064656661756C7420636F6E6638
:100EF00069672900207C20417574686F723A200070
:100F0000323031352D31322D30312031323A3030DE
:100F100000204C61737420557064617465643A20DC
:100F20000020004D61726C696E0020536F6674770B
:100F3000617265205265736574002057617463683F
:100F4000646F67205265736574002042726F776E1C
:100F5000206F757420526573657400204578746540
:100F6000726E616C20526573657400506F776572A4
:100F70005570007374617274002200656E7175653E
:100F80007565696E67202200FFFFFF0000A040002A
:100F900000A0400000004000005C4300005C4300F3
:100FA00000A5430000000000000000000000000059
:100FB000005C4300005C430000A54300000000000B
:100FC000000000000000006563686F3A004572721F
:100FD0006F723A0020746F6F206C6F6E67206578B7
:100FE00074727573696F6E2070726576656E746564
:100FF000640020636F6C6420657874727573696F28
:101000006E2070726576656E746564007C3C3E5E31
:101010002B3D3F2F5B5D3B2C2A225C004D3834205A
:10102000582059205A204500656E6473746F7073A0
:10103000206869743A205A00205A3A00656E647339
:10104000746F7073206869743A20590020593A000F
:10105000656E6473746F7073206869743A20580009
:1010600020583A00656E6473746F707320686974F9
:101070003A200024F4D43050C38E20C2A2401782FC
:101080008B7011127A910D816CD90AA861E108C7A1
:10109000586607615143061E4B5D05C145A7041AFA
:1010A000411104093D9803713931034036DB026573
:1010B000339102D4305402802E1D02632CEE017550
:1010C0002AC501B028A001102781018F2564012BBA
:1010D000244B01E0223401AC211F018D200D018041
:1010E0001FFC00841EED00971DDF00B81CD200E637
:1010F0001BC600201BBC00641AB200B219A8000A6B
:1011000019A0006A189900D117910040178B00B5FB
:1011100016840031167E00B31579003A157300C7A6
:10112000146F0058146A00EE1366008813630025DC
:10113000135E00C7125B006C12570015125400C1F9
:1011400011510070114F0021114B00D61049008D34
:101150001047004610440002104200C00F400080BB
:101160000F3E00420F3C00060F3B00CB0E380093B1
:101170000E37005C0E3500270E3400F30D3200C12F
:101180000D3100900D3000600D2E00320D2D000548
:101190000D2C00D90C2B00AE0C2900850C29005C0D
:1011A0000C2700350C27000E0C2600E80B2400C489
:1011B0000B2400A00B23007D0B23005A0B210039C8
:1011C0000B2100180B2000F80A1F00D90A1E00BBD3
:1011D0000A1E009D0A1D00800A1D00630A1C0047AC
:1011E0000A1B002C0A1B00110A1A00F7091A00DD5D
:1011F000091900C4091900AB091900920917007BED
:10120000091800630917004C09160036091600205A
:101210000916000A091500F5081500E0081400CCAD
:10122000081400B8081400A4081400900813007DE6
:101230000812006B08130058081200460812003408
:10124000081100230811001208110001081100F014
:10125000071000E0071000D0071000C0071000B012
:10126000070F00A107100091070E0083070F0074FD
:10127000070F0065070E0057070E0049070E003BD9
:10128000070D002E070E0020070D0013070D0006A6
:10129000070D00F9060C00ED060D00E0060C00D469
:1012A000060C00C8060C00BC060C00B0060C00A41E
:1012B000060B0099060C008D060B0082060B0077CA
:1012C000060B006C060B0061060A0057060B004C6B
:1012D000060A0042060A0038060A002E060A002402
:1012E000060A001A060A001006090007060A00FD91
:1012F000050900F4050900EB050900E2050900D91C
:10130000050900D0050900C7050900BE050900B59B
:10131000050800AD050800A50509009C0508009416
:101320000508008C050800840508007C0508007489
:101330000508006C050700650508005D05070056F7
:101340000508004E0507004705070040050800385E
:10135000050700310507002A050700230507001CC3
:10136000050600160507000F050700080506000220
:10137000050700FB040600F5040700EE040600E87C
:10138000040600E2040700DB040600D5040600CFD3
:10139000040600C9040600C3040600BD040600B725
:1013A000040600B1040500AC040600A6040600A073
:1013B0000405009B04060095040500900406008ABD
:1013C00004050085040500800406007A0405007504
:1013D000040500700405006B040500660405006147
:1013E0000405005C04050057040500520405004D87
:1013F00004050048040500430405003E0404003AC7
:1014000004050035040500300404002C0405002701
:10141000040400230405001E0404001A040400163A
:10142000040500110404000D04040009040500046F
:1014300004040000040400FC030400F8030400F4A6
:10144000030400F0030400EC030400E8030400E4D8
:10145000030400E0030400DC030400D8030400D408
:10146000030400D0030400CC030400C8030300C538
:1014700003030024F404D9201BC40C5C0E9804C49C
:10148000095F0265077101F405F900FB04B3004828
:10149000048700C10369005803550003034500BEDB
:1014A000023A008402310053022A00290225000476
:1014B000022000E4011C00C8011900AF01170098C8
:1014C000011400840113007101100061011000512A
:1014D000010E0043010D0036010B002B010B002013
:1014E000010B00150109000C01090003010800FBB4
:1014F000000800F3000800EB000700E4000600DE2F
:10150000000600D8000600D2000600CC000500C787
:10151000000500C2000500BD000400B9000400B5CC
:10152000000400B1000400AD000400A9000400A5FF
:10153000000300A20003009F0004009B000300982A
:101540000003009500020093000300900003008D4B
:101550000002008B00030088000200860002008465
:10156000000300810002007F0002007D0002007B7A
:10157000000200790002007700010076000200748A
:1015800000020072000100710002006F0002006D95
:101590000001006C0002006A00010069000200679F
:1015A00000010066000100650001006400020062A5
:1015B00000010061000100600001005F0002005DA9
:1015C0000001005C0001005B0001005A00010059AD
:1015D00000010058000100570001005600010055AD
:1015E00000010054000100530000005300010052AC
:1015F00000010051000100500001004F0001004EA9
:101600000000004E0001004D0001004C0001004BA5
:101610000000004B0001004A0001004900010048A1
:10162000000000480001004700010046000000469D
:101630000001004500000045000100440001004396
:101640000000004300010042000000420001004190
:1016500000000041000100400001003F0000003F89
:101660000001003E0000003E0001003D0000003D82
:101670000001003C0000003C0000003C0001003B79
:101680000000003B0001003A0000003A0001003970
:101690000000003900010038000000380000003868
:1016A000000100370000003700010036000000365E
:1016B0000000003600010035000000350000003554
:1016C0000001003400000034000000340001003349
:1016D000000000330000003300010032000000323F
:1016E0000000003200010031000000310000003134
:1016F0000001003000000030000000300001002F29
:101700000000002F0000002F0000002F0001002E1D
:101710000000002E0000002E0001002D0000002D12
:101720000000002D0000002D0001002C0000002C06
:101730000000002C0000002C0001002B0000002BFA
:101740000000002B0000002B0001002A0000002AEE
:101750000000002A0000002A0001002900000029E2
:1017600000000029000000290000002900010028D5
:1017700000000028000000280000002800000028C9
:1017800000010027000000270000002700000027BC
:1017900000000027000100260000002600000026AF
:1017A00000000026000000260001002500000025A2
:1017B0000000002500000025000000250000002595
:1017C0000001002400000024000000240000002488
:1017D000000000240001002300000023000000237B
:1017E000000000230000002300000023000000236D
:1017F0000001002200000022000000220000002260
:101800000000002200000022000100210000002151
:101810000000002100000021000000210000002144
:101820000000002100010020000000200000002036
:101830000000002000000020000000200000002028
:10184000000000200001001F0000001F0000001F1A
:101850000000001F0000001F0000001F0000001F0C
:101860000001001E0000001E0000001E0000001EFF
:101870000000004D494E54454D5020747269676711
:1018800065726564004572723A204D494E54454D6B
:101890005020424544004D415854454D50207472EB
:1018A00069676765726564004572723A204D4158F8
:1018B00054454D5020424544004572723A204D49EE
:1018C0004E54454D50004D494E54454D5020747274
:1018D00069676765726564004572723A204D494ECA
:1018E00054454D50004572723A204D494E54454D75
:1018F00050004572723A204D415854454D500045B4
:1019000072723A204D494E54454D50004572723A1C
:10191000204D415854454D5000626564002C2073A1
:10192000797374656D2073746F70706564212048DD
:1019300065617465725F49443A20004572723A20CD
:101940004D415854454D50004D415854454D50203F
:10195000747269676765726564004572723A204DFA
:10196000415854454D50004B64200023646566691E
:101970006E65202044454641554C545F004B69201C
:101980000023646566696E65202044454641554CD8
:10199000545F004B70200023646566696E652020EB
:1019A00044454641554C545F0050494420417574AC
:1019B0006F74756E652066696E6973686564212051
:1019C00050757420746865206C617374204B702CA2
:1019D000204B6920616E64204B6420636F6E7374CA
:1019E000616E74732066726F6D2062656C6F772014
:1019F000696E746F20436F6E666967757261746992
:101A00006F6E2E6800504944204175746F74756E76
:101A100065206661696C6564212074696D656F7508
:101A2000740020403A00543A00423A0050494420A1
:101A30004175746F74756E65206661696C656421AB
:101A40002054656D706572617475726520746F6F76
:101A5000206869676800204B643A2000204B693A8F
:101A60002000204B703A200020436C61737369633F
:101A70002050494420002054753A2000204B753AEC
:101A80002000206D61783A2000206D696E3A2000B8
:101A900020643A200020626961733A200070012CB2
:101AA0000190012701B0012201C0011D01F00118C0
:101AB000011002130130020E0160020901900204BC
:101AC00001C002FF000003FA004003F5008003F0AC
:101AD00000D003EB002004E6007004E100E004DC29
:101AE000004005D700C005D2004006CD00D006C892
:101AF000008007C3003008BE00F008B900C009B478
:101B000000B00AAF00B00BAA00D00CA500000EA0D8
:101B100000500F9B00C01096005012910000148CD2
:101B200000C0158700B0178200B0197D00D01B7867
:101B300000001E730040206E0090226900F02464B3
:101B40000040275F0090295A00E02B5500102E50CE
:101B50000020304B0010324600E033410090353C0D
:101B6000001037370070383200A0392D00B03A2805
:101B700000A03B2300603C1E00103D1900903D1466
:101B800000103E0F00703E0A00C03E0500003F00FE
:101B900000436172642072656D6F76656400436115
:101BA000726420696E736572746564002D2D3A2D20
:101BB0002D002D2D2D005344005A200020590001E6
:101BC0002000012000466C6F7700466C6F7700465E
:101BD000616E2073706565640046616E2073706588
:101BE00065640042656400426564004E6F7A7A6CF9
:101BF00065004E6F7A7A6C650053706565640053BA
:101C000070656564004D61696E004D6F76652058A2
:101C1000004D6F76652059004D6F7665205A00455E
:101C20007874727564657200457874727564657253
:101C3000004D6F7665205A004D6F76652059004D36
:101C40006F76652058004D6F766520617869730066
:101C50004D6F766520302E316D6D004D6F766520AD
:101C6000316D6D004D6F76652031306D6D005072B5
:101C70006570617265005072656865617420504CD2
:101C80004120426564005072656865617420504C63
:101C900041005072657061726500507265686561DF
:101CA000742041425320426564005072656865614A
:101CB0007420414253005072657061726500436F39
:101CC0006F6C646F776E0050726568656174204157
:101CD0004253005072656865617420504C41004D5C
:101CE00038340044697361626C6520737465707088
:101CF000657273004D6F76652061786973004732B5
:101D000039004C6576656C206265640047323800A6
:101D10004175746F20686F6D65004D61696E004696
:101D2000616E2073706565640046616E2073706536
:101D300065640042656400426564004E6F7A7A6CA7
:101D400065004E6F7A7A6C6500436F6E74726F6CCB
:101D500000526573746F7265206661696C736166A9
:101D6000650054656D7065726174757265004D61D2
:101D7000696E004D383400473238205830205930D1
:101D800000473238205830205930004D313039204A
:101D90005325692E67004D313430205325692E6755
:101DA000004D3234004D323320257300052E2E00B5
:101DB0004D61696E004E6F20534420636172640070
:101DC0005072696E742066726F6D205344005374B4
:101DD0006F70207072696E7400526573756D652046
:101DE0007072696E74005061757365207072696EEF
:101DF0007400436F6E74726F6C0050726570617224
:101E0000650054756E6500496E666F207363726578
:101E1000656E00207A3A200020793A200020783A36
:101E2000200000000A0B02090C0D0E080703040134
:101E300000000000000000000000000000000000A2
:101E4000000000000000000000000000000012116F
:101E50001000000000000000000000000000000072
:101E600000000000000000000102102020080810FF
:101E700020401020408002010201080402010102FA
:101E800004081020408080402010080402018004D3
:101E9000020180402010080402010804020101022E
:101EA000040810204080010204081020408005052D
:101EB0000505070508080808020202020A0A0808C0
:101EC00004040404010101010101010103030303EE
:101ED00003030303040707070C0C0C0C0C0C0C0C7D
:101EE0000202020206060606060606060B0B0B0B8E
:101EF0000B0B0B0B000020002300260029002C00F8
:101F00002F0032000001000003010601090100005A
:101F10002200250028002B002E0031003400020191
:101F20000000050108010B0100002100240027002A
:101F30002A002D00300033000101000004010701D8
:101F40000A014E414E494E495459494E46CDCCCCDA
:101F50003D0AD7233C17B7D13877CC2B329595E67D
:101F6000241FB14F0A000020410000C84200401C5D
:101F70004620BCBE4CCA1B0E5AAEC59D7400005C08
:101F800030AE86C4045C11241FBECFEFD1E2DEBFA9
:101F9000CDBF00E00CBF14E0A0E0B2E0EAECFBEA49
:101FA00001E00BBF02C007900D92AC3BB107D9F71F
:101FB00023E1ACEBB4E001C01D92A03FB207E1F712
:101FC0001FE1C4E8DFE100E006C022970109FE013D
:101FD0000BBF0E94A6CFCE37D10780E00807A9F734
:101FE0000E9453CA0C94D4D50C940000452B31F0B8
:101FF000389A409A0E9414C8409808950C9414C8C6
:10200000FC0114821782138212828DE294E0918384
:10201000808308952DE234E0FC0131832083278101
:10202000222319F004960C94A4870895CF92DF928E
:10203000EF92FF920F931F93CF93DF93EC018F9654
:10204000DFDFCE01805B9F4FDBDF7E012FE6E20EFC
:10205000F11C87016E013BE5C31A3EEFD30AC801AC
:10206000CFDF015E1F4F0C151D05C9F7FE01E955B5
:10207000FE4F89E1818314823596178ACE018653FB
:102080009E4FBEDFFE01E558FD4F10821182128285
:102090001382389610821182128213821A821B8256
:1020A00018821982F80111821082FE01E751FE4F59
:1020B000108286E391E0F7019C011192215030409B
:1020C000E1F7FE01E957FD4F81E080831EA61DA6C2
:1020D0000E94E5C7C158DD4F68577C4E8F4F9F4F18
:1020E000688379838A839B83DF91CF911F910F91BE
:1020F000FF90EF90DF90CF900895FC0120E03EE24A
:10210000DB014C91403241F0283011F4308331969C
:10211000DB014C91408331962F5F6F5F7F4F2B30F7
:1021200079F7108208952F923F924F925F926F92AB
:102130007F928F929F92AF92BF92CF92DF92EF9257
:10214000FF920F931F93CF93DF93CDB7DEB7C657A0
:10215000D1090FB6F894DEBF0FBECDBF8C016B0165
:102160005A0129012DB73EB7E3963FAF2EAFE39753
:10217000AD961FAEAD9734E0A30EB11C4296E59626
:102180009FAF8EAFE597180198E7291A9DEF390A9E
:10219000F801E657FD4FAF96FFAFEEAFAF973801AE
:1021A000F5E06F0E711C7E012FE5E20EF11C80E45C
:1021B00090E08C0F9D1F0496E7969FAF8EAFE79738
:1021C000E5964EAD5FADE597BE016F5F7F4FC501F0
:1021D0000E940A8618160CF03EC12C85322F3871E9
:1021E000303109F0BCC0F1018081918101970297E3
:1021F00008F4B5C02DB73EB7E1963FAF2EAFE197DB
:10220000BE016F5F7F4FC70178DF81E0F6019081EB
:1022100091119DC0E1E0F0E0D7010D900020E9F7B9
:10222000EE19FF09EA0FFB1F31962DB73EB72E1BA3
:102230003F0B0FB6F8943EBF0FBE2DBFEDB7FEB7F4
:1022400031964F01882319F06BE373E001C0B601AA
:10225000C4010E94EBD2B701C4010E94CCD26BE34F
:1022600073E0C4010E94CCD2CE01805C9F4FC8DED7
:1022700021E0A701B501E7968EAD9FADE7970E94DB
:102280009B89811137C0F10180819181892B91F562
:10229000E7ECFFE08491882341F09091C00095FF26
:1022A000FCCF8093C6003196F5CFEDE3F3E081914A
:1022B000882339F09091C00095FFFCCF8093C60031
:1022C000F6CF8091C00085FFFCCF8AE08093C600E6
:1022D000F7018191882339F09091C00095FFFCCFE0
:1022E0008093C600F6CF8091C00085FFFCCF8AE0C6
:1022F0008093C6008BE1FE01EC5BFF4FDE019596FB
:1023000001900D928A95E1F724968EAD9FAD2497AA
:102310009CA38BA38DE294E09AA389A320E030E0F4
:10232000AE014F5D5F4FB401C801FDDECE01819665
:1023300071DECE01805C9F4F6DDEE1962EAD3FAD2C
:10234000E1970FB6F8943EBF0FBE2DBF39CF80E0A6
:1023500001900020E9F73197EC19FD095DCF8981E3
:10236000882309F478C08E3209F42ACFF8018289D3
:102370008E3209F425CF23FD23CF81E0303109F0DF
:1023800080E0F8018483811108C08985873409F0D1
:1023900017CF8A858E3709F413CFF101808191819F
:1023A0008130910569F08230910581F1892B09F026
:1023B00007CFBE016F5F7F4FC3019FDEF60110C0E4
:1023C000AF96EEADFFADAF9780819181019691837D
:1023D0008083F6CE9091C00095FFFCCF8093C6001D
:1023E00081918111F7CFF3018191882339F0909188
:1023F000C00095FFFCCF8093C600F6CF8091C0004F
:1024000085FFFCCF8AE08093C600DACEBE016F5F05
:102410007F4FC30172DE4114510439F0B301C20190
:102420000E94B9D2892B79F416C0AD96FFADAD9755
:102430002F2F30E0AF96EEADFFADAF978081918149
:102440002817390741F0AD96FFADAD97FF5FAD9608
:10245000FFAFAD97B5CEE3962EAD3FADE3970FB688
:10246000F8943EBF0FBE2DBFCA58DF4F0FB6F89489
:10247000DEBF0FBECDBFDF91CF911F910F91FF90B7
:10248000EF90DF90CF90BF90AF909F908F907F9014
:102490006F905F904F903F902F900895EF92FF9232
:1024A0000F931F93CF93DF93CDB7DEB76F970FB620
:1024B000F894DEBF0FBECDBF8C01FC01E857FD4F85
:1024C000118210827C0183E3E80EF11C40E050E0B1
:1024D000BA01C7010E94C1868BE1F701DE011596A2
:1024E00001900D928A95E1F7F80181A992A99C8348
:1024F0008B838DE294E09A83898320E030E0AE0103
:102500004F5F5F4F64E474E0C8010DDECE010196B9
:1025100081DD6F960FB6F894DEBF0FBECDBFDF91A1
:10252000CF911F910F91FF90EF9008952BE1FB0148
:102530003496DC01149601900D922A95E1F7FB0187
:1025400022813381FC01338322830895EF92FF922D
:102550000F931F93CF93DF93EC011B828EA98823E7
:1025600021F0CE01C3960E94A4877E0189E5E81A76
:102570008EEFF80A45E360E0C7010E9421828111D5
:102580001FC0E7ECFFE08491882341F09091C000E8
:1025900095FFFCCF8093C6003196F5CFE8E7F3E0D6
:1025A0008491882341F09091C00095FFFCCF8093E7
:1025B000C6003196F5CF8091C00085FFFCCF76C074
:1025C0008E0104551E4F41E0B701C8010E94A58F3E
:1025D000811126C040E0B701C8010E94A58F81117A
:1025E0001FC0EDECFFE08491882341F09091C00082
:1025F00095FFFCCF8093C6003196F5CFE5E6F3E07A
:102600008491882341F09091C00095FFFCCF809386
:10261000C6003196F5CF8091C00085FFFCCF46C043
:10262000B801CE01C3960E94AE8481111FC0EDECAB
:10263000FFE08491882341F09091C00095FFFCCF8A
:102640008093C6003196F5CFE5E5F3E084918823C9
:1026500041F09091C00095FFFCCF8093C600319669
:10266000F5CF8091C00085FFFCCF20C081E08B8337
:10267000E7ECFFE08491882341F09091C00095FF42
:10268000FCCF8093C6003196F5CFEAE4F3E0849165
:10269000882341F09091C00095FFFCCF8093C60045
:1026A0003196F5CF8091C00085FFFCCF8AE0809302
:1026B000C6008E01015D1F4FB801CE01805B9F4FA8
:1026C00035DFC25BDF4F19830883DF91CF911F9104
:1026D0000F91FF90EF900895FC01128213820895EC
:1026E000FC012381222311F021E022830895FC01C3
:1026F0002281211112820895AF92BF92CF92DF9270
:10270000EF92FF920F931F93CF93DF931F92CDB75A
:10271000DEB78C018FE2FB0181935F01D12C41E098
:102720007801FBE5EF1AFEEFFF0A8FE1C82E2D2D91
:1027300030E0F7018081918128173907D8F4C29ED3
:10274000C001C39E900D11248D589F4FB501800F7D
:10275000911F49830E945584C50149815C010196FE
:10276000F5012081222321F04D3810F44F5FF6CF80
:10277000D394DDCF47FD11C0B501C80182539E4FF0
:102780000F90DF91CF911F910F91FF90EF90DF900D
:10279000CF90BF90AF900C945584F50110820F90AC
:1027A000DF91CF911F910F91FF90EF90DF90CF902D
:1027B000BF90AF9008953F924F925F926F927F9239
:1027C0008F929F92AF92BF92CF92DF92EF92FF9241
:1027D0000F931F93CF93DF93CDB7DEB7AC970FB6B0
:1027E000F894DEBF0FBECDBF7C015B01FC0183818D
:1027F000882309F4EDC0C70182539E4F0E94A4872D
:10280000F7011282CE0101966C01FADB27019EE4EA
:10281000490E511CC7018F96F20191838083F50107
:1028200080818F3209F077C06FE270E0C5010E94AD
:10283000D7D28C010F5F1F4F9AE0392E0115110579
:1028400009F46FC06FE270E0C8010E94D7D24C015A
:10285000009709F467C00817190708F063C03C0126
:10286000601A710AA301B801CE0180960E9400D3BC
:10287000E0E2F0E0EC0FFD1FE60DF71D1082FE0117
:10288000B0968191882339F09091C00095FFFCCFDC
:102890008093C600F6CF8091C00085FFFCCF3092B8
:1028A000C600F201608171816115710519F06C5FDC
:1028B0007F4F02C060E070E021E0AE01405E5F4FFC
:1028C000CE0105960E949B8981111EC0E6E2F2E0CE
:1028D0008491882341F09091C00095FFFCCF8093B4
:1028E000C6003196F5CFFE01B0968191882339F06C
:1028F0009091C00095FFFCCF8093C600F6CF8091E9
:10290000C00085FFFCCF5FC0F201D182C08284018C
:102910000F5F1F4F93CFC701805B9F4FF2019183E1
:1029200080838501F20180819181009711F00496E6
:1029300002C080E090E0B8010E94718A811103C05A
:10294000E0E0F2E02EC0E8E1F2E08491882341F07B
:102950009091C00095FFFCCF8093C6003196F5CFD3
:10296000F8018191882339F09091C00095FFFCCF48
:102970008093C600F6CF8091C00085FFFCCF8AE02F
:102980008093C600F701ED57FD4F1082118212822D
:1029900013821CC09091C00095FFFCCF8093C600AD
:1029A000319684918111F6CFF8018191882339F015
:1029B0009091C00095FFFCCF8093C600F6CF809128
:1029C000C00085FFFCCF8EE28093C600C60122DBEB
:1029D000AC960FB6F894DEBF0FBECDBFDF91CF919E
:1029E0001F910F91FF90EF90DF90CF90BF90AF902D
:1029F0009F908F907F906F905F904F903F90089541
:102A0000CF93DF93EC018B81811103C0EEEDF1E0F8
:102A100039C0EEEEF1E08491882341F09091C0003E
:102A200095FFFCCF8093C6003196F5CFFE01ED57A0
:102A3000FD4F40815181628173812AE030E08CEB4F
:102A400094E00E9418238091C00085FFFCCF8FE2A4
:102A50008093C600C558DD4F488159816A817B81CA
:102A60002AE030E08CEB94E00E9418238091C000B3
:102A700085FFFCCF0EC09091C00095FFFCCF8093E6
:102A8000C600319684918111F6CF8091C00085FFF8
:102A9000FCCF8AE08093C600DF91CF910895AF927A
:102AA000BF92CF92DF92EF92FF920F931F93CF933B
:102AB000DF935C01EB01FB0101900020E9F78F013E
:102AC00001501109061B170B6C01F2E3CF1AFEEF40
:102AD000DF0AF60110826EE470E0CE010E94D7D2C8
:102AE0007C01009729F4F8013197EC0FFD1F0DC010
:102AF00060E270E00E94D7D2EC0121966AE270E0B9
:102B0000C7010E94D7D2FC0131978DE081838AE012
:102B100082831382BE01C50186539E4F0E944E8C54
:102B2000F6018081882309F1EDECFFE08491882390
:102B300041F09091C00095FFFCCF8093C600319684
:102B4000F5CFE8ECF1E08491882341F09091C0004A
:102B500095FFFCCF8093C6003196F5CF8091C000E1
:102B600085FFFCCF8AE08093C600DF91CF911F9153
:102B70000F91FF90EF90DF90CF90BF90AF900895AE
:102B80002F923F924F925F926F927F928F929F927D
:102B9000AF92BF92CF92DF92EF92FF920F931F936B
:102BA000CF93DF93CDB7DEB7CC5BD1090FB6F894E6
:102BB000DEBF0FBECDBF8C0189579D4F5C016111F7
:102BC00012C0FC018081882309F4B1C03897C0800D
:102BD000D180E280F3800E94E5C7C616D706E806DA
:102BE000F90608F4A4C0F5011082F801838181116F
:102BF00007C0C801ABDCF8018381882309F497C0C2
:102C0000F80186A58F9385A58F938FEB91E09F9315
:102C10008F937E01F3EBEF0EF11CFF92EF920E9477
:102C20000FD30F900F900F900F900F900F90B12C2B
:102C3000F70101900020E9F73197EE19FF09BE1660
:102C400084F46701CB0CD11CB7FCDA94F6018081C7
:102C5000992787FD90950E945AD2F6018083B394FC
:102C6000E7CF4801F3E38F0E911C40E050E0BA013A
:102C7000C4010E94C186512C6E0183E9C80ED11C8B
:102C800028EB622E21E0722EFE0131965F0140E0BA
:102C900050E0B601C4010E940A861816E4F5412CE2
:102CA000F60101900020E9F73197EC19FD094E1665
:102CB00074F41601240C311C47FC3A94F101808114
:102CC00090E00E945AD2F10180834394E9CFF6014B
:102CD00081858E37E1F245E050E0B701C6010E94E0
:102CE000F2D2892BA1F6FF92EF927F926F92BF9260
:102CF000AF920E940FD3C5010E94522484EB91E051
:102D00000E941B250F900F900F900F900F900F9027
:102D100055245394BCCF511004C08FEF9FEFF8019E
:102D200004C0F80185A596A5019696A785A7C45469
:102D3000DF4F0FB6F894DEBF0FBECDBFDF91CF914E
:102D40001F910F91FF90EF90DF90CF90BF90AF90C9
:102D50009F908F907F906F905F904F903F902F90BB
:102D600008950F931F93CF93DF93EC018C010253CF
:102D70001E4FC8010E945A87C8010E94A487198269
:102D80001882DF91CF911F910F910895CF92DF921A
:102D9000EF92FF920F931F93CF93DF93CDB7DEB7E0
:102DA0006F970FB6F894DEBF0FBECDBF8C016A01DE
:102DB0007C018EE4E80EF11CC801805B9F4FF70197
:102DC00091838083E65CFD4F22E030E031832083F5
:102DD00032967183608340E050E0BA0104960E940D
:102DE000C186F701808191812BE1FC013496DE01DF
:102DF000159601900D922A95E1F7FC01828193814D
:102E00009C838B838DE294E09A8389839601AE0143
:102E10004F5F5F4F64E474E0C80185D9CE0101962D
:102E2000F9D86F960FB6F894DEBF0FBECDBFDF9115
:102E3000CF911F910F91FF90EF90DF90CF90089569
:102E40002F923F924F925F926F927F928F929F92BA
:102E5000AF92BF92CF92DF92EF92FF920F931F93A8
:102E6000CF93DF93CDB7DEB7AC970FB6F894DEBF44
:102E70000FBECDBF8C016B01342EFC0183818823F2
:102E800009F4CDC2EF52FE4F8081882309F4FAC0C5
:102E9000222319F0E7ECFFE0CDC07801F7E1EF1A4B
:102EA000FEEFFF0AF7018081811103C0E7ECFFE02C
:102EB00035C0EDECFFE08491882341F09091C00093
:102EC00095FFFCCF8093C6003196F5CFE7E0F3E0A5
:102ED0008491882341F09091C00095FFFCCF8093AE
:102EE000C6003196F5CF4AE050E061E070E08CEB2F
:102EF00094E00E94EC228091C00085FFFCCF8AE024
:102F00008093C6008EEF92E00E94204488C2909188
:102F1000C00095FFFCCF8093C6003196849181114B
:102F2000F6CFE5EEF2E08491882341F09091C00065
:102F300095FFFCCF8093C6003196F5CFF6018191C5
:102F4000882339F09091C00095FFFCCF8093C60094
:102F5000F6CFEAEDF2E08491882341F09091C00031
:102F600095FFFCCF8093C6003196F5CFF7018081A5
:102F70004DE8B42EB801B89E600D711D1124625148
:102F80007E4FC801B9DBF7018081F801B89EE00DE2
:102F9000F11D1124E251FE4F8191882339F0909167
:102FA000C00095FFFCCF8093C600F6CFE4EDF2E0C1
:102FB0008491882341F09091C00095FFFCCF8093CD
:102FC000C6003196F5CF5801FDE7AF1AFDEFBF0AF5
:102FD000F50140815181628173812AE030E08CEB00
:102FE00094E00E9418238091C00085FFFCCF8AE006
:102FF0008093C600F7012081F80184E0289FE00D4E
:10300000F11D1124AF0146515E4FF5018081918180
:10301000A281B381FA0180839183A283B3832F5F5E
:10302000F701208329C09091C00095FFFCCF8093C9
:10303000C600319684918111F6CFE3ECF2E08491E1
:10304000882341F09091C00095FFFCCF8093C6008B
:103050003196F5CFF6018191882339F09091C00027
:1030600095FFFCCF8093C600F6CF8091C00085FF0E
:10307000FCCF8AE08093C600C80182539E4F0E9415
:10308000A48730C0F801E751FE4F1082E7ECFFE063
:103090008491882341F09091C00095FFFCCF8093EC
:1030A000C6003196F5CFE2EBF2E08491882341F03F
:1030B0009091C00095FFFCCF8093C6003196F5CF6C
:1030C000F6018191882339F09091C00095FFFCCFE3
:1030D0008093C600F6CF8091C00085FFFCCF8AE0C8
:1030E0008093C600F8011282CE0101965C010E9415
:1030F000001028019EE4490E511CC8018F96F20170
:1031000091838083F60180818F3209F077C0760148
:10311000FFEFEF1AFF0A3AE0232EE114F10409F45D
:1031200073C06FE270E0C7010E94D7D24C010097D4
:1031300009F46BC0E816F90608F067C03C016E1888
:103140007F08A301B701CE0180960E9400D3E0E280
:10315000F0E0EC0FFD1FE60DF71D1082FE01B096AA
:103160008191882339F09091C00095FFFCCF809326
:10317000C600F6CF8091C00085FFFCCF2092C6002C
:10318000F201608171816115710519F06C5F7F4FEB
:1031900002C060E070E021E0AE01405E5F4FCE0112
:1031A00005960E949B89811121C0EEE9F2E084918D
:1031B000882341F09091C00095FFFCCF8093C6001A
:1031C0003196F5CFFE01B0968191882339F0909128
:1031D000C00095FFFCCF8093C600F6CF8091C00061
:1031E00085FFFCCF8EE28093C60016C1F201B1824A
:1031F000A0827401FFEFEF1AFF0A8FCFC801805B36
:103200009F4FF201918380837601C80182539E4FC4
:103210004C01F20160817181332009F4A3C0611572
:10322000710519F06C5F7F4F02C060E070E021E033
:10323000A701C4010E949B89811103C0E6E6F2E068
:1032400075C0980125583D4FF40181899289A38961
:10325000B489F90180839183A283B383E0E9F2E02A
:103260008491882341F09091C00095FFFCCF80931A
:10327000C6003196F5CFF7018191882339F09091FE
:10328000C00095FFFCCF8093C600F6CFE8E8F2E0DF
:103290008491882341F09091C00095FFFCCF8093EA
:1032A000C6003196F5CFF901408151816281738169
:1032B0002AE030E08CEB94E00E9418238091C0005B
:1032C00085FFFCCF8AE08093C600F801ED57FD4FE3
:1032D0001082118212821382EAE7F2E0849188233D
:1032E00041F09091C00095FFFCCF8093C6003196CD
:1032F000F5CF8091C00085FFFCCF8AE08093C600A7
:10330000A70160E070E0C80141DDF80182898823EF
:1033100019F0C801429601C0C70160E07BC09091DE
:10332000C00095FFFCCF8093C60031968491811137
:10333000F6CFF7018191882339F09091C00095FF75
:10334000FCCF8093C600F6CFE3E6F2E084918823B9
:1033500009F462C09091C00095FFFCCF8093C60035
:103360003196F4CF6115710519F06C5F7F4F02C083
:1033700060E070E026E5A701C4010E949B898111ED
:1033800025C0EFE4F2E08491882341F09091C000E1
:1033900095FFFCCF8093C6003196F5CFF701819160
:1033A000882339F09091C00095FFFCCF8093C60030
:1033B000F6CFECE4F2E08491882371F19091C000A3
:1033C00095FFFCCF8093C6003196F5CF81E0F801E0
:1033D0008083EAE3F2E08491882341F09091C00079
:1033E00095FFFCCF8093C6003196F5CFF601819111
:1033F000882339F09091C00095FFFCCF8093C600E0
:10340000F6CF8091C00085FFFCCF8AE08093C60094
:1034100060E0C7010E94AFA9C5010E940A10AC96E6
:103420000FB6F894DEBF0FBECDBFDF91CF911F91D5
:103430000F91FF90EF90DF90CF90BF90AF909F9053
:103440008F907F906F905F904F903F902F90089556
:1034500021E0FC01218340E0F3CCCF92DF92EF9298
:10346000FF920F931F93CF93DF93CDB7DEB76F9784
:103470000FB6F894DEBF0FBECDBF8C016C012EE4F9
:10348000C20ED11C805B9F4FF60191838083E65C66
:10349000FD4F21E030E0318320837801F6E7EF1A19
:1034A000FDEFFF0AF7011182108240E050E0BA01FF
:1034B00004960E94C186F601808191812BE1FC0176
:1034C0003496DE01159601900D922A95E1F7FC01E4
:1034D000828193819C838B838DE294E09A8389839C
:1034E00020E030E0AE014F5F5F4F64E474E0C8015C
:1034F0000E949310CE0101960E940A10F70180816C
:1035000091816F960FB6F894DEBF0FBECDBFDF91ED
:10351000CF911F910F91FF90EF90DF90CF90089582
:10352000AF92BF92CF92DF92EF92FF920F931F93D1
:10353000CF93DF93CDB7DEB76F970FB6F894DEBFAA
:103540000FBECDBF8C017B01CE0101960E94001001
:10355000F801E95AFF4F80816801811104C02FE210
:10356000C20ED11C03C080E5C80ED11C21E0A7010A
:10357000B6016C5F7F4FCE0105960E949B89811139
:103580002DC0E7ECFFE08491882341F09091C000CA
:1035900095FFFCCF8093C6003196F5CFEEE9F1E0C0
:1035A0008491882341F09091C00095FFFCCF8093D7
:1035B000C6003196F5CFF7018191882339F09091BB
:1035C000C00095FFFCCF8093C600F6CF8091C0006D
:1035D00085FFFCCF8AE08093C60036C0F801EB552A
:1035E000FE4F808191818A30910530F59C012F5FDB
:1035F0003F4F318320832FE1289F7001299FF00CDA
:1036000011242FE6E20EF11CE00EF11E5C01B70161
:10361000C7014F960E94961281E0A81AB1082FE1C7
:10362000E21AF1088FEFA816B80689F7B601C801AB
:1036300081599F4F0E949612BE016F5F7F4FC80154
:10364000805B9F4F0E949612CE0101960E940A1045
:103650006F960FB6F894DEBF0FBECDBFDF91CF914E
:103660001F910F91FF90EF90DF90CF90BF90AF90A0
:103670000895EF92FF920F931F93CF93DF93EC0186
:10368000CB55DE4F2881398121153105F9F02150C4
:103690003109398328838C0101591F4FB801805BA0
:1036A0009F4F0E949612C80100E010E07C012FE1BC
:1036B000E20EF11C288139810217130738F40F5FDD
:1036C0001F4FB7010E949612C701F0CFDF91CF9133
:1036D0001F910F91FF90EF900895EF92FF920F933B
:1036E0001F93CF93DF93EC010E948D998E010751B8
:1036F0001E4FF80180819E0122533E4F790188239D
:10370000A1F1C9010E94A487F801808181508083C2
:10371000BE01FDE88F9F600D711D112462517E4F27
:1037200021E041E0CE018CDBF8018081FE0124E044
:10373000829FE00DF11D1124E651FE4F4081518121
:1037400062817381FE01ED57FD4F40835183628397
:103750007383C7010E94C186CE01DF91CF911F9173
:103760000F91FF90EF900C947013C9010E94A487F1
:103770001A8282E991E00E941B258091C80E88235D
:10378000F9F01092C80EC0916605D0E0CC0FDD1F95
:10379000C854DD4E68817981882777FD8095982F00
:1037A0000E9423CC20913B0230913C0240913D028B
:1037B00050913E020E9484CD181614F4198218828A
:1037C000DF91CF911F910F91FF90EF900895AF92ED
:1037D000BF92DF92EF92FF920F931F93CF93DF93ED
:1037E000CDB7DEB7E0970FB6F894DEBF0FBECDBF02
:1037F00080E1E5ECF2E0DE01919601900D928A9570
:10380000E1F780E1E5EDF2E0DE01519601900D92E5
:103810008A95E1F780E1E5EEF2E0DE011196019094
:103820000D928A95E1F77E0181E2E80EF11C09E034
:103830001FE0BE016F5E7F4F49E15FE09E012F5F99
:103840003F4F99EFA92E9EE0B92ED12CF70181911F
:103850009191A191B1917F01F80181939193A193ED
:10386000B1938F01FB0181919191A191B191BF0120
:10387000FA0181939193A193B193AF01F9018191E1
:103880009191A191B1919F01F50181939193A193A0
:10389000B1935F01D394F4E0DF12D8CF0E946F6F31
:1038A00080E090E0AAEFB3E48093F10E9093F20EE3
:1038B000A093F30EB093F40E8093ED0E9093EE0E62
:1038C000A093EF0EB093F00E80E090E0AAE7B4E48E
:1038D0008093E90E9093EA0EA093EB0EB093EC0E5A
:1038E0001092F50E1092F60E1092F70E1092F80E3E
:1038F00080E29EE4A0E0B0E08093290F90932A0F2D
:10390000A0932B0FB0932C0F1092D90E1092DA0EB9
:103910001092DB0E1092DC0E80E090E0A0EAB1E4A1
:103920008093E50E9093E60EA093E70EB093E80E19
:103930008DEC9CECACECBEE38093E10E9093E20E38
:10394000A093E30EB093E40E80E090E0A0EAB0E430
:103950008093DD0E9093DE0EA093DF0EB093E00E09
:1039600010927B0510927C0510927D0510927E05C9
:1039700010927705109278051092790510927A05C9
:1039800010927305109274051092750510927605C9
:103990008DEC9CECACE4BEEB80930E0290930F0296
:1039A000A0931002B093110289EB90E090931B1347
:1039B00080931A138DE290E090931913809318135B
:1039C000109217131092161380EF90E09093151336
:1039D000809314138CE390E090931313809312134D
:1039E00010921113109210138AE999E9A1EBB1E436
:1039F0008093810290938202A0938302B093840209
:103A000061E77DE38AE89FE30E949EA660937D02C2
:103A100070937E0280937F029093800260E070E05A
:103A200084EE92E40E94AAA66093790270937A02CF
:103A300080937B0290937C0280E090E0A8ECB2E45B
:103A40008093750290937602A0937702B0937802E8
:103A500084E190E090930B0280930A020E94949B71
:103A600010927F0580E090E0A0E4B0E4809329020A
:103A700090932A02A0932B02B0932C020E948156AD
:103A8000E7ECFFE08491882341F09091C00095FF1E
:103A9000FCCF8093C6003196F5CFE0EEF5E084913F
:103AA000882341F09091C00095FFFCCF8093C60021
:103AB0003196F5CF8091C00085FFFCCF8AE08093DE
:103AC000C600E0960FB6F894DEBF0FBECDBFDF9103
:103AD000CF911F910F91FF90EF90DF90BF90AF902B
:103AE0000895CF93C82F882369F14091090F509111
:103AF0000A0F60910B0F70910C0F88EC95E09FD628
:103B000040910D0F50910E0F60910F0F7091100F9B
:103B100085EC95E094D64091110F5091120F609171
:103B2000130F7091140F82EC95E089D64091150F18
:103B30005091160F6091170F7091180F8FEB95E051
:103B40007ED62FC0E7ECFFE08491882341F090916E
:103B5000C00095FFFCCF8093C6003196F5CFE0ED15
:103B6000F5E08491882341F09091C00095FFFCCF4F
:103B70008093C6003196F5CF8091C00085FFFCCFC1
:103B80008AE08093C600E7ECFFE08491882309F483
:103B9000ACCF9091C00095FFFCCF8093C6003196CA
:103BA000F4CF8091C00085FFFCCF8AE08093C600EF
:103BB000CC2369F14091190F50911A0F60911B0F9E
:103BC00070911C0F8CE995E03AD640911D0F5091F1
:103BD0001E0F60911F0F7091200F89E995E02FD67D
:103BE0004091210F5091220F6091230F7091240F6B
:103BF00086E995E024D64091250F5091260F6091DB
:103C0000270F7091280F83E995E019D62FC0E7ECB4
:103C1000FFE08491882341F09091C00095FFFCCF94
:103C20008093C6003196F5CFE5EAF5E084918823CC
:103C300041F09091C00095FFFCCF8093C600319673
:103C4000F5CF8091C00085FFFCCF8AE08093C6004D
:103C5000E7ECFFE08491882309F4ACCF9091C00099
:103C600095FFFCCF8093C6003196F4CF8091C000C1
:103C700085FFFCCF8AE08093C600CC2369F1409198
:103C8000F90E5091FA0E6091FB0E7091FC0E8CE6CD
:103C900095E0F7D54091FD0E5091FE0E6091FF0E1C
:103CA0007091000F89E695E0ECD54091010F50919D
:103CB000020F6091030F7091040F86E695E0E1D545
:103CC0004091050F5091060F6091070F7091080FFA
:103CD00083E695E0D6D52FC0E7ECFFE084918823FA
:103CE00041F09091C00095FFFCCF8093C6003196C3
:103CF000F5CFE5E7F5E08491882341F09091C0008D
:103D000095FFFCCF8093C6003196F5CF8091C0001F
:103D100085FFFCCF8AE08093C600E7ECFFE084914A
:103D2000882309F4ACCF9091C00095FFFCCF80931D
:103D3000C6003196F4CF8091C00085FFFCCF8AE0A9
:103D40008093C600CC2311F14091F10E5091F20EF8
:103D50006091F30E7091F40E88E295E070D5409179
:103D6000ED0E5091EE0E6091EF0E7091F00E85E227
:103D700095E065D54091E90E5091EA0E6091EB0E09
:103D80007091EC0E82E295E05AD52FC0E7ECFFE08F
:103D90008491882341F09091C00095FFFCCF8093DF
:103DA000C6003196F5CFE1E3F5E08491882341F038
:103DB0009091C00095FFFCCF8093C6003196F5CF5F
:103DC0008091C00085FFFCCF8AE08093C600E7ECBD
:103DD000FFE08491882309F4B7CF9091C00095FF4C
:103DE000FCCF8093C6003196F4CF8091C00085FF50
:103DF000FCCF8AE08093C600CC2309F443C04091F5
:103E0000F50E5091F60E6091F70E7091F80E86E661
:103E100094E015D54091D90E5091DA0E6091DB0EE9
:103E20007091DC0E83E694E00AD54091290F509101
:103E30002A0F60912B0F70912C0F80E694E021D512
:103E40004091E50E5091E60E6091E70E7091E80EFC
:103E50008DE594E0F4D44091E10E5091E20E609132
:103E6000E30E7091E40E8AE594E0E9D44091DD0E12
:103E70005091DE0E6091DF0E7091E00E87E594E0C8
:103E8000DED42FC0E7ECFFE08491882341F09091CD
:103E9000C00095FFFCCF8093C6003196F5CFEFE6CA
:103EA000F4E08491882341F09091C00095FFFCCF0D
:103EB0008093C6003196F5CF8091C00085FFFCCF7E
:103EC0008AE08093C600E7ECFFE08491882309F440
:103ED00096CF9091C00095FFFCCF8093C60031969D
:103EE000F4CF8091C00085FFFCCF8AE08093C600AC
:103EF000CC2311F1409173055091740560917505C3
:103F0000709176058CE394E09AD4409177055091B6
:103F100078056091790570917A0589E394E08FD4F2
:103F200040917B0550917C0560917D0570917E05E7
:103F300086E394E084D42FC0E7ECFFE084918823EB
:103F400041F09091C00095FFFCCF8093C600319660
:103F5000F5CFE5E4F4E08491882341F09091C0002E
:103F600095FFFCCF8093C6003196F5CF8091C000BD
:103F700085FFFCCF8AE08093C600E7ECFFE08491E8
:103F8000882309F4B7CF9091C00095FFFCCF8093B0
:103F9000C6003196F4CF8091C00085FFFCCF8AE047
:103FA0008093C600CC2311F140911A1350911B133A
:103FB000662757FD6095762F8EE094E062D440919D
:103FC000181350911913662757FD6095762F8BE0D3
:103FD00094E057D44091161350911713662757FD5C
:103FE0006095762F88E094E04CD42FC0E7ECFFE09A
:103FF0008491882341F09091C00095FFFCCF80937D
:10400000C6003196F5CFEAE1F4E08491882341F0CF
:104010009091C00095FFFCCF8093C6003196F5CFFC
:104020008091C00085FFFCCF8AE08093C600E7EC5A
:10403000FFE08491882309F4B7CF9091C00095FFE9
:10404000FCCF8093C6003196F4CF8091C00085FFED
:10405000FCCF8AE08093C600CC2311F14091141369
:1040600050911513662757FD6095762F8CEF93E0DE
:1040700008D44091121350911313662757FD609591
:10408000762F89EF93E0FDD34091101350911113D7
:10409000662757FD6095762F86EF93E0F2D30DC02B
:1040A000E7ECFFE084918823C9F29091C00095FF6E
:1040B000FCCF8093C6003196F5CF8091C00085FF7C
:1040C000FCCF8AE08093C600CC2309F43CC0409129
:1040D00081025091820260918302709184028FED7F
:1040E00093E0ADD360917D0270917E0280917F025A
:1040F000909180020E94A4A6AB01BC018CED93E0DC
:104100009ED36091790270917A0280917B029091A6
:104110007C020E94B0A6AB01BC0189ED93E08FD375
:104120004091750250917602609177027091780209
:1041300086ED93E084D360910A0270910B0283EDC7
:1041400093E06CD32FC0E7ECFFE08491882341F02B
:104150009091C00095FFFCCF8093C6003196F5CFBB
:10416000E8EEF3E08491882341F09091C00095FF40
:10417000FCCF8093C6003196F5CF8091C00085FFBB
:10418000FCCF8AE08093C600E7ECFFE084918823AF
:1041900009F49DCF9091C00095FFFCCF8093C6009D
:1041A0003196F4CF8091C00085FFFCCF8AE08093E8
:1041B000C600CC2361F04091290250912A026091FF
:1041C0002B0270912C028DEA93E039D345C0E7ECC5
:1041D000FFE08491882341F09091C00095FFFCCFCF
:1041E0008093C6003196F5CFE0ECF3E0849188230C
:1041F00041F09091C00095FFFCCF8093C6003196AE
:10420000F5CF80917F05811103C0E6EBF3E00CC090
:104210008091C00085FFFCCF0EC09091C00095FF3B
:10422000FCCF8093C600319684918111F6CF8091A6
:10423000C00085FFFCCF8AE08093C600E7ECFFE07A
:104240008491882309F4B7CF9091C00095FFFCCFEB
:104250008093C6003196F4CF8091C00085FFFCCFDB
:104260008AE08093C60080917F05811123C0C1112F
:104270000DC0E7ECFFE007C09091C00095FFFCCFB8
:104280008093C600319684918111F6CFE3EAF3E082
:1042900007C09091C00095FFFCCF8093C600319677
:1042A00084918111F6CF8091C00085FFFCCF8AE018
:1042B0008093C600CC2361F040910E0250910F0212
:1042C000609110027091110285E893E0B8D22EC07F
:1042D000E7ECFFE08491882341F09091C00095FFC6
:1042E000FCCF8093C6003196F5CFEEE8F3E08491E1
:1042F000882341F09091C00095FFFCCF8093C600C9
:104300003196F5CF8091C00085FFFCCF8AE0809385
:10431000C600E7ECFFE08491882371F29091C00021
:1043200095FFFCCF8093C6003196F5CF8091C000F9
:1043300085FFFCCF8AE08093C600CF9108951F923D
:104340000F920FB60F9211240BB60F922F933F933B
:104350004F935F936F938F939F93EF93FF9360912E
:10436000C60020913D0530913E05C90101968F7729
:10437000992740913F05509140058417950741F0DA
:10438000F901E354FB4F608390933E0580933D0514
:10439000FF91EF919F918F916F915F914F913F911D
:1043A0002F910F900BBE0F900FBE0F901F9018957E
:1043B0009A01AB01211581EE38074105510549F1FC
:1043C00082E08093C00060E079E08DE390E00E949D
:1043D00074CF2150310941095109CA01B90122E0C4
:1043E00030E040E050E00E9474CF3093C50020934D
:1043F000C4008091C10080618093C1008091C100A0
:1044000088608093C1008091C10080688093C10062
:1044100008951092C00020E130E0E7CF20913F05E1
:104420003091400580913D0590913E05821793079C
:1044300071F0F901E354FB4F80812F5F3F4F2F77DD
:1044400033273093400520933F0590E008958FEF88
:104450009FEF089580913F059091400590933E0510
:1044600080933D0508954F925F926F927F928F9255
:104470009F92AF92BF92CF92DF92EF92FF920F93F3
:104480001F93CF93DF93CDB7DEB7A0970FB6F89405
:10449000DEBF0FBECDBF5C01411551056105710541
:1044A000E9F420E030E040E350E060E070E0A09606
:1044B0000FB6F894DEBF0FBECDBFDF91CF911F9135
:1044C0000F91FF90EF90DF90CF90BF90AF909F90B3
:1044D0008F907F906F905F904F905BC08E010F5FC9
:1044E0001F4FC12CD12C76014801422E512C612C3A
:1044F000712C8FEFC81AD80AE80AF80ACB01BA0162
:10450000A30192010E9452CFCA01F80161938F0169
:10451000A901BC01411551056105710551F7F1E093
:10452000CF1AD108E108F108F401EC0DFD1D8081DE
:104530008A3010F440E301C047E3480F552747FD98
:104540005095652F752F20E030E0C50122D081E025
:10455000C81AD108E108F108EFEFCE16DE06EE0624
:10456000FE0611F7A0960FB6F894DEBF0FBECDBFC2
:10457000DF91CF911F910F91FF90EF90DF90CF903F
:10458000BF90AF909F908F907F906F905F904F9073
:1045900008952115310539F48091C00085FFFCCFC5
:1045A0004093C60008952A30310509F41CC05BCF42
:1045B000CF93DF93EC0120E030E04DE050E060E08D
:1045C00070E0E7DF20E030E04AE050E060E070E0DB
:1045D000CE01DF91CF91DDCF9A01AB01662757FD68
:1045E0006095762FD6CFCF92DF92EF92FF92CF9346
:1045F000DF93EC016A017B0177FF0FC020E030E020
:104600004DE250E060E070E0C4DFF094E094D094BC
:10461000C094C11CD11CE11CF11C2AE0B701A60109
:10462000CE01DF91CF91FF90EF90DF90CF901BCF25
:104630002115310539F48091C00085FFFCCF4093EE
:10464000C600089510CF9A01462F50E060E070E058
:10465000EFCFCF93DF93EC019A01AB0160E070E004
:10466000E7DFCE01DF91CF91A3CF8F929F92AF92E0
:10467000BF92CF92DF92EF92FF921F93CF93DF937F
:10468000EC016A017B01122F20E030E0A901C70193
:10469000B6010E9481CB87FF0CC020E030E04DE2E4
:1046A00050E060E070E0CE0174DFF7FAF094F7F8C4
:1046B000F094B12C60E070E080E09FE3B11641F02F
:1046C00020E030E040E251E40E9488CBB394F6CF82
:1046D0009B01AC01C701B6010E94A8CA6B017C0115
:1046E0000E94F5CB4B015C010E9421CC9B01AC01E7
:1046F000C701B6010E94A7CA6B017C012AE0B5017F
:10470000A401CE01B0DE112341F020E030E04EE202
:1047100050E060E070E0CE013CDF112319F120E0B1
:1047200030E040E251E4C701B6010E9456CE6B0171
:104730007C010E94F0CB4B01AA2497FCA094BA2CD8
:10474000B501A401CE014FDFC501B4010E9423CC05
:104750009B01AC01C701B6010E94A7CA6B017C0195
:104760001150DBCFDF91CF911F91FF90EF90DF9041
:10477000CF90BF90AF909F908F90089576CFFC011F
:10478000659175918591949108950E94E5C7609314
:1047900056057093570580935805909359050895D1
:1047A0008091310290913202A0913302B091340293
:1047B00080933B0790933C07A0933D07B0933E073F
:1047C00080912F0290913002909381058093800513
:1047D00084E690E09093300280932F02D6DF81E050
:1047E0000C94749180E00E94749180913B079091A9
:1047F0003C07A0913D07B0913E0780933102909312
:104800003202A0933302B0933402809180059091DC
:1048100081059093300280932F02B7CFFC01249141
:10482000222341F03091C00035FFFCCF2093C60019
:104830000196F4CF4AE050E08CEB94E0CDCEFC0141
:104840002491222341F03091C00035FFFCCF20930A
:10485000C6000196F4CF22E030E08CEB94E08ECFDE
:10486000FC012491222341F03091C00035FFFCCFA0
:104870002093C6000196F4CF22E030E08CEB94E068
:104880007DCFFC012491222341F03091C00035FFFF
:10489000FCCF2093C6000196F4CF2AE030E08CEBE9
:1048A00094E0C6CECF93DF93FC0120812B3309F433
:1048B00067C02091060730910707243031050CF0BE
:1048C0005FC0209108073091090740E6429FE00150
:1048D000439FD00D1124CA57DA4FBC01CE010E946C
:1048E000EBD2E7ECFFE08491882341F09091C00087
:1048F00095FFFCCF8093C6003196F5CFEBE7FFE044
:104900008491882371F09091C00095FFFCCF809333
:10491000C6003196F5CF9091C00095FFFCCF8093F3
:10492000C60089918111F7CFE9E7FFE084918823E0
:1049300041F09091C00095FFFCCF8093C600319666
:10494000F5CF8091C00085FFFCCF8AE08093C60040
:104950008091080790910907019664E070E00E9439
:104960003FCF9093090780930807809106079091A5
:1049700007070196909307078093060781E001C01F
:1049800080E0DF91CF910895DF92EF92FF920F9335
:104990001F93CF93DF93CDB7DEB76E970FB6F89422
:1049A000DEBF0FBECDBF60915A0570915B056115EA
:1049B0007105A1F04DE150E08E010F5F1F4FC8015E
:1049C0000E947AD21E8EF8017F01E01AF10AD1907E
:1049D000DD2031F08AE0D812F7CF02C080E01DC0A0
:1049E000F801EE0DFF1D1082C8015CDF8823A1F0E5
:1049F000DD2071F08FEFE81AF80A80915A05909146
:104A00005B058E0D9F1D90935B0580935A0504C036
:104A100010925B0510925A0581E06E960FB6F894DD
:104A2000DEBF0FBECDBFDF91CF911F910F91FF90E1
:104A3000EF90DF90089590935B0580935A05A4CF83
:104A40009898A09A0895269A2E980895F9DFFBDF8A
:104A500040E052EC61E070E08CEB94E0A9DCE3E72D
:104A6000FFE08491882341F09091C00095FFFCCF36
:104A70008093C6003196F5CF8091C00085FFFCCFB2
:104A80008AE08093C600E7ECFFE08491882341F040
:104A90009091C00095FFFCCF8093C6003196F5CF72
:104AA00084B780FF14C0EBE6FFE09491992341F0B6
:104AB0002091C00025FFFCCF9093C6003196F5CF22
:104AC0009091C00095FFFCCF9AE09093C60081FFC3
:104AD00014C0EBE5FFE09491992341F02091C000D0
:104AE00025FFFCCF9093C6003196F5CF9091C00082
:104AF00095FFFCCF9AE09093C60082FF14C0EAE4D1
:104B0000FFE09491992341F02091C00025FFFCCF54
:104B10009093C6003196F5CF9091C00095FFFCCFE1
:104B20009AE09093C60083FF14C0EAE3FFE09491FB
:104B3000992341F02091C00025FFFCCF9093C6003F
:104B40003196F5CF9091C00095FFFCCF9AE09093FD
:104B5000C60085FF14C0EAE2FFE08491882341F09B
:104B60009091C00095FFFCCF8093C6003196F5CFA1
:104B70008091C00085FFFCCF8AE08093C60014BE00
:104B8000E3E2FFE08491882341F09091C00095FF1B
:104B9000FCCF8093C6003196F5CFE1E2FFE084912F
:104BA000882341F09091C00095FFFCCF8093C60010
:104BB0003196F5CF8091C00085FFFCCF8AE08093CD
:104BC000C600E7ECFFE08491882341F09091C0009B
:104BD00095FFFCCF8093C6003196F5CFE1E1FFE071
:104BE0008491882341F09091C00095FFFCCF809381
:104BF000C6003196F5CFE0E0FFE08491882341F0D4
:104C00009091C00095FFFCCF8093C6003196F5CF00
:104C1000E4EFFEE08491882341F09091C00095FF7D
:104C2000FCCF8093C6003196F5CFEDEDFEE0849188
:104C3000882341F09091C00095FFFCCF8093C6007F
:104C40003196F5CF8091C00085FFFCCF8AE080933C
:104C5000C600E2EDFEE08491882341F09091C0000F
:104C600095FFFCCF8093C6003196F5CFE6ECFEE0D1
:104C70008491882341F09091C00095FFFCCF8093F0
:104C8000C6003196F5CF8091C00085FFFCCF8AE049
:104C90008093C600E7ECFFE08491882341F0909177
:104CA000C00095FFFCCF8093C6003196F5CFE7EBAF
:104CB000FEE08491882341F09091C00095FFFCCFE5
:104CC0008093C6003196F5CF0E94268C4AE050E0D2
:104CD000BC018CEB94E080DCE0EAFEE08491882368
:104CE00041F09091C00095FFFCCF8093C6003196B3
:104CF000F5CF4AE050E060ED74E08CEB94E06CDCC2
:104D00008091C00085FFFCCF8AE08093C60010929E
:104D100044051092450510924605109247050E94E1
:104D2000E71B80E00E94711D0E946CAA0E94C69E33
:104D30000E94BC5F0E94FB9860E082E00E94BCC9B8
:104D400061E082E00E94F5C961E081E40E94BCC993
:104D500060E081E40C94F5C90F931F93CF93DF9328
:104D600000915C0510915D0565E470E0C8010E944A
:104D7000D7D2EC01C8010196209761F0188260E05B
:104D800070E00E94B9CF25E42883DF91CF911F9175
:104D90000F91089560E070E0DF91CF911F910F9126
:104DA0000C94B9CF80915C0590915D054AE050E08C
:104DB00060E070E001960C9421D180915C059091A7
:104DC0005D054AE050E060E070E001960E9421D16C
:104DD000CB010895682F772767FD709580910C07A8
:104DE00090910D070E94D7D290935D0580935C054A
:104DF00021E0892B09F420E0822F08950F931F935F
:104E0000CF93DF9300D000D0CDB7DEB726E0E5EF3B
:104E1000F2E0DE01119601900D922A95E1F7FC0176
:104E2000EE0FFF1F21E030E02C0F3D1FE20FF31FBC
:104E300060817181161617061CF1E7ECFFE02491E2
:104E4000222341F03091C00035FFFCCF2093C600F3
:104E50003196F5CFE6E8FCE02491222341F0309131
:104E6000C00035FFFCCF2093C6003196F5CF2091CE
:104E7000C00025FFFCCF2AE02093C6006AE070E066
:104E80008C01000F111F000F111F075E1B4F882799
:104E900077FD8095982F0E9423CC9B01AC01F801EF
:104EA00060817181828193810E9488CB60933102FD
:104EB00070933202809333029093340226960FB699
:104EC000F894DEBF0FBECDBFDF91CF911F910F9140
:104ED00008958F929F92AF92BF92CF92DF92EF92FE
:104EE000FF920F931F9320E030E040E752E460917F
:104EF00031027091320280913302909134020E940B
:104F000088CB4B015C01E0903307F09034070091AF
:104F100035071091360720912F07309130074091C7
:104F200031075091320760912B0770912C078091C7
:104F30002D0790912E07E0916605EF93E7E3CE2EC3
:104F4000E7E0DE2E0E941C610F901F910F91FF90F1
:104F5000EF90DF90CF90BF90AF909F908F9008958B
:104F60004F925F926F927F928F929F92AF92BF9279
:104F7000EF92FF920F931F93CF93DF93CDB7DEB7DE
:104F800028970FB6F894DEBF0FBECDBF4B015C0172
:104F90008091310290913202A0913302B09134029B
:104FA00089839A83AB83BC83412C512CF0E76F2E0D
:104FB000F3E47F2E4092310250923202609233022B
:104FC00070923402E0923307F09234070093350771
:104FD000109336072D833E834F8358877ADF0E94D4
:104FE0008D996091120270911302882777FD809548
:104FF000982F0E9423CC60933102709332028093E9
:1050000033029093340280922B0790922C07A09247
:105010002D07B0922E072D813E814F815885209318
:105020002F0730933007409331075093320751DFF9
:105030000E948D9989819A81AB81BC8180933102D4
:1050400090933202A0933302B093340228960FB6A5
:10505000F894DEBF0FBECDBFDF91CF911F910F91AE
:10506000FF90EF90BF90AF909F908F907F906F9048
:105070005F904F9008954F925F926F927F928F92C0
:105080009F92AF92BF92CF92DF92EF92FF920F93D7
:105090001F932B013C0120E030E040E752E4609197
:1050A00031027091320280913302909134020E9459
:1050B00088CB4B015C0120912F0730913007409144
:1050C00031075091320760912B0770912C07809126
:1050D0002D0790912E07E0916605EF93A7E3CA2E66
:1050E000A7E0DA2E830172010E941C610F901F91CC
:1050F0000F91FF90EF90DF90CF90BF90AF909F9077
:105100008F907F906F905F904F9008958F929F92B5
:10511000AF92BF92CF92DF92EF92FF920F931F93C5
:1051200020E030E040E752E40E9488CB4B015C0174
:10513000E0902307F090240700912507109126079F
:1051400020911F073091200740912107509122079D
:1051500060911B0770911C0780911D0790911E079D
:10516000E0916605EF93B7E2CB2EB7E0DB2E0E940D
:105170001C610F901F910F91FF90EF90DF90CF90E7
:10518000BF90AF909F908F90089560913102709181
:1051900032028091330290913402B8CFCF92DF92E5
:1051A000EF92FF920F931F93E0903307F090340734
:1051B000009135071091360720912F073091300765
:1051C000409131075091320760912B0770912C0765
:1051D00080912D0790912E07E7E3CE2EE7E0DE2E9B
:1051E0000E94316E1F910F91FF90EF90DF90CF9052
:1051F00008952F923F924F925F926F927F928F927B
:105200009F92AF92BF92CF92DF92EF92FF920F9355
:105210001F93CF93DF9300D01F92CDB7DEB78C01E1
:105220009A838983FC01E857F04FF4909C01220F88
:10523000331F220F331F3C832B83255D384F190109
:10524000F9011082118212821382A8DF8B819C8166
:105250008956904F94DA2B013C016F2D772767FD1B
:105260007095872F972F0E9423CC4B015C012B81D7
:105270003C81255E384F790120E030E040EC5FE36F
:10528000C301B2010E9456CEA50194010E9456CEE0
:10529000F7016083718382839383EB81FC81E75EF6
:1052A000FB4F80819181A281B381809331029093E1
:1052B0003202A0933302B093340267DF0E948D99CB
:1052C000F101108211821282138268DF80E00E9455
:1052D00074912B813C812557304F6901C9014FDA08
:1052E0009058A50194010E9456CEF7016083718306
:1052F000828393834ADF0E948D9981E00E9474919A
:10530000C8017CDDC6013BDA9B01AC010E94A8CA42
:10531000A50194010E9456CEF701608371838283B8
:10532000938333DF0E948D998B819C818D55904FA3
:1053300026DA2B813C812D583A4F7901F9012081E1
:105340003181428153810E94A8CAF1016083718337
:10535000828393838B819C818554904F10DA2B81BB
:105360003C8129593A4F6901F701208131814281FD
:1053700053810E94A8CAF60160837183828393835C
:105380008B819C818155904FFAD92B813C81275E7E
:105390003D4F6901F70120813181428153810E9493
:1053A000A8CAF601608371838283938329813A813D
:1053B00022303105D1F420910E0230910F0240913C
:1053C000100250911102609133077091340780915F
:1053D0003507909136070E94A7CA609333077093F0
:1053E00034078093350790933607D8DEEB81FC8134
:1053F000E55EF84FAB81BC81A55DB84F8D919D9165
:105400000D90BC91A02D80839183A283B3831092D1
:1054100031021092320210923302109234020E9432
:10542000DF90F801E85EF84F81E080830F900F90E5
:105430000F900F90DF91CF911F910F91FF90EF9000
:10544000DF90CF90BF90AF909F908F907F906F90A4
:105450005F904F903F902F9008958F929F92AF92C0
:10546000BF92CF92DF92EF92FF920F931F9383E44C
:1054700092E00E9498C180E090E0A0E7B3E48093BE
:10548000310290933202A0933302B093340260E071
:1054900070E08AEA93ECEFDD0E948D9982E090E063
:1054A0000E94F2994B015C0120912F073091300747
:1054B000409131075091320760912B0770912C0772
:1054C00080912D0790912E07A7E3CA2EA7E0DA2E30
:1054D000850174010E94316E83E99FE050D99B01E0
:1054E000AC01C501B4010E94A8CA4B015C01C3DD37
:1054F0000E948D990E94DF9082E090E07FDC83E93A
:105500009FE03DD99B01AC010E94A8CA9B01AC0160
:10551000C501B4010E94A7CAAEDD0E948D990E9408
:10552000DF9082E090E00E94F299609333077093DD
:10553000340780933507909336071F910F91FF90A2
:10554000EF90DF90CF90BF90AF909F908F9026CE3E
:1055500080E1EBE1F7E0ABE2B7E001900D928A95D4
:10556000E1F70895CF92DF92EF92FF920F931F938E
:10557000CF93DF93B5E1EB2EB4E0FB2E0BE117E008
:10558000CBE2D7E082E8C82E85E0D82EF7018191E2
:105590007F0120DC8823C9F0DFDBF60120812111A7
:1055A00004C020916205222329F0288139814A8193
:1055B0005B8103C020E030E0A9010E94A8CAF80185
:1055C000608371838283938309C088819981AA81D2
:1055D000BB81F80180839183A283B3830C5F1F4F4B
:1055E0002496FFEFCF1ADF0A89E1E81684E0F80677
:1055F00069F686E4EFDB882391F0AEDB6B017C017A
:1056000020E030E0A9010E9484CD181644F4C09235
:105610003102D0923202E0923302F0923402DF91F2
:10562000CF911F910F91FF90EF90DF90CF90089551
:10563000E7ECFFE08491882341F09091C00095FF52
:10564000FCCF8093C6003196F5CFE9E1FDE084916F
:10565000882341F09091C00095FFFCCF8093C60055
:105660003196F5CFE0910E07F0910F0781918823D5
:1056700039F09091C00095FFFCCF8093C600F6CF23
:10568000E6E1FDE08491882341F09091C00095FF10
:10569000FCCF8093C6003196F5CF08954F925F926C
:1056A0006F927F928F929F92AF92BF92CF92DF9232
:1056B000EF92FF920F931F930E948D9983E492E0E3
:1056C0000E9498C16DD880E1EBE2F7E0ABE1B7E072
:1056D00001900D928A95E1F71092310210923202F8
:1056E000109233021092340288E574DB982E89E51B
:1056F00071DBA82E8AE56EDBB82E911005C0A110D3
:1057000007C091E0982705C0AA2011F0982F01C08A
:1057100090E090930C02911102C0992019F080E062
:1057200090E067DD80910C02811102C0AA2019F07F
:1057300081E090E05EDD80910C02882309F462C074
:1057400010923307109234071092350710923607E3
:1057500025DD80E090E0ACEDB2E480931B079093F0
:105760001C07A0931D07B0931E0780931F079093FB
:105770002007A0932107B0932207EAE8FFE0649195
:1057800088EF6802B0011124882777FD8095982F53
:105790000E9423CC609323077093240780932507EE
:1057A0009093260780E090E8ABE3B5E48093310264
:1057B00090933202A0933302B0933402E6DC0E944D
:1057C0008D9980911B0790911C07A0911D07B091A6
:1057D0001E0780932B0790932C07A0932D07B0935F
:1057E0002E0780911F0790912007A0912107B0916B
:1057F000220780932F0790933007A0933107B0932F
:10580000320788C0BB2009F4D3C0809118078823D1
:1058100009F4A8C080911907882309F4A3C08090D7
:105820002B0790902C07A0902D07B0902E0740904A
:105830002F0750903007609031077090320720E0BA
:1058400030E0A901C501B4010E9484CD87FD66C086
:1058500020E030E04CE553E4C501B4010E9481CB67
:1058600018160CF45BC020E030E0A901C301B201BE
:105870000E9484CD87FD52C020E030E04CE553E427
:10588000C301B2010E9481CB18160CF447C01092DC
:10589000330710923407109235071092360797E3BA
:1058A000C92E97E0D92EE12CF12C8701A30192019A
:1058B000C501B4010E94316EEAE8FFE0649188EF0F
:1058C0006802B0011124882777FD8095982F0E94E7
:1058D00023CC60932307709324078093250790932C
:1058E000260720E030E040E752E46091210F7091FC
:1058F000220F8091230F9091240F0E9456CE609327
:1059000031027093320280933302909334023DDC73
:105910000E948D9982E090E06CDC4AC060E08CEDE2
:105920009CE00E94F9A9E7ECFFE08491882341F014
:105930009091C00095FFFCCF8093C6003196F5CFC3
:10594000EBECFCE08491882341F09091C00095FF3E
:10595000FCCF8093C6003196F5CF8091C00085FFC3
:10596000FCCF23C060E089EB9CE00E94F9A9E7EC42
:10597000FFE08491882341F09091C00095FFFCCF17
:105980008093C6003196F5CFE7EAFCE08491882346
:1059900041F09091C00095FFFCCF8093C6003196F6
:1059A000F5CF8091C00085FFFCCF8AE08093C600D0
:1059B000F5DB80E00E94749180913B0790913C0759
:1059C000A0913D07B0913E0780933102909332023F
:1059D000A0933302B09334028091800590918105A9
:1059E0009093300280932F020E94C5231F910F9144
:1059F000FF90EF90DF90CF90BF90AF909F908F90EF
:105A00007F906F905F904F900C94DF90EEE0FDE000
:105A10002491222379F03091C00035FFFCCF2093F0
:105A2000C6003196F5CF3091C00035FFFCCF2093F2
:105A3000C6000196FC0124912111F5CFE6EFFCE0B0
:105A40008491882341F09091C00095FFFCCF809312
:105A5000C6003196F5CF8091C00085FFFCCF8AE06B
:105A60008093C60008950E948D990E94D02380E003
:105A700090E0A0E7B3E48093310290933202A093C8
:105A80003302B0933402E9DCECECFAE08491882331
:105A900041F09091C00095FFFCCF8093C6003196F5
:105AA000F5CF27E137EB41ED58E360912B0770917B
:105AB0002C0780912D0790912E070E94A8CAAB0158
:105AC000BC0122E030E08CEB94E00E94BE23E7ECC6
:105AD000FAE08491882341F09091C00095FFFCCFBB
:105AE0008093C6003196F5CF27E137EB41ED58E3BF
:105AF00060912F07709130078091310790913207A4
:105B00000E94A8CAAB01BC0122E030E08CEB94E01B
:105B10000E94BE23E2ECFAE08491882341F0909148
:105B2000C00095FFFCCF8093C6003196F5CF27E1EA
:105B300037EB41ED58E36091330770913407809162
:105B40003507909136070E94A8CAAB01BC0122E03C
:105B500030E08CEB94E00E94BE238091C00085FF72
:105B6000FCCF8AE08093C6000C94F223BF92CF92C0
:105B7000DF92EF92FF920F931F93CF93DF9300D0AA
:105B80001F92CDB7DEB785E425D9811102C00E94EE
:105B90008D9925E1C22E24E0D22E3BE2E32E37E0A0
:105BA000F32E00E010E0B12CF60181916F0112D9C3
:105BB0008823A1F0D1D8F701608371838283938316
:105BC00069837A838B839C830330110529F4CE018A
:105BD00001960E94526F02C0BB24B3940F5F1F4F07
:105BE000F4E0EF0EF11C04301105F1F6B110D6DA35
:105BF0000F900F900F900F90DF91CF911F910F9109
:105C0000FF90EF90DF90CF90BF900895E9E7FAE022
:105C10008491882341F09091C00095FFFCCF809340
:105C2000C6003196F5CF8091C00085FFFCCF8AE099
:105C30008093C6008FE397E00E944E12EBE6FAE0F5
:105C40008491882341F09091C00095FFFCCF809310
:105C5000C6003196F5CF8091C00085FFFCCF8AE069
:105C60008093C60008950F931F93CF93DF93CDB712
:105C7000DEB76E970FB6F894DEBF0FBECDBF0E94A1
:105C8000E5C760934A0570934B0580934C0590934C
:105C90004D0500914E0510914F0520915005309112
:105CA0005105601B710B820B930B28EE33E040E033
:105CB00050E00E9452CFCA01B9012CE330E040E02D
:105CC00050E00E9452CF7F936F933F932F938CE5C8
:105CD0009AE09F938F938E010F5F1F4F1F930F9337
:105CE0000E940FD30FB6F894DEBF0FBECDBFE7EC16
:105CF000FFE08491882341F09091C00095FFFCCF94
:105D00008093C6003196F5CFF8018191882339F050
:105D10009091C00095FFFCCF8093C600F6CF809194
:105D2000C00085FFFCCF8AE08093C60060E0C80118
:105D30000E94AFA98091C80E882309F11092C80E65
:105D40000091660510E0000F111F08541D4EF80168
:105D500060817181882777FD8095982F0E9423CCE0
:105D600020913B0230913C0240913D0250913E0215
:105D70000E9484CD18161CF4F801118210826E96D0
:105D80000FB6F894DEBF0FBECDBFDF91CF911F914C
:105D90000F9108951F93CF93DF9380914107811155
:105DA0000E948D99C0910C07D0910D0761E270E0BF
:105DB000CE010E94D7D2009711F0EC01219680E528
:105DC00009D8882341F011E080915C0590915D0530
:105DD0008C179D0708F010E0809142078823C9F1D5
:105DE00021E0212741E0BE018FE397E00E942017C8
:105DF00083E50E94EA26882339F080915C05909122
:105E00005D058C179D0788F08FE397E00E94701363
:105E100011111FC00E94E5C760934E0570934F0596
:105E2000809350059093510514C00E94DD26AC016B
:105E3000662757FD6095762F4093C2095093C3099A
:105E40006093C4097093C5098DE099E00E94C186F2
:105E5000DBCFDF91CF911F9108950F931F93CF93C5
:105E6000DF9383E50E94EA268823B9F10E94DD26AC
:105E70008C0180E50E94EA26882321F00F3F11055E
:105E800041F138F1CDE0D0E0EFEDF3E08191919177
:105E90008C179D0711F184E0E531F807B9F7C93097
:105EA000D10529F4109365050093640502C0D7FD60
:105EB00014C061E08C2F0E94BCC9602F8C2F0E94FF
:105EC000F5C9B8018C2FDF91CF911F910F910C94E0
:105ED000A6C80E94DD26EC01D7CFDF91CF911F919C
:105EE0000F9108952F923F924F925F926F927F92FF
:105EF0008F929F92AF92BF92CF92DF92EF92FF92DA
:105F00000F931F93CF93DF93CDB7DEB7CC5ED1094C
:105F10000FB6F894DEBF0FBECDBF86E50E94EA261D
:105F20008823F9F00E94DD26C353DF4F8883CD5CC0
:105F3000D040853070F0E7E3FAE08491882309F4DB
:105F4000A9C69091C00095FFFCCF8093C600319602
:105F5000F4CFC353DF4F2881CD5CD0402223A1F082
:105F600006C031E0C353DF4F3883CD5CD040E7E15A
:105F7000FAE08491882341F09091C00095FFFCCF16
:105F80008093C6003196F5CF80E50E94EA268823EB
:105F9000C1F00E94DD26C551DF4F8883CB5ED04023
:105FA00084508F32A0F0E3EFF9E08491882309F464
:105FB00071C69091C00095FFFCCF8093C6003196CA
:105FC000F4CF4AE0C551DF4F4883CB5ED04080E03C
:105FD00090E00E94F299CA52DF4F6883C65DD040BC
:105FE000C652DF4F7883CA5DD040C152DF4F8883ED
:105FF000CF5DD040CF51DF4F9883C15ED04081E06C
:1060000090E00E94F299362E272ECD51DF4F8883E3
:10601000C35ED040C951DF4F9883C75ED04082E055
:1060200090E00E94F2994B015C0183E090E00E94B5
:10603000F299C753DF4F688379838A839B83C95C56
:10604000D04085E40E94EA26C451DF4F8883CC5EAD
:10605000D04088E50E94EA268823E1F10E94AC2620
:10606000C253DF4F6883CE5CD040C153DF4F78838B
:10607000CF5CD040C053DF4F8883C05DD040CF524B
:10608000DF4F9883C15DD04020E030E0A9010E943D
:1060900081CB87FD1CC020E030E04CE553E4C253C7
:1060A000DF4F6881CE5CD040C153DF4F7881CF5C39
:1060B000D040C053DF4F8881C05DD040CF52DF4F0A
:1060C0009881C15DD0400E9484CD18165CF581EFA7
:1060D00099E069C0CA52DF4F5881C65DD040C253B3
:1060E000DF4F5883CE5CD040C652DF4F8881CA5DF7
:1060F000D040C153DF4F8883CF5CD040C152DF4FC7
:106100009881CF5DD040C053DF4F9883C05DD040B1
:10611000CF51DF4FA881C15ED040CF52DF4FA8835F
:10612000C15DD04089E50E94EA26882309F43DC07C
:106130000E94AC26CE52DF4F6883C25DD040CD5264
:10614000DF4F7883C35DD040CC52DF4F8883C45D7E
:10615000D040CB52DF4F9883C55DD04020E030E087
:10616000A9010E9481CB87FD1CC020E030E04CE5F6
:1061700053E4CE52DF4F6881C25DD040CD52DF4F35
:106180007881C35DD040CC52DF4F8881C45DD04060
:10619000CB52DF4F9881C55DD0400E9484CD181648
:1061A00014F58FEE99E032DC75C5CE52DF4F3882A0
:1061B000C25DD040CD52DF4F2882C35DD040CD516B
:1061C000DF4FB881C35ED040CC52DF4FB883C45D8F
:1061D000D040C951DF4FE881C75ED040CB52DF4F7E
:1061E000E883C55DD0408CE40E94EA268823C9F08C
:1061F0000E94DD26C252DF4F8883CE5DD0408130C1
:10620000B1F08031D0F0ECEBF9E08491882309F40F
:1062100041C59091C00095FFFCCF8093C600319698
:10622000F4CFC252DF4F1882CE5DD04006C0F2E0FC
:10623000C252DF4FF883CE5DD04020E030E040E72F
:1062400051E4C501B4010E94A8CA2B013C010E947F
:106250008D9983E492E00E9498C180916605C753AE
:10626000DF4F288139814A815B81C95CD040298315
:106270003A834B835C838F93812C912CB0E8AB2EB7
:10628000B0E4BB2EAE014F5F5F4F6A018301720124
:10629000232D322DCD51DF4F4881C35ED040C951EF
:1062A000DF4F5881C75ED040CA52DF4F6881C65D5C
:1062B000D040C652DF4F7881CA5DD040C152DF4F17
:1062C0008881CF5DD040CF51DF4F9881C15ED040F3
:1062D0000E941C610E948D990F90C353DF4F58811B
:1062E000CD5CD040533008F009C180916605C7539A
:1062F000DF4F288139814A815B81C95CD040298385
:106300003A834B835C838F93812C912CE8E4AE2EEF
:10631000E2E4BE2EAE014F5F5F4F6A01830172015E
:10632000CE52DF4F2881C25DD040CD52DF4F388141
:10633000C35DD040CC52DF4F4881C45DD040CB52CA
:10634000DF4F5881C55DD040C253DF4F6881CE5CBE
:10635000D040C153DF4F7881CF5CD040C053DF4F76
:106360008881C05DD040CF52DF4F9881C15DD04061
:106370000E941C610E948D9980E090E00E94F29939
:1063800060932B0770932C0780932D0790932E0713
:1063900081E090E00E94F29960932F07709330079C
:1063A000809331079093320782E090E00E94F29947
:1063B00060933307709334078093350790933607C3
:1063C00083E090E00E94F2994B015C0160933707F3
:1063D000709338078093390790933A070E94D0232F
:1063E0003CD882E090E00E94F2996093330770936A
:1063F0003407809335079093360782E090E00E943F
:10640000F29920E030E040E751E40E94A8CAC65269
:10641000DF4F688379838A839B83CA5DD0408091F4
:10642000660589829A82AB82BC828F93812C912CE3
:10643000F8E4AF2EF2E4BF2EC652DF4FE880F980B9
:106440000A811B81CA5DD040CE52DF4F2881C25DD8
:10645000D040CD52DF4F3881C35DD040CC52DF4FAA
:106460004881C45DD040CB52DF4F5881C55DD040DC
:10647000C253DF4F6881CE5CD040C153DF4F78817B
:10648000CF5CD040C053DF4F8881C05DD040CF5239
:10649000DF4F9881C15DD0400E941C610E948D99A0
:1064A00082E090E00E94F299C951DF4F68837983BE
:1064B0008A839B83C75ED040609333077093340711
:1064C0008093350790933607C152DF4FD982C88237
:1064D000CF5DD0400F900F9022242394312CC252D4
:1064E000DF4FF881CE5DD040EF2FF0E03197CF51F4
:1064F000DF4FF983E883C15ED04071C0E2EAF9E082
:106500008491882309F4F1CE9091C00095FFFCCFCF
:106510008093C6003196F4CFC353DF4F9881CD5C92
:10652000D040911154C3809166058F93812C912C9A
:1065300050E8A52E50E4B52E67E3C62E67E0D62EB0
:10654000C652DF4FE880F9800A811B81CA5DD040C6
:10655000CE52DF4F2881C25DD040CD52DF4F38810F
:10656000C35DD040CC52DF4F4881C45DD040CB5298
:10657000DF4F5881C55DD040C253DF4F6881CE5C8C
:10658000D040C153DF4F7881CF5CD040C053DF4F44
:106590008881C05DD040CF52DF4F9881C15DD0402F
:1065A0000E941C610E948D990F90C451DF4FA881F9
:1065B000CC5ED040AA2331F068EE73E080E090E03A
:1065C0000E9414C8BFEF2B1A3B0A8FEF820DC551F2
:1065D000DF4FE881CB5ED0408E1708F000C3CC249B
:1065E000CA94C20CC652DF4FE880F9800A811B8131
:1065F000CA5DD040CE52DF4F2881C25DD040CD521F
:10660000DF4F3881C35DD040CC52DF4F4881C45D3D
:10661000D040CB52DF4F5881C55DD040C253DF4FD1
:106620006881CE5CD040C153DF4F7881CF5CD040D1
:10663000C053DF4F8881C05DD040CF52DF4F98817B
:10664000C15DD0400E94B027C252DF4F2881CE5D8D
:10665000D040222309F4B4C10E94E5C7D62E972E5C
:106660005C0127E330E040E050E00E9452CF0E94FE
:1066700021CC2B013C016D2D792DC50128E631E09F
:1066800040E050E00E9452CF0E9421CC2BED3FE031
:1066900049E450E40E9456CE20E030E044E353E465
:1066A0000E9488CBCA52DF4F688379838A839B8399
:1066B000C65DD040D0FE0DC080E090E0A0E8BFE312
:1066C000CD51DF4F88839983AA83BB83C35ED040BB
:1066D0000CC020E030E040E85FEBCD51DF4F288375
:1066E00039834A835B83C35ED040D12C8D2D90E0EB
:1066F000CF51DF4FE881F981C15ED0408E179F07EF
:106700000CF02CC10E94E5C74B015C0124E130E094
:1067100040E050E00E9452CF0E9421CC9B01AC018E
:10672000CD51DF4F688179818A819B81C35ED040E2
:106730000E9456CE2BED3FE049E450E40E9456CE35
:1067400020E030E044E353E40E9488CB9B01AC019D
:10675000CA52DF4F688179818A819B81C65DD040B2
:106760000E94A8CACA52DF4F688379838A839B83B9
:10677000C65DD040C501B4012AE030E040E050E001
:106780000E9452CF65507109810991090E9421CC64
:106790009B01AC01C301B2010E94A8CA2B013C01BC
:1067A00020E030E0A9010E9481CB87FF04C077FA86
:1067B000709477F87094CA52DF4F688179818A812A
:1067C0009B81C65DD0400E9485CBA30192010E94AF
:1067D00056CE9B01AC01C253DF4F6881CE5CD040E6
:1067E000C153DF4F7881CF5CD040C053DF4F8881E9
:1067F000C05DD040CF52DF4F9881C15DD0400E9434
:10680000A8CAC753DF4F688379838A839B83C95C97
:10681000D04020E030E0A9010E9481CB87FD1DC05F
:1068200020E030E04CE553E4C753DF4F68817981C5
:106830008A819B81C95CD0400E9484CD1816ACF43B
:1068400080E090E0ACE5B3E4C753DF4F88839983E1
:10685000AA83BB83C95CD04008C0C753DF4F1882EE
:1068600019821A821B82C95CD040CA52DF4F6881EC
:1068700079818A819B81C65DD0400E94B9CEA301F7
:1068800092010E9456CE9B01AC01CE52DF4F68812F
:10689000C25DD040CD52DF4F7881C35DD040CC5235
:1068A000DF4F8881C45DD040CB52DF4F9881C55DFA
:1068B000D0400E94A8CA4B015C0120E030E0A90151
:1068C0000E9481CB87FD11C020E030E04CE553E40D
:1068D000C501B4010E9484CD181654F4812C912C6A
:1068E0007CE5A72E73E4B72E03C0812C912C5401B4
:1068F000C353DF4F9881CD5CD0409430C9F4C75367
:10690000DF4F488159816A817B81C95CD0408EE923
:1069100099E00E943024B501A4018AE999E00E941F
:1069200030248091C00085FFFCCFAAE0A093C60070
:10693000C951DF4FE880F9800A811B81C75ED040D2
:10694000A5019401C753DF4F688179818A819B81BA
:10695000C95CD0400E94B027D394C8CEC652DF4F46
:10696000E880F9800A811B81CA5DD040CE52DF4F9A
:106970002881C25DD040CD52DF4F3881C35DD04009
:10698000CC52DF4F4881C45DD040CB52DF4F58819D
:10699000C55DD040C253DF4F6881CE5CD040C1534B
:1069A000DF4F7881CF5CD040C053DF4F8881C05D1E
:1069B000D040CF52DF4F9881C15DD0400E94B027B8
:1069C000C451DF4FF881CC5ED040FF2331F068EE38
:1069D00073E080E090E00E9414C80E94D0230E94DF
:1069E0002D2A8091330790913407A0913507B091FB
:1069F0003607C152DF4FE881F981CF5DD0408193E6
:106A00009193A193B193C152DF4FF983E883CF5D96
:106A1000D040D12C812C912C5401E1E0F0E0EC0F1E
:106A2000FD1F24E0D29EE00DF11D11242081318153
:106A300042815381C501B4010E94A8CA4B015C0187
:106A4000D394CD1450F7B101882777FD8095982F06
:106A50000E9423CC2B013C019B01AC01C501B40178
:106A60000E9488CBC753DF4F688379838A839B83D7
:106A7000C95CD040D12C812C912C5401E1E0F0E094
:106A8000EC0FFD1F34E0D39EE00DF11D1124C75320
:106A9000DF4F288139814A815B81C95CD0406081A8
:106AA0007181828193810E94A7CA9B01AC010E94DF
:106AB00056CE9B01AC01C501B4010E94A8CA4B018E
:106AC0005C01D394CD14D0F6A30192010E9488CB2F
:106AD0000E94C3CE2B013C01C353DF4F4881CD5CE4
:106AE000D040423008F418CD4AE050E0B1018CEBC0
:106AF00094E00E94EC22E5E9F9E08491882341F0DA
:106B00009091C00095FFFCCF8093C6003196F5CFE1
:106B1000C551DF4F5881CB5ED040652F70E04AE011
:106B200050E08CEB94E00E94EC22EEE8F9E08491D6
:106B3000882341F09091C00095FFFCCF8093C60060
:106B40003196F5CF40913307509134076091350766
:106B50007091360726E030E08CEB94E00E94BE2373
:106B6000C353DF4F8881CD5CD040823081F1E6E8AD
:106B7000F9E08491882341F09091C00095FFFCCF0B
:106B80008093C6003196F5CF26E030E0C753DF4F43
:106B9000488159816A817B81C95CD0408CEB94E04B
:106BA0000E94BE23EBE7F9E08491882341F09091A5
:106BB000C00095FFFCCF8093C6003196F5CF26E04C
:106BC00030E0B301A2018CEB94E00E94BE238091DF
:106BD000C00085FFFCCF8AE08093C600A4CCC451DE
:106BE000DF4FF881CC5ED040F11106C068EE73E053
:106BF00080E090E00E9414C80E94F223C353DF4F4C
:106C00002881CD5CD040222311F1E4E7F9E08491A2
:106C1000882341F09091C00095FFFCCF8093C6007F
:106C20003196F5CF26E030E0C753DF4F48815981D8
:106C30006A817B81C95CD0408CEB94E00E94BE23CA
:106C40008091C00085FFFCCF8AE08093C600EFE50D
:106C5000F9E08491882341F09091C00095FFFCCF2A
:106C60008093C6003196F5CF26E030E0B301A20153
:106C70008CEB94E00E94BE238091C00085FFFCCF86
:106C80008AE08093C6008091C00085FFFCCF8AE037
:106C90008093C600C451DF4F0FB6F894DEBF0FBE1D
:106CA000CDBFDF91CF911F910F91FF90EF90DF90BB
:106CB000CF90BF90AF909F908F907F906F905F909C
:106CC0004F903F902F90089583E50E94EA268823F5
:106CD00019F00E94DD2601C082E18093350280FF19
:106CE00021C0E7ECFFE08491882341F09091C0003F
:106CF00095FFFCCF8093C6003196F5CFECE4F9E028
:106D00008491882341F09091C00095FFFCCF80933F
:106D1000C6003196F5CF8091C00085FFFCCF8AE098
:106D20008093C6008091350283FF23C0E7ECFFE02B
:106D30008491882341F09091C00095FFFCCF80930F
:106D4000C6003196F5CFE7E3F9E08491882341F05E
:106D50009091C00095FFFCCF8093C6003196F5CF8F
:106D60008091C00085FFFCCF8AE08093C6000C9420
:106D7000809F089583E50E94EA26882349F10E94B6
:106D8000DD26823010F1EDECFFE08491882341F0A4
:106D90009091C00095FFFCCF8093C6003196F5CF4F
:106DA000E2E9F7E08491882341F09091C00095FFDB
:106DB000FCCF8093C6003196F5CF8091C00085FF4F
:106DC000FCCF8AE08093C6000895813009F444C066
:106DD00088E40E94EA26882391F00E94DD268A3A00
:106DE00091053CF0853021E092072CF084E091E0A1
:106DF00002C08AEA90E090931B1380931A1386E4F2
:106E00000E94EA26882381F00E94DD268F3F9105AB
:106E100019F014F08FEF90E097FF02C080E090E04F
:106E2000909317138093161382E40E94EA26882316
:106E300009F454C00E94DD268530910534F08A366D
:106E400091052CF089E690E002C085E090E09093F7
:106E5000191380931813089588E40E94EA26882362
:106E600091F00E94DD268A3A91053CF0853021E0C0
:106E700092072CF084E091E002C08AEA90E09093BF
:106E800015138093141386E40E94EA26882381F068
:106E90000E94DD268F3F910519F014F08FEF90E0EE
:106EA00097FF02C080E090E090931113809310133D
:106EB00082E40E94EA26882389F00E94DD2685303C
:106EC000910534F08A3691052CF089E690E002C0F5
:106ED00085E090E09093131380931213089583E557
:106EE0000E94EA26882399F00E94AC2620E030E038
:106EF0004AE754E40E9456CE0E94F5CB60931502F7
:106F0000709316028093170290931802089588E5F3
:106F10000E94EA26811111C089E50E94EA268111AA
:106F20000CC08AE50E94EA26811107C085E40E9410
:106F3000EA26811102C00C94089A0E948D9988E576
:106F40000E94EA26882319F05F9A1092180789E5B3
:106F50000E94EA26882319F08A9A109219078AE576
:106F60000E94EA26882351F09FB7F8948091080187
:106F70008160809308019FBF10921A0785E40E94E8
:106F8000EA26882311F0129A089508953F924F92AD
:106F90005F926F927F928F929F92AF92BF92CF92A9
:106FA000DF92EF92FF920F931F93CF93DF93C5E190
:106FB0008C2EC4E09C2EC9E0DFE019E1A12E1FE079
:106FC000B12E09EC1EE0312CF40181914F010E9499
:106FD000EA26882309F458C0F3E03F124FC00E940C
:106FE000AC266B017C0120E030E040EA51E40E94D5
:106FF00081CB87FF3EC0A7019601688179818A8194
:107000009B810E9488CB2B013C019B01AC016091CC
:10701000DD0E7091DE0E8091DF0E9091E00E0E94E9
:1070200056CE6093DD0E7093DE0E8093DF0E90934C
:10703000E00EA3019201F50160817181828193814B
:107040000E9456CEF5016083718382839383F80199
:1070500060817181828193810E9421CCA301920180
:107060000E9456CE0E94F5CBF80160837183828323
:107070009383C882D982EA82FB8206C00E94AC2632
:10708000688379838A839B8333942496F4E0AF0EDC
:10709000B11C0C5F1F4F84E0381296CFDF91CF9167
:1070A0001F910F91FF90EF90DF90CF90BF90AF9026
:1070B0009F908F907F906F905F904F903F9008953A
:1070C000EAEFF7E08491882341F09091C00095FFAA
:1070D000FCCF8093C6003196F5CF40912B0750919D
:1070E0002C0760912D0770912E0722E030E08CEB89
:1070F00094E00E94BE23E6EFF7E08491882341F0FC
:107100009091C00095FFFCCF8093C6003196F5CFDB
:1071100040912F07509130076091310770913207ED
:1071200022E030E08CEB94E00E94BE23E2EFF7E037
:107130008491882341F09091C00095FFFCCF80930B
:10714000C6003196F5CF40913307509134076091D6
:1071500035077091360722E030E08CEB94E00E9416
:10716000BE23EEEEF7E08491882341F09091C000B9
:1071700095FFFCCF8093C6003196F5CF409137073D
:10718000509138076091390770913A0722E030E05A
:107190008CEB94E00E94BE23E3EEF7E08491882319
:1071A00041F09091C00095FFFCCF8093C6003196CE
:1071B000F5CF80E090E00E94F299AB01BC0122E0A3
:1071C00030E08CEB94E00E94BE23EFEDF7E0849179
:1071D000882341F09091C00095FFFCCF8093C600BA
:1071E0003196F5CF81E090E00E94F299AB01BC01AD
:1071F00022E030E08CEB94E00E94BE23EBEDF7E060
:107200008491882341F09091C00095FFFCCF80933A
:10721000C6003196F5CF82E090E00E94F299AB0172
:10722000BC0122E030E08CEB94E00E94BE23809110
:10723000C00085FFFCCF8AE08093C6000895EFE58B
:10724000F3E08191882339F09091C00095FFFCCF45
:107250008093C600F6CF8091C00085FFFCCF8AE006
:107260008093C600E3EDF7E08491882341F090918C
:10727000C00095FFFCCF8093C6003196F5CF65998D
:1072800003C0E0E5F3E009C0EAE5F3E006C0909151
:10729000C00095FFFCCF8093C60081918111F7CF8C
:1072A0008091C00085FFFCCF8AE08093C600EBECA4
:1072B000F7E08491882341F09091C00095FFFCCFC6
:1072C0008093C6003196F5CF8091030181FF03C002
:1072D000E0E5F3E009C0EAE5F3E006C09091C00004
:1072E00095FFFCCF8093C60081918111F7CF8091EB
:1072F000C00085FFFCCF8AE08093C600E3ECF7E096
:107300008491882341F09091C00095FFFCCF809339
:10731000C6003196F5CF8091030180FD03C0E0E502
:10732000F3E009C0EAE5F3E006C09091C00095FFE4
:10733000FCCF8093C60081918111F7CF8091C0006E
:1073400085FFFCCF8AE08093C600EBEBF7E08491E9
:10735000882341F09091C00095FFFCCF8093C60038
:107360003196F5CF4B9903C0E0E5F3E009C0EAE5BB
:10737000F3E006C09091C00095FFFCCF8093C6005B
:1073800081918111F7CF8091C00085FFFCCF8AE009
:107390008093C600E3EBF7E08491882341F090915D
:1073A000C00095FFFCCF8093C6003196F5CF4A9977
:1073B00003C0E0E5F3E009C0EAE5F3E006C0909120
:1073C000C00095FFFCCF8093C60081918111F7CF5B
:1073D0008091C00085FFFCCF8AE08093C6000895AD
:1073E00083E50E94EA268823F9F00E94AC26AB01CF
:1073F000BC014093F10E5093F20E6093F30E709324
:10740000F40E4093E90E5093EA0E6093EB0E7093E6
:10741000EC0E8AE697E00E941F248091C00085FF51
:10742000FCCF8AE08093C60080E50E94EA2688238C
:10743000B9F00E94AC26AB01BC014093F10E509311
:10744000F20E6093F30E7093F40E8DE497E00E94B9
:107450001F248091C00085FFFCCF8AE08093C60086
:1074600082E50E94EA268823B9F00E94AC26AB018F
:10747000BC014093ED0E5093EE0E6093EF0E7093AF
:10748000F00E8EE297E00E941F248091C00085FFDD
:10749000FCCF8AE08093C60084E50E94EA26882318
:1074A000B9F00E94AC26AB01BC014093E90E5093A9
:1074B000EA0E6093EB0E7093EC0E80E197E00E9471
:1074C0001F248091C00085FFFCCF8AE08093C60016
:1074D000089583E50E94EA26882351F00E94AC2695
:1074E0006093F50E7093F60E8093F70E9093F80E5E
:1074F00084E50E94EA26882351F00E94AC2660931E
:10750000D90E7093DA0E8093DB0E9093DC0E82E43A
:107510000E94EA26882361F00E94AC260E94F5CBE7
:107520006093290F70932A0F80932B0F90932C0F49
:1075300088E50E94EA26882351F00E94AC266093D9
:10754000E50E7093E60E8093E70E9093E80E8AE5C1
:107550000E94EA26882351F00E94AC266093E10E37
:107560007093E20E8093E30E9093E40E85E40E9404
:10757000EA26882351F00E94AC266093DD0E7093BA
:10758000DE0E8093DF0E9093E00E089585E40E9456
:10759000EA26811110C080E50E94EA268823A9F01E
:1075A0000E94AC26609381027093820280938302D2
:1075B000909384020AC00E94AC260E94F0CB16165B
:1075C00017064CF7E7ECFFE0D4C089E40E94EA26F6
:1075D000882361F00E94AC260E949EA660937D02E3
:1075E00070937E0280937F029093800284E40E94D5
:1075F000EA26882361F00E94AC260E94AAA6609326
:10760000790270937A0280937B0290937C0283E4E8
:107610000E94EA26882351F00E94AC2660937502EE
:107620007093760280937702909378028CE40E94A4
:10763000EA26882341F00E94AC260E94F0CB70938A
:107640000B0260930A0280910A0290910B02C39789
:1076500034F082E390E090930B0280930A020E9440
:10766000949BE8E7F3E08191882339F09091C00082
:1076700095FFFCCF8093C600F6CFEBE7F3E0819156
:10768000882339F09091C00095FFFCCF8093C6000D
:10769000F6CF4091810250918202609183027091F5
:1076A000840222E030E08CEB94E00E94BE23EFE7FE
:1076B000F3E08191882339F09091C00095FFFCCFD1
:1076C0008093C600F6CF60917D0270917E0280911A
:1076D0007F02909180020E94A4A6AB01BC0122E02F
:1076E00030E08CEB94E00E94BE23E3E8F3E081916C
:1076F000882339F09091C00095FFFCCF8093C6009D
:10770000F6CF6091790270917A0280917B0290911C
:107710007C020E94B0A6AB01BC0122E030E08CEB01
:1077200094E00E94BE23E7E8F3E08191882339F0DA
:107730009091C00095FFFCCF8093C600F6CF40919A
:10774000750250917602609177027091780222E082
:1077500030E08CEB94E00E94BE238091C00085FF56
:10776000FCCF1AC09091C00095FFFCCF8093C6005B
:10777000319684918111F6CFEBE8F3E08191882373
:1077800039F09091C00095FFFCCF8093C600F6CFF2
:107790008091C00085FFFCCF8AE08093C6000895E9
:1077A0000F931F93CF93DF9385E40E94EA268823EB
:1077B00021F00E94DD26EC0102C0C0E0D0E083E4AD
:1077C0000E94EA26882321F00E94DD268C0102C057
:1077D00005E010E083E50E94EA26882319F00E9464
:1077E000AC260BC0D7FF05C060E070E08CE892E4E7
:1077F00004C060E070E086E193E49801AE01DF919F
:10780000CF911F910F910C949A9F2F923F924F927C
:107810005F926F927F928F929F92AF92BF92CF9220
:10782000DF92EF92FF920F931F93CF93DF93CDB729
:10783000DEB768970FB6F894DEBF0FBECDBF8CE001
:10784000EBE2F7E0DE01119601900D928A95E1F7E7
:107850008CE0E3E7F5E0DE011D9601900D928A953C
:10786000E1F708E1202E07E0302E4E018DE0880E72
:10787000911CFE0131965F0100E010E0F101819161
:107880001F01882309F484C0F50140805180628083
:107890007380F801E75EFD4F208131814281538181
:1078A000F801E959FA4F60817181828193810E94C8
:1078B000A8CA20E030E040E05FE30E9456CE9B0182
:1078C000AC01C301B2010E9484CD181644F4C80172
:1078D0008D55904F0E94BF236B017C0103C0C12CCA
:1078E000D12C7601A7019601C301B2010E94A7CA5B
:1078F0002B013C0120E030E040EA51EC0E9484CDB5
:1079000018161CF0EDECFFE025C020E030E040EA66
:1079100051E4C301B2010E9481CB87FFF3CFA301E1
:107920009201F40160817181828193810E94A7CAD2
:10793000F4016083718382839383F501C082D182D5
:10794000E282F38225C09091C00095FFFCCF809326
:10795000C600319684918111F6CFE3EFF6E0849171
:10796000882341F09091C00095FFFCCF8093C60022
:107970003196F5CF8091C00085FFFCCF8AE08093DF
:10798000C60085EE96E00E9411AA87ED96E026C01B
:10799000F4E08F0E911C0C5F1F4F84E0A80EB11C09
:1079A0000C30110509F06ACF8CE0FE013196ABE294
:1079B000B7E001900D928A95E1F78CE0FE013D96CB
:1079C000A3E7B5E001900D928A95E1F70E94CE28D9
:1079D00087EC96E00E9411AA89EA96E090935B05F5
:1079E00080935A0568960FB6F894DEBF0FBECDBFE0
:1079F000DF91CF911F910F91FF90EF90DF90CF908B
:107A0000BF90AF909F908F907F906F905F904F90BE
:107A10003F902F900C94C424CF92DF92EF92FF926C
:107A2000E7ECFFE08491882341F09091C00095FF3E
:107A3000FCCF8093C6003196F5CFE0EAF6E0849162
:107A4000882341F09091C00095FFFCCF8093C60041
:107A50003196F5CF8091C00085FFFCCF80E2809306
:107A6000C6008AE50E94EA26882309F457C00E94CE
:107A7000AC266B017C0120E030E040EA51EC0E9432
:107A800084CD87FD0AC020E030E040EA51E4C70120
:107A9000B6010E9481CB18161CF4E5E9F6E01DC082
:107AA000C0920E02D0920F02E0921002F0921102E8
:107AB000EDE9F6E08491882309F43CC09091C00080
:107AC00095FFFCCF8093C6003196F4CF9091C00013
:107AD00095FFFCCF8093C600319684918111F6CF3B
:107AE0004AE050E06CEE7FEF8CEB94E00E94EC22D9
:107AF000EDE8F6E08491882341F09091C00095FF75
:107B0000FCCF8093C6003196F5CF4AE050E064E1A7
:107B100070E08CEB94E00E94EC220CC040910E02CD
:107B200050910F0260911002709111028AE896E064
:107B30000E941F248091C00085FFFCCF8AE08093C3
:107B4000C600FF90EF90DF90CF900895CF92DF9224
:107B5000EF92FF92882361F1E7ECFFE09491992383
:107B600041F02091C00025FFFCCF9093C6003196D4
:107B7000F5CF9091C00095FFFCCF94E59093C6009F
:107B80004AE050E0682F8CEB94E00E942323EBE85E
:107B9000F3E08191882339F09091C00095FFFCCFEC
:107BA0008093C600F6CF8091C00085FFFCCF40C017
:107BB0001092490586E40E94EA26882399F00E94E3
:107BC000AC266B017C0120E030E0A9010E9484CD4D
:107BD000181644F4C0923102D0923202E09233027D
:107BE000F0923402E7ECFFE08491882341F0909119
:107BF000C00095FFFCCF8093C6003196F5CFECE92D
:107C0000F3E08191882339F09091C00095FFFCCF7B
:107C10008093C600F6CF6091660570E04AE050E0C0
:107C20008CEB94E00E94EC228091C00085FFFCCF99
:107C30008AE08093C600FF90EF90DF90CF90089588
:107C40000E94C523E0910A07F0910B07EC5BFA4F05
:107C50008081811114C0EEE7F6E08491882341F021
:107C60009091C00095FFFCCF8093C6003196F5CF70
:107C70008091C00085FFFCCF8AE08093C600089504
:107C80008CEB94E00E942A22E1E8F6E084918823BC
:107C900041F09091C00095FFFCCF8093C6003196D3
:107CA000F5CF409110075091110760911207709124
:107CB00013074F5F5F4F6F4F7F4F2AE030E08CEB31
:107CC00094E00E94C9228091C00085FFFCCF8AE029
:107CD0008093C600B5CFCF93C62FEDECFFE0249183
:107CE000222379F03091C00035FFFCCF2093C600ED
:107CF0003196F5CF3091C00035FFFCCF2093C60000
:107D00000196FC0124912111F5CF4091100750916B
:107D1000110760911207709113072AE030E08CEB95
:107D200094E00E94C9228091C00085FFFCCF8AE0C8
:107D30008093C600C111A4DF1092600510925F0508
:107D4000CF9108958F929F92AF92BF92CF92DF9280
:107D5000EF92FF92CF93DF93EC01C0906705D09034
:107D60006805E0906905F0906A05A70196016881B1
:107D700079818A819B810E9481CB87FF04C0C88260
:107D8000D982EA82FB82C0906B05D0906C05E090AE
:107D90006D05F0906E05A70196016C817D818E8145
:107DA0009F810E9481CB87FF04C0CC82DD82EE825E
:107DB000FF82C0900E02D0900F02E0901002F0906F
:107DC000110220E030E0A901C701B6010E9481CB79
:107DD00087FF0AC020E030E0A901C701B6010E9478
:107DE000A8CA6B017C0103C0C12CD12C7601809004
:107DF0007B0590907C05A0907D05B0907E0520E0ED
:107E000030E0A901C501B4010E9481CB87FF08C001
:107E1000A5019401C701B6010E94A8CA6B017C01AB
:107E200020916F0530917005409171055091720558
:107E3000C701B6010E94A8CA6B017C019B01AC017D
:107E4000688579858A859B850E9481CB87FF04C0E0
:107E5000C886D986EA86FB86C0901902D0901A029D
:107E6000E0901B02F0901C02A701960168817981C5
:107E70008A819B810E9484CD181624F4C882D982FD
:107E8000EA82FB82C0901D02D0901E02E0901F0289
:107E9000F0902002A70196016C817D818E819F81E7
:107EA0000E9484CD181624F4CC82DD82EE82FF82FB
:107EB000C0902102D0902202E0902302F090240290
:107EC000A7019601688579858A859B850E9484CD66
:107ED000181624F4C886D986EA86FB86DF91CF91EE
:107EE000FF90EF90DF90CF90BF90AF909F908F90DA
:107EF00008958F929F92AF92BF92CF92DF92EF92AE
:107F0000FF920F931F93CF93DF93EC018B0180912E
:107F1000350283FD90C0FB0180809180A280B380F8
:107F2000288139814A815B81C501B4010E94A7CAB9
:107F30006B017C0120E030E0A9010E9481CB882305
:107F400009F479C0E091660524E0E29FF001112474
:107F5000E256FD4E20910602309107024091080240
:107F60005091090260817181828193810E9481CB4D
:107F700087FF25C088829982AA82BB82E7ECFFE056
:107F80008491882341F09091C00095FFFCCF8093AD
:107F9000C6003196F5CFE4E6F6E08491882341F0FF
:107FA0009091C00095FFFCCF8093C6003196F5CF2D
:107FB0008091C00085FFFCCF8AE08093C600C70196
:107FC000B6010E94F0CB97FF07C090958095709501
:107FD00061957F4F8F4F9F4F693B714081059105A0
:107FE00054F1F80180819181A281B38188839983C2
:107FF000AA83BB83E7ECFFE08491882341F0909152
:10800000C00095FFFCCF8093C6003196F5CFE6E423
:10801000F6E08491882341F09091C00095FFFCCF59
:108020008093C6003196F5CF8091C00085FFFCCFCC
:108030008AE08093C600DF91CF911F910F91FF904E
:10804000EF90DF90CF90BF90AF909F908F9008956A
:108050008BE197E077DE0E94C52367E277E087E354
:1080600097E047DF20911B0730911C0740911D07C7
:1080700050911E0760912B0770912C0780912D075E
:1080800090912E070E9481CB811117C020911F076C
:1080900030912007409121075091220760912F07CE
:1080A0007091300780913107909132070E9481CB07
:1080B000811103C00E94C5281CC060912F027091DD
:1080C0003002882777FD8095982F0E9423CC20913D
:1080D00031023091320240913302509134020E94B9
:1080E00056CE20E030E048EC52E40E9488CB0E945B
:1080F00086280C94A82A2F923F924F925F926F92FB
:108100007F928F929F92AF92BF92CF92DF92EF9227
:10811000FF920F931F93CF93DF93CDB7DEB7C65473
:10812000D1090FB6F894DEBF0FBECDBF1C017EA7EC
:108130006DA7142FDB0114968D909D90AD90BC908F
:108140001797CD90DD90ED90FC90A5019401C701AB
:10815000B6010E9491CD23966CAF7DAF8EAF9FAFDD
:10816000239780912B0790912C07A0912D07B09118
:108170002E078D8F9E8FAF8FB8A3A7019601BC01EC
:10818000CD010E94A8CA6FAB78AF89AF9AAF80913A
:108190002F0790913007A0913107B091320789A342
:1081A0009AA3ABA3BCA3A5019401BC01CD010E947D
:1081B000A8CA6BAF7CAF8DAF9EAF80913307909113
:1081C0003407A0913507B09136078D8B9E8BAF8B0E
:1081D000B88F9C01AD01D10118966D917D918D9163
:1081E0009C911B970E94A7CA6DA37EA38FA398A7FB
:1081F000D1011C968D919D910D90BC91A02D27963B
:108200008CAF9DAFAEAFBFAF2797809137079091EE
:108210003807A0913907B0913A0789A79AA7ABA769
:10822000BCA7D701C601B058898F9A8FAB8FBC8F7E
:10823000D501C401B058898B9A8BAB8BBC8BD10113
:108240008D919D910D90BC91A02D8FA798ABA9AB5E
:10825000BAAB2FA938AD49AD5AADBC01CD010E94D2
:10826000A7CA6B017C01D10114968D919D910D904F
:10827000BC91A02D8BAB9CABADABBEAB2BAD3CADE5
:108280004DAD5EADBC01CD010E94A7CA4B015C01A2
:10829000A7019601698D7A8D8B8D9C8D0E9456CE9B
:1082A0002B013C01A501940169897A898B899C89FC
:1082B0000E9456CE9B01AC01C301B2010E94A8CA24
:1082C0002B013C01A5019401698D7A8D8B8D9C8DCC
:1082D0000E9456CE4B015C01A701960169897A89FB
:1082E0008B899C890E9456CE9B01AC01C501B401CB
:1082F0000E94A7CAA30192010E941BCB6B017C01C3
:1083000020E030E0A9010E9481CB87FF0AC02BED5D
:108310003FE049EC50E4C701B6010E94A8CA6B01D6
:108320007C01112351F02BED3FE049EC50E4C701F3
:10833000B6010E94A7CA6B017C012FA538A949A9E3
:108340005AA96D8D7E8D8F8D98A10E9481CB811150
:108350001FC02BA93CA94DA95EA969A17AA18BA137
:108360009CA10E9481CB811113C020E030E0A901C3
:10837000C701B6010E9481CB81110AC02BED3FE0FD
:1083800049EC50E4C701B6010E94A8CA6B017C0108
:1083900023962CAD3DAD4EAD5FAD2397C701B60121
:1083A0000E9456CE2DA13EA14FA158A55F770E94F5
:1083B00091CD4B015C012FE632E143E85AE30E9484
:1083C00081CB87FDC2C1C501B4010E945ECC0E9471
:1083D000F5CB7E8F6D8FFB01EF2B21F421E030E098
:1083E0003E8F2D8FAD8DBE8DBD0180E090E00E944F
:1083F00021CC4B015C019B01AC01C701B6010E947D
:1084000088CB2B013C01A50194016DA17EA18FA118
:1084100098A50E9488CB6FA778AB89AB9AAB29A5AA
:108420003AA54BA55CA527966CAD7DAD8EAD9FADF5
:1084300027970E94A7CAA50194010E9488CB6BAB25
:108440007CAB8DAB9EAB20E030E040E05FE3C3014E
:10845000B2010E9456CEA30192010E9456CE9B010A
:10846000AC0160E070E080E89FE30E94A7CA6DA3C2
:108470007EA38FA398A78D899E89AF89B88D8987A0
:108480009A87AB87BC8789A59AA5ABA5BCA58D8724
:108490009E87AF87B88B60912F027091300288273A
:1084A00077FD8095982F0E9423CC20913102309146
:1084B000320240913302509134020E9456CE20E0A5
:1084C00030E040E752E40E9488CB20E030E048EC06
:1084D00052E40E9488CB69A77AA78BA79CA71D8A24
:1084E000A1E0B0E0BAA3A9A389A19AA1AD8DBE8DE8
:1084F0008A179B0708F00CC1BD89B9310CF042C046
:108500002DA13EA14FA158A569897A898B899C89A3
:108510000E9456CE6B017C01A3019201698D7A8D78
:108520008B8D9C8D0E9456CEA70196010E94A8CAF1
:108530006B017C012DA13EA14FA158A5698D7A8DBB
:108540008B8D9C8D0E9456CE4B015C01A301920144
:1085500069897A898B899C890E9456CE9B01AC01DE
:10856000C501B4010E94A7CA698F7A8F8B8F9C8F37
:10857000ED89EF5FED8BA601B701498B5A8B6B8BB1
:108580007C8B6BC029A13AA1B90180E090E00E94E8
:1085900021CCA30192010E9456CE6B017C010E9466
:1085A00085CB698B7A8B8B8B9C8BC701B6010E9424
:1085B000B9CE4B015C01ADA5BEA5CD90DD90ED908F
:1085C000FC901397F7FAF094F7F8F09414968D91C5
:1085D0009D910D90BC91A02D8D8B9E8BAF8BB88FF4
:1085E00029893A894B895C89C701B6010E9456CE18
:1085F000698F7A8F8B8F9C8FA50194016D897E89FD
:108600008F89988D0E9456CE9B01AC01698D7A8D21
:108610008B8D9C8D0E94A8CA698F7A8F8B8F9C8FBF
:10862000A5019401C701B6010E9456CE6B017C01E1
:1086300029893A894B895C896D897E898F89988DD2
:108640000E9456CE9B01AC01C701B6010E94A7CA89
:10865000698B7A8B8B8B9C8B1D8A298D3A8D4B8DE8
:108660005C8D6FA978AD89AD9AAD0E94A8CA698367
:108670007A838B839C8329893A894B895C896BAD8A
:108680007CAD8DAD9EAD0E94A8CA6D837E838F8325
:1086900098872FA538A949A95AA969857A858B8514
:1086A0009C850E94A8CA69877A878B879C872BA99B
:1086B0003CA94DA95EA96D857E858F8598890E940C
:1086C000A8CA6D877E878F87988BCE0101963ADB8B
:1086D000E984FA840B851C852D813E814F81588564
:1086E00069817A818B819C81E0916605EF9389A4F1
:1086F0009AA4ABA4BCA4FE013D966F010E941C612C
:1087000029A13AA12F5F3F4F3AA329A30F90ECCEA6
:108710006101BCE0CB0ED11CF101E084F184028543
:1087200013852481358146815781608171818281E1
:108730009381E0916605EF9389A49AA4ABA4BCA4AD
:108740000E941C610E94A82A0F90CA5BDF4F0FB6DF
:10875000F894DEBF0FBECDBFDF91CF911F910F9177
:10876000FF90EF90DF90CF90BF90AF909F908F9051
:108770007F906F905F904F903F902F9008951F9340
:10878000CF93DF93CDB7DEB728970FB6F894DEBF4F
:108790000FBECDBF182F80913602882349F10E9469
:1087A000B22A89E40E94EA26882319F00E94AC26A6
:1087B00003C060E070E0CB0169837A838B839C8384
:1087C0008AE40E94EA26882319F00E94AC2603C09E
:1087D00060E070E0CB016D837E838F839887412FAB
:1087E000BE016F5F7F4F8BE197E085DC0E94C52360
:1087F00028960FB6F894DEBF0FBECDBFDF91CF91A4
:108800001F9108955F988A989FB7F894E8E0F1E087
:1088100080818E7F80839FBF129808955F9A109207
:1088200018078A9A109219079FB7F894E8E0F1E0C8
:108830008081816080839FBF10921A07129A0895E9
:108840000E9411AAF8940E94809FE8DF60E08CE00B
:108850000E94BCC9EDECFFE08491882341F0909127
:10886000C00095FFFCCF8093C6003196F5CFE5E1BF
:10887000F6E08491882341F09091C00095FFFCCFF1
:108880008093C6003196F5CF8091C00085FFFCCF64
:108890008AE08093C6007894C6E0D0E0219749F042
:1088A00068EC70E080E090E00E9414C80E9486AA04
:1088B000F5CFF894FFCF2F923F924F925F926F9235
:1088C0007F928F929F92AF92BF92CF92DF92EF9260
:1088D000FF920F931F93CF93DF93CDB7DEB76E97C1
:1088E0000FB6F894DEBF0FBECDBF0E94C424811125
:1088F000D6C230E6932E44E0A42EB12C5AE0752E59
:1089000066246394209106073091070724303105CF
:108910007CF480913D0590913E0540913F0550913A
:108920004005841B950B8F779927892B09F044C04C
:1089300080914107882309F4B2C280915F0590912C
:108940006005892B09F0ABC2232B11F4109243056B
:1089500098EE292E93E0392E412C512C2CE3C22E77
:10896000D12CE12CF12C8E010F5F1F4F80E6682E79
:10897000772473944091C2095091C3096091C4094E
:108980007091C5098091BA099091BB09A091BC0969
:10899000B091BD09481759076A077B0708F07FC2E5
:1089A000809106079091070704970CF078C2809198
:1089B0004305811174C253C18CEB94E00E940E22D6
:1089C0008093610520915F05309160058A3031F018
:1089D0008D3021F02F3531050CF4FCC010925E056E
:1089E0002115310509F45BC2409108075091090730
:1089F000949EC001959E900D11248A579A4FFC01B8
:108A0000E20FF31F1082FA01EC5BFA4F10828C0127
:108A1000DC012C9101962032D1F378012E3411F033
:108A200000E010E06AE270E0C7010E94D7D26C015A
:108A30000115110509F477C062E87EE0C7010E94C4
:108A400089D288248394892B11F4812C09C06EE487
:108A500070E0C70104960E94D7D2009709F08C01FC
:108A60004AE050E060E070E0C80101960E9421D128
:108A70006093140770931507809316079093170758
:108A80002091100730911107409112075091130760
:108A90002F5F3F4F4F4F5F4F621773078407950754
:108AA00031F0811004C061E08FE49EE022C0C11467
:108AB000D10409F180E010E0F701E80FF11D908189
:108AC0009A3219F08F5F1927F7CF4AE050E060E043
:108AD00070E0C60101960E9421D1012F10E020E034
:108AE00030E0601771078207930761F061E080E36F
:108AF0009EE0F1D8D4C10E151F0521F461E086E097
:108B00009EE0F7CF8091140790911507A09116076A
:108B1000B09117078093100790931107A093120745
:108B2000B093130706C0009721F060E08CED9DE044
:108B3000E0CF80913602811129C067E470E0C7015F
:108B40000E94D7D2009711F14AE050E060E070E057
:108B500001960E9421D164307105C0F4E6E6FDE083
:108B60008491882341F09091C00095FFFCCF8093C1
:108B7000C6003196F5CF8091C00085FFFCCF709282
:108B8000C60060E08CE59DE00E94F9A96EEA73E002
:108B9000C7010E94E2D2892B19F483E59DE050DEE3
:108BA00080910807909109070196B5010E943FCF77
:108BB0009093090780930807809106079091070713
:108BC0000196909307078093060710926005109214
:108BD0005F0598CE8C3529F580913D0590913E0535
:108BE00020913F0530914005821B930B8F77992789
:108BF000892B09F487CE8091060790910707049787
:108C00000CF080CE8CEB94E00E940E2280936105E4
:108C1000409108075091090720915F053091600548
:108C20000CC08B3311F460925E0590915E0591113A
:108C300069CE4091080750910907B9016F5F7F4FD6
:108C40007093600560935F05949EF001959EF00D12
:108C50001124E20FF31FEA57FA4F808353CE80911D
:108C6000150990911609A0911709B09118098093E0
:108C7000C2099093C309A093C409B093C5098DE0BC
:108C800099E00E94F485482F809361058A30B1F005
:108C90004D30A1F0433211F04A3321F420915E05AA
:108CA000222361F020915F05309160052F35310559
:108CB0002CF48F3FBFEF9B0709F0D3C04091C2094E
:108CC0005091C3096091C4097091C5098091BA0996
:108CD0009091BB09A091BC09B091BD0948175907F3
:108CE0006A077B0708F481C0E0E4FDE084918823F3
:108CF00041F09091C00095FFFCCF8093C600319663
:108D0000F5CF8091C00085FFFCCFEAE0E093C6007C
:108D10000E94E5C760934A0570934B0580934C050C
:108D200090934D0580904E0590904F05A090500572
:108D3000B0905105681979098A099B09A20191012E
:108D40000E9452CF49015A01CA01B901A7019601F7
:108D50000E9452CFCA01B901A70196010E9452CFC9
:108D60007F936F93C501B40120E13EE040E050E005
:108D70000E9452CF3F932F93ACE2BDE0BF93AF93DD
:108D80001F930F930E940FD30FB6F894DEBF0FBE50
:108D9000CDBFE7ECFFE08491882341F09091C000C3
:108DA00095FFFCCF8093C6003196F5CFF8018191F5
:108DB000882339F09091C00095FFFCCF8093C600C6
:108DC000F6CF8091C00085FFFCCF9AE09093C6005B
:108DD00061E0C8010E94AFA98FE397E00E946D1B7C
:108DE00061E08FE397E00E94C015809161058332B6
:108DF00011F47092430520915F05309160052115B3
:108E0000310519F410925E054AC0809108079091CF
:108E10000907689EF001699EF00D1124E20FF31F0F
:108E2000EA57FA4F1082FC01EC5BFA4F70822091F6
:108E30000607309107072F5F3F4F309307072093B6
:108E40000607019664E070E00E943FCF9093090707
:108E50008093080710925E051092600510925F05DE
:108E600089CD4B3311F470925E0540915E0541113E
:108E70007DCD4091080750910907B9016F5F7F4F81
:108E80007093600560935F05649EF001659EF00D30
:108E90001124E20FF31FEA57FA4F80836BCD6E96D1
:108EA0000FB6F894DEBF0FBECDBFDF91CF911F91FB
:108EB0000F91FF90EF90DF90CF90BF90AF909F9079
:108EC0008F907F906F905F904F903F902F9008957C
:108ED000CF92DF92EF92FF920F931F93CF93C82F01
:108EE000809106079091070703970CF4E4DC0E9439
:108EF000E5C7C0905205D0905305E0905405F0901E
:108F00005505C114D104E104F104A1F00091560506
:108F10001091570520915805309159050C0D1D1DD4
:108F20002E1D3F1D061717072807390718F48DE374
:108F300096E03DC0C0901502D0901602E090170256
:108F4000F0901802C114D104E104F104B9F00091C9
:108F500056051091570520915805309159050C0D73
:108F60001D1D2E1D3F1D061717072807390730F452
:108F7000C11104C08091F7098091F60980914105E3
:108F800090914205909902C0019604C018161906E6
:108F90002CF40197909342058093410580914105FF
:108FA000909142058E3E92401CF084E396E048DCAE
:108FB000CF911F910F91FF90EF90DF90CF900C9485
:108FC000FF600E940E9E80E083DF0C9486AA8F9241
:108FD0009F92AF92BF92CF92DF92EF92FF9280E585
:108FE0000E94EA26882329F00E94D2264B015C01C8
:108FF00003C0812C912C540183E50E94EA2688232A
:1090000061F00E94AC2620E030E04AE754E40E9480
:1090100056CE0E94F5CB4B015C010E948D990E94B7
:10902000C523C0905605D0905705E0905805F090A4
:109030005905C80CD91CEA1CFB1C0E94A8A9811167
:1090400005C060E08DEE9CE00E94F9A90E94E5C792
:109050006C157D058E059F0510F4B3DFF7CFFF90EB
:10906000EF90DF90CF90BF90AF909F908F9008953A
:109070002F923F924F925F926F927F928F929F9228
:10908000AF92BF92CF92DF92EF92FF920F931F9316
:10909000CF93DF93CDB7DEB7CB58D1090FB6F89495
:1090A000DEBF0FBECDBF2DB73EB7E9963FAF2EAFA7
:1090B000E99780911807882321F080911907811181
:1090C00024C060E084E79CE00E94F9A9E7ECFFE09F
:1090D0008491882341F09091C00095FFFCCF80934C
:1090E000C6003196F5CFE2E6FCE08491882341F09A
:1090F0009091C00095FFFCCF8093C6003196F5CFCC
:109100008091C00085FFFCCF29C086E50E94EA2639
:10911000882339F00E94DD266F969FAF8EAF6F9740
:1091200006C041E050E06F965FAF4EAF6F976F960D
:109130008EAD9FAD6F970597B0F0EBE3FCE08491A7
:10914000882341F09091C00095FFFCCF8093C6002A
:109150003196F5CF8091C00085FFFCCF8AE08093E7
:10916000C6000C94D05084E40E94EA26AA968FAFE1
:10917000AA9785E40E94EA266F96AEADBFAD6F97C1
:1091800013976CF484E50E94EA26EE968FAFEE9773
:109190006F96EEADFFAD6F97EF2B59F104C0F1E084
:1091A000EE96FFAFEE97E4E2FCE08491882341F075
:1091B0009091C00095FFFCCF8093C6003196F5CF0B
:1091C000AA962FADAA972223A1F0ECE0FCE08491AF
:1091D000882341F09091C00095FFFCCF8093C6009A
:1091E0003196F5CF8091C00085FFFCCF8AE0809357
:1091F000C60080E50E94EA268823A1F00E94DD26B1
:109200001C01823091058CF4E4EDFBE0849188230D
:1092100009F4C6C79091C00095FFFCCF8093C600AB
:109220003196F4CF72E0272E312C83E50E94EA2696
:10923000882319F00E94DD2602C088EB9BE0909302
:109240001302809312028CE40E94EA26882339F0EC
:109250000E94DD266D969FAF8EAF6D9706C04AE0E7
:1092600050E06D965FAF4EAF6D9782E50E94EA26A3
:10927000882321F00E94DD267C0103C06FEAE62EE0
:10928000F12C86E40E94EA26882321F00E94DD2644
:109290008C0102C00AE010E082E40E94EA268823E2
:1092A00021F00E94DD266C0103C058ECC52ED12CA4
:1092B0006D968EAD9FAD6D9731E097FD0AC0C701E9
:1092C00009976D96AEADBFAD6D97A817B9070CF4B1
:1092D00030E021E0BDEDEB16F1044CF46D968EAD5F
:1092E0009FAD6D9709968E159F050CF420E0AA247A
:1092F000A39417FD06C0C6010997081719070CF4B7
:10930000A12CBB24B394EDEDCE16D10434F4C801E6
:1093100009968C159D050CF4B12C31110CC022233B
:1093200029F085EC9BE00E94062D15C0A11013C00A
:10933000B11017C01EC08DEC9BE0C557DF4F2883CE
:10934000CB58D0400E94062DC557DF4F2881CB58FF
:10935000D0402111E6CFAA2021F08DEB9BE00E94A6
:10936000062DBB2009F41CC786EB9BE00E94062D4E
:1093700017C70E948D99AA96FFADAA97F1112EC02A
:1093800083E492E00E9498C1CE0101960E94B76DDD
:1093900089819A81AB81BC8180932B0790932C07A4
:1093A000A0932D07B0932E078D819E81AF81B88544
:1093B00080932F0790933007A0933107B093320723
:1093C00089859A85AB85BC85809333079093340754
:1093D000A0933507B09336070E94CE280E94D02371
:1093E00080E090E0A0E7B3E48093310290933202F2
:1093F000A0933302B0933402910121503109659654
:109400003FAF2EAF6597C7016D964EAD5FAD6D97BF
:10941000841B950BB9010E943FCFC258DF4F79835F
:109420006883CE57D040229CC001239C900D900DA4
:109430001124A3969FAF8EAFA397880F991FE5962F
:109440009FAF8EAFE597A396AEADBFADA3978A0F42
:109450009B1F880F991F880F991FEDB7FEB7E81B58
:10946000F90B0FB6F894FEBF0FBEEDBF2DB73EB798
:109470002F5F3F4FA7963FAF2EAFA797AA0FBB1FF7
:10948000AA0FBB1FED96BFAFAEAFED974DB75EB75E
:109490004A1B5B0B0FB6F8945EBF0FBE4DBF8DB776
:1094A0009EB70196AC969FAF8EAFAC97ADB7BEB7E7
:1094B000A396EEADFFADA397AE1BBF0B0FB6F8940E
:1094C000BEBF0FBEADBF2DB73EB72F5F3F4FE79674
:1094D0003FAF2EAFE797322D3170E3963FAFE39762
:1094E000C601801B910B65966EAD7FAD65970E949E
:1094F0003FCFCC57DF4F79836883C458D040E29682
:109500001FAF0EAFE2972CEFE5964EAD5FADE5973E
:109510002403C001259F900D1124C058DF4F99836B
:109520008883C058D040A5961FAE1EAEA5976996F9
:109530001FAE1EAE6997812C912C5401E296AEAD00
:10954000BFADE297BD01882777FD8095982F0E94D7
:1095500023CC2B013C01E396BFADE397BB2379F00D
:10956000EB963FAE2EAEEB97E1E0F0E0A996FFAFB1
:10957000EEAFA9976B961FAE1EAE6B9714C06596A3
:109580002EAD3FAD65976B963FAF2EAF6B974FEF0C
:109590005FEFA9965FAF4EAFA9978FEF9FEFEB9666
:1095A0009FAF8EAFEB9781E0E3969FADE39798274F
:1095B000E3969FAFE3976996AEADBFAD6997E59629
:1095C000EEADFFADE597AE0FBF1FAA0FBB1FAA0FF1
:1095D000BB1FA7962EAD3FADA7972A0F3B1F6796DF
:1095E0003FAF2EAF6797A9968EAD9FADA997C25892
:1095F000DF4FA881B981CE57D0408A9FA0018B9FB1
:10960000500D9A9F500D1124CE57DF4F5983488338
:10961000C258D0406B962EAD3FAD6B972A9FF0019C
:109620002B9FF00D3A9FF00D11246D964EAD5FAD5E
:109630006D974E0F5F1FA1965FAF4EAFA197E79654
:109640008EAD9FADE797A596AEADBFADA5978A0F3E
:109650009B1FCA57DF4F99838883C658D0406B96AB
:109660008EAD9FAD6B97EB96AEADBFADEB978A1706
:109670009B0709F436C1A196EEADFFADA197BF01DE
:10968000882777FD8095982F0E9423CCE0966CAFB9
:109690007DAF8EAF9FAFE09769962EAD3FAD6997D6
:1096A000232B89F020E030E040EA50E4609133075A
:1096B0007091340780913507909136070E94A8CAAF
:1096C0007B018C0104C0E12CF12C00E711E4209116
:1096D0002F07309130074091310750913207609148
:1096E0002B0770912C0780912D0790912E070E94D7
:1096F000B027E0903307F0903407009135071091C0
:109700003607A3019201E0966CAD7DAD8EAD9FADA5
:10971000E0970E94B0270E942D2AC0903307D09076
:109720003407E0903507F09036076F964EAD5FAD89
:109730006F97433051050CF44AC0EEEDFAE0849186
:10974000882341F09091C00095FFFCCF8093C60024
:109750003196F5CF23E030E0E0964CAD5DAD6EADD7
:109760007FADE0978CEB94E00E94BE23E9EDFAE038
:109770008491882341F09091C00095FFFCCF8093A5
:10978000C6003196F5CF23E030E0B301A2018CEBA7
:1097900094E00E94BE23E4EDFAE08491882341F036
:1097A0009091C00095FFFCCF8093C6003196F5CF15
:1097B00023E030E0B701A6018CEB94E00E94BE23C9
:1097C0008091C00085FFFCCF5AE05093C600A701EE
:1097D0009601C501B4010E94A8CA4B015C016996BB
:1097E000EEADFFAD6997EE0FFF1FEE0FFF1FAC96BA
:1097F0008EAD9FADAC97E80FF91FC082D182E28297
:10980000F3826796EEADFFAD6797C058DF4FA88132
:10981000B981C058D040EA0FFB1FE0962CAD3DAD9A
:109820004EAD5FADE0972083318342835383ED9645
:109830004EAD5FADED97E40FF51F4082518262821D
:1098400073826796EEADFFAD679780E090E0A0E889
:10985000BFE381939193A193B1936796FFAFEEAF6E
:1098600067976B962EAD3FAD6B97229DF001239DC0
:10987000F00D329DF00D1124CA57DF4F48815981F8
:10988000C658D040E40FF51F68965FAD68975083C7
:1098900069968EAD9FAD6997019669969FAF8EAF21
:1098A00069978FDB6B96AEADBFAD6B97A996EEADAA
:1098B000FFADA997AE0FBF1F6B96BFAFAEAF6B9753
:1098C000A1962EAD3FADA197CE57DF4F488159816C
:1098D000C258D040240F351FA1963FAF2EAFA1979D
:1098E000BECEA596EEADFFADA5973196A596FFAF7E
:1098F000EEAFA597E2962EAD3FADE297CC57DF4F86
:1099000048815981C458D040240F351FE2963FAF9B
:109910002EAFE297E215F3050CF410CE0E94F2236D
:10992000AC960EAD1FADAC97A7962EAD3FADA797E9
:1099300043E050E0A3966EAD7FADA397CE0149966C
:109940000E948580A396AEADBFADA397BD018827C9
:1099500077FD8095982F0E9423CC9B01AC01C50117
:10996000B4010E9488CB4B015C016F96EEADFFAD58
:109970006F97EF2B09F46FC0E0EAFBE08491882336
:1099800041F09091C00095FFFCCF8093C6003196C6
:10999000F5CF498D5A8D6B8D7C8D28E030E08CEBB6
:1099A00094E00E94BE23EBE9FBE08491882341F020
:1099B0009091C00095FFFCCF8093C6003196F5CF03
:1099C0004D8D5E8D6F8D78A128E030E08CEB94E0BA
:1099D0000E94BE23E6E9FBE08491882341F0909148
:1099E000C00095FFFCCF8093C6003196F5CF49A10A
:1099F0005AA16BA17CA128E030E08CEB94E00E949E
:109A0000BE238091C00085FFFCCF8AE08093C60012
:109A10006F962EAD3FAD6F9723303105E4F0EDE743
:109A2000FBE08491882341F09091C00095FFFCCF2A
:109A30008093C6003196F5CF28E030E0B501A4014F
:109A40008CEB94E00E94BE238091C00085FFFCCF88
:109A50008AE08093C600AA963FADAA9731115DC0F7
:109A60000D8D1E8D2F8D38A13058498D5A8D6B8DDF
:109A70007C8D7058C12CD12CE0E8EE2EEFE3FE2E49
:109A8000CE010D960E9450BF63EB73E0CE010D96A0
:109A90000E94CDC0CD84DE84EF84F88809891A89BC
:109AA0002B893C894D895E896F89788DCE01899695
:109AB0000E94C2C184E2FE01B996A3E4B2E0019023
:109AC0000D928A95E1F7CE0101960E94B76D8981CA
:109AD0009A81AB81BC8180932B0790932C07A09334
:109AE0002D07B0932E078D819E81AF81B88580931D
:109AF0002F0790933007A0933107B09332078985E1
:109B00009A85AB85BC858093330790933407A093E7
:109B10003507B09336070E94CE28EE964FADEE97EC
:109B2000442309F485C2E2E6FBE08491882341F0F6
:109B30009091C00095FFFCCF8093C6003196F5CF81
:109B4000E3E5FBE08491882341F09091C00095FF0C
:109B5000FCCF8093C6003196F5CFE4E4FBE084911E
:109B6000882341F09091C00095FFFCCF8093C60000
:109B70003196F5CFE5E3FBE08491882341F09091A5
:109B8000C00095FFFCCF8093C6003196F5CFE6E28A
:109B9000FBE08491882341F09091C00095FFFCCFB9
:109BA0008093C6003196F5CFE7E1FBE084918823EE
:109BB00041F09091C00095FFFCCF8093C600319694
:109BC000F5CF65960EAD1FAD6597F12CB0ECEB2E81
:109BD00089E7D82E94E4C92ECE0101962F969FAF27
:109BE0008EAF2F97DE011D966196BFAFAEAF619726
:109BF000FE01B5966396FFAFEEAF63976896FFAE32
:109C000068976A96EFAE6A976C96DFAE6C97A096EF
:109C1000CFAEA09767961FAE1EAE6797E7964EAD84
:109C20005FADE797400F511FA9965FAF4EAFA99761
:109C300067962EAD3FAD6797229DF001239DF00DF5
:109C4000329DF00D1124A9964EAD5FADA997E40F9A
:109C5000F51FE080FF24E7FCF0946701CC0CDD1CCD
:109C6000CC0CDD1CAC968EAD9FADAC978C0D9D1DC4
:109C7000A5969FAF8EAFA597A5019401DC016D91CC
:109C80007D918D919C910E94A7CA2B013C01A796C2
:109C9000EEADFFADA797EC0DFD1D80819181A281F6
:109CA000B3818DA39EA3AFA3B8A7A396EEADFFADDE
:109CB000A397EE0DFF1DEE0FFF1FEE0FFF1FA796E0
:109CC0002EAD3FADA797E20FF31F80819181A28156
:109CD000B3818D879E87AF87B88B19821A821B82CA
:109CE0001C822F963FAD2F973F932E964FAD2E9708
:109CF0004F9361965FAD61975F9360968FAD60976C
:109D00008F9363969FAD63979F936296AFAD629773
:109D1000AF93EDB7FEB7B4970FB6F894FEBF0FBE82
:109D2000EDBFADB7BEB71196E3E4F2E084E2019077
:109D30000D928A95E1F70E942BC129813A814B81CE
:109D40005C81A596AEADBFADA5976D917D918D91CE
:109D50009C910E94A7CAF62EE72ED82EC92EEDB7E9
:109D6000FEB7BA960FB6F894FEBF0FBEEDBF689669
:109D70002FAD68976A963FAD6A976C964FAD6C971A
:109D8000A0965FADA0970E9481CB87FD0CC068961E
:109D9000FFAC68976A96EFAC6A976C96DFAC6C97ED
:109DA000A096CFACA09720E030E0A901C301B2019A
:109DB0000E9484CD87FD0DC0E4E1FBE084918823FF
:109DC00079F09091C00095FFFCCF8093C60031964A
:109DD000F5CF8091C00085FFFCCFF0E2F093C60084
:109DE00025E030E0B301A2018CEB94E00E94BE2399
:109DF00067962EAD3FAD67972F5F3F4F67963FAF9A
:109E00002EAF6797221533056CF46896FFAE6897FE
:109E10006A96EFAE6A976C96DFAE6C97A096CFAE5F
:109E2000A09706CF8091C00085FFFCCF3AE0309329
:109E3000C6000150110917FFE1CE8091C00085FFD7
:109E4000FCCF8AE08093C6006F968EAD9FAD6F9772
:109E5000049709F0EDC0E9EEFAE08491882341F01F
:109E60009091C00095FFFCCF8093C6003196F5CF4E
:109E7000DE0111962F96BFAFAEAF2F973E01BDE02A
:109E80006B0E711CFE01B5966196FFAFEEAF619748
:109E900000E010E0E7964EAC5FACE79765968EADBC
:109EA0009FAD6597480E591E029DF001039DF00D70
:109EB000129DF00D1124E40DF51D8081992787FD79
:109EC00090955C01AA0CBB1CAA0CBB1CA796EEAD1E
:109ED000FFADA797EA0DFB1D40815181628173811F
:109EE0004DA35EA36FA378A7A396EEADFFADA39796
:109EF000E80FF91FEE0FFF1FEE0FFF1FA7962EAD05
:109F00003FADA797E20FF31F80819181A281B381BA
:109F10008D879E87AF87B88B19821A821B821C821D
:109F20002F963FAD2F973F932E964FAD2E974F9381
:109F30007F926F9261965FAD61975F9360968FADF0
:109F400060978F93ADB7BEB794970FB6F894BEBF26
:109F50000FBEADBF1196E3E4F2E084E201900D92F2
:109F60008A95E1F70E942BC1AC96EEADFFADAC97A0
:109F7000EA0DFB1D29813A814B815C8160817181F1
:109F8000828193810E94A7CA2F2D3E2D4D2D5C2DDD
:109F90000E94A7CA4B015C01EDB7FEB7BA960FB697
:109FA000F894FEBF0FBEEDBF20E030E0A9010E9493
:109FB00084CD87FD0DC0E6EEFAE08491882379F028
:109FC0009091C00095FFFCCF8093C6003196F5CFED
:109FD0008091C00085FFFCCFF0E2F093C60025E041
:109FE00030E0B501A4018CEB94E00E94BE230F5F2A
:109FF0001F4F021513050CF457CF8091C00085FF49
:10A00000FCCF2AE02093C60065964EAD5FAD659704
:10A010004150510965965FAF4EAF659757FF38CFF6
:10A020008091C00085FFFCCF8AE08093C60006C007
:10A030006F96AEADBFAD6F97AB2B31F06FEB73E0AA
:10A0400083E492E00E9483C3AA96BFADAA97B111A0
:10A050009DC020E030E0A90160912B0770912C0792
:10A0600080912D0790912E070E94A8CA6DA37EA310
:10A070008FA398A720E030E0A90160912F0770918D
:10A08000300780913107909132070E94A8CA6D87EE
:10A090007E878F87988B8091330790913407A091AA
:10A0A0003507B091360789839A83AB83BC8382E0FE
:10A0B00090E00E94F2999B01AC01CE0101969F9322
:10A0C0008F930C969F938F9348969F938F93EDB7A2
:10A0D000FEB7B4970FB6F894FEBF0FBEEDBFADB795
:10A0E000BEB7119684E2E3E4F2E001900D928A9506
:10A0F000E1F7C557DF4F2883CB58D040C857DF4F13
:10A100003883C858D040C757DF4F4883C958D0401C
:10A11000C657DF4F5883CA58D0400E942BC1C5573D
:10A12000DF4F2881CB58D040C857DF4F3881C858FF
:10A13000D040C757DF4F4881C958D040C657DF4F7E
:10A140005881CA58D04069817A818B819C810E9454
:10A15000A7CA20910E0230910F0240911002509137
:10A1600011020E94A7CA609333077093340780934B
:10A170003507909336072DB73EB7265D3F4F0FB694
:10A18000F8943EBF0FBE2DBF0E94CE28E9964EAD7B
:10A190005FADE9970FB6F8945EBF0FBE4DBF09C023
:10A1A000E9968EAD9FADE9970FB6F8949EBF0FBEAE
:10A1B0008DBFE996AEADBFADE9970FB6F894BEBFBF
:10A1C0000FBEADBFC557DF4F0FB6F894DEBF0FBE51
:10A1D000CDBFDF91CF911F910F91FF90EF90DF9056
:10A1E000CF90BF90AF909F908F907F906F905F9037
:10A1F0004F903F902F9008958F929F92AF92BF9271
:10A20000CF92DF92EF92FF921F93CF93DF93C09193
:10A210000C07D0910D0780E50E94EA26882379F08B
:10A220000E94DD266C01EE24D7FCE094FE2C11E0A8
:10A23000C114D104E104F10431F410E004C010E0D1
:10A24000C12CD12C760183E50E94EA268823D9F01F
:10A250000E94AC2620E030E04AE754E40E9456CE4B
:10A260000E94F5CB6B017C0111110FC061157105C6
:10A270008105910551F48881882339F061E0CE0190
:10A280000E94AFA907C01123B1F360E081EB9AE00F
:10A290000E94F9A981E00E947EA90E948D990E94E6
:10A2A000C523C114D104E104F104C1F08090560526
:10A2B00090905705A0905805B09059058C0C9D1CA6
:10A2C000AE1CBF1C0E94E5C7681579058A059B0571
:10A2D00080F40E94D1AB81110CC025C00E94CFAB8D
:10A2E000882321F10E94D1AB811106C00E94E14771
:10A2F000F9CF80E00E947EA98091410760E0882329
:10A3000019F082EA9AE002C082E99AE0DF91CF91E7
:10A310001F91FF90EF90DF90CF90BF90AF909F90F4
:10A320008F900C94F9A90E94E147CCCFDF91CF9197
:10A330001F91FF90EF90DF90CF90BF90AF909F90D4
:10A340008F9008958F929F92AF92BF92CF92DF929B
:10A35000EF92FF92CF938091350283FDEDC060E0D4
:10A360008BED98E00E94F9A983E50E94EA2680938C
:10A3700014028111D8C082E50E94EA268111D3C05F
:10A380000E94E5C76B017C01109263056091B612D3
:10A390007091B712882777FD8095982F0E9423CC63
:10A3A000C1E0209198123091991240919A125091E7
:10A3B0009B120E9484CD18160CF0C0E0C093480593
:10A3C000CAE0809148056091B6127091B712882357
:10A3D00009F482C08091630581117EC0882777FDD2
:10A3E0008095982F0E9423CC209198123091991239
:10A3F00040919A1250919B120E9484CD18160CF035
:10A4000082C00E94E5C74B015C01D701C60188519B
:10A410009C4FAF4FBF4F88159905AA05BB0508F0A3
:10A4200058C0E091660584E0E89FF0011124E256EF
:10A43000FD4E4081518162817381E8EDF8E08491A5
:10A44000882341F09091C00095FFFCCF8093C60017
:10A450003196F5CF22E030E08CEB94E00E94BE23F1
:10A46000E4EDF8E08491882341F09091C00095FFDD
:10A47000FCCF8093C6003196F5CF6091660570E001
:10A480004AE050E08CEB94E00E94EC22E0EDF8E032
:10A490008491882341F09091C00095FFFCCF809378
:10A4A000C6003196F5CF4091981250919912609163
:10A4B0009A1270919B1221E030E08CEB94E00E94A4
:10A4C000BE238091C00085FFFCCFC093C6007501FC
:10A4D00064010E94E14775CF882777FD8095982F0A
:10A4E0000E9423CC209198123091991240919A1297
:10A4F00050919B120E9481CB87FF05C0809114026E
:10A50000882309F47ECF60E086EC98E00E94F9A9E8
:10A51000CF91FF90EF90DF90CF90BF90AF909F9042
:10A520008F900C94C5230E94AC260E94F0CB7093B0
:10A53000B7126093B61224CFCF91FF90EF90DF90C7
:10A54000CF90BF90AF909F908F900895CF92DF9261
:10A55000EF92FF92CF93DF9380E50E94EA26882353
:10A5600009F44FC00E94AC266B017C0183E50E9478
:10A57000EA26882331F00E94AC260E94F0CBEB0142
:10A5800002C0CFEFDFEFCE0101960397D0F5C701F0
:10A59000B6010E94F0CBF62E262F372FEFEDF3E019
:10A5A000419151914217530761F184E0E531F80779
:10A5B000B9F737FD26C00E948D99EF2C60E08F2DF2
:10A5C0000E94BCC9CF3F8FEFD80729F0219771F0C7
:10A5D000C0E0D0E00DC08F2D0E942ACA31E020E0FB
:10A5E000892B09F030E0C32FD22F02C0C1E0D0E0A8
:10A5F0008E2D0E942ACA8C179D0719F00E94E147F0
:10A60000F7CFDF91CF91FF90EF90DF90CF9008953B
:10A61000CF93DF93EC01809166058093490584E533
:10A620000E94EA26811102C080E03EC00E94DD2621
:10A63000809349058823C1F3E7ECFFE084918823E8
:10A6400041F09091C00095FFFCCF8093C6003196F9
:10A65000F5CF8091C00085FFFCCF8DE48093C600CC
:10A660004AE050E0BE018CEB94E00E94EC22E2E074
:10A67000F6E08491882341F09091C00095FFFCCFD3
:10A680008093C6003196F5CF40E050E060914905D7
:10A690008CEB94E00E9423238091C00085FFFCCFC7
:10A6A0008AE08093C60081E0DF91CF91089589E62A
:10A6B00090E0AEDF81110BC1EBE2F9E084918823D9
:10A6C00041F09091C00095FFFCCF8093C600319679
:10A6D000F5CFE7E2F9E08491882341F09091C00042
:10A6E00095FFFCCF8093C6003196F5CFE0914905E8
:10A6F00084E0E89FF0011124E256FD4E4081518133
:10A700006281738121E030E08CEB94E00E94BE23F3
:10A71000E4E2F9E08491882341F09091C00095FF34
:10A72000FCCF8093C6003196F5CFE0914905F0E06B
:10A73000EE0FFF1FE854FD4E60817181882777FD81
:10A740008095982F0E9423CCAB01BC0121E030E022
:10A750008CEB94E00E94BE23E0E2F9E08491882330
:10A7600041F09091C00095FFFCCF8093C6003196D8
:10A77000F5CF409198125091991260919A12709170
:10A780009B1221E030E08CEB94E00E94BE23EDE1CF
:10A79000F9E08491882341F09091C00095FFFCCFAF
:10A7A0008093C6003196F5CF6091B6127091B712C2
:10A7B000882777FD8095982F0E9423CCAB01BC01A0
:10A7C00021E030E08CEB94E00E94BE23EAE1F9E066
:10A7D0008491882341F09091C00095FFFCCF809335
:10A7E000C6003196F5CF4AE050E060E070E08CEBB7
:10A7F00094E00E94EC228091C00085FFFCCF8AE3A8
:10A800008093C60040919E1250919F126091A012B9
:10A810007091A11221E030E08CEB94E00E94BE2305
:10A82000E7E1F9E08491882341F09091C00095FF21
:10A83000FCCF8093C6003196F5CF6091B81270912D
:10A84000B912882777FD8095982F0E9423CCAB0101
:10A85000BC0121E030E08CEB94E00E94BE23E3E1F8
:10A86000F9E08491882341F09091C00095FFFCCFDE
:10A870008093C6003196F5CF8091490590E00E9403
:10A88000B39B4AE050E0BC018CEB94E00E94EC22C8
:10A89000EEE0F9E08491882341F09091C00095FFAB
:10A8A000FCCF8093C6003196F5CF8FEF9FEF0E94CB
:10A8B000B39B4AE050E0BC018CEB94E00E94EC2298
:10A8C0008091C00085FFFCCF8AE08093C600089588
:10A8D0004F925F926F927F928F929F92AF92BF92B0
:10A8E000CF92DF92EF92FF921F93CF93DF938DE68B
:10A8F00090E08EDE8111BCC18091350283FDB8C12C
:10A9000060E083E099E00E94F9A983E50E94EA26CD
:10A910008093140281117CC082E50E94EA26811195
:10A9200077C086E40E94EA268093C80E882351F0FF
:10A930000E94AC26609337027093380280933902EC
:10A9400090933A0283E50E94EA26882351F00E9400
:10A95000AC2660933B0270933C0280933D0290933F
:10A960003E0282E40E94EA26882351F00E94AC262F
:10A9700060933F02709340028093410290934202A1
:10A980000E94E5C74B015C01C0914905D0E0FE0182
:10A99000EE0FFF1FE854FD4E60817181882777FD1F
:10A9A0008095982F0E9423CCFE01EE0FFF1FEE0F23
:10A9B000FF1FE256FD4EC1E020813181428153816B
:10A9C0000E9484CD18160CF0C0E0C0934805109288
:10A9D0006305CC24CA94DC2C760158EE452E53E056
:10A9E000552E612C712C1AE08091630581111EC0D7
:10A9F0008FEFC816D806E806F80681F1F7FC16C0F6
:10AA00000E94E5C76C197D096031774238F10EC0AC
:10AA10000E94AC26C0914905D0E0CC0FDD1FC85480
:10AA2000DD4E0E94F0CB798368837BCF60E088EEB7
:10AA300098E00E94F9A90E94C52380915605909143
:10AA40005705A0915805B091590580934E059093F4
:10AA50004F05A0935005B09351050AC10E94E5C768
:10AA6000A501940128513C4F4F4F5F4F26173707E0
:10AA70004807590708F481C00E94E1478FEFC816C4
:10AA8000D806E806F80609F042C080914805E09132
:10AA90004905F0E0EF01CC0FDD1FCC0FDD1FC256E2
:10AAA000DD4EEE0FFF1FE854FD4E6081718188235B
:10AAB000B9F0882777FD8095982F0E9423CC20E05D
:10AAC00030E040E85FE30E94A7CA9B01AC016881C7
:10AAD00079818A819B810E9484CD87FF49C084CF80
:10AAE000882777FD8095982F0E9423CC20E030E0C6
:10AAF00040E85FE30E94A8CA9B01AC0168817981AC
:10AB00008A819B810E9481CB181694F56DCFF7FC4A
:10AB10006BCFE0914905F0E0EF01CC0FDD1FCC0FCA
:10AB2000DD1FC256DD4EEE0FFF1FE854FD4E608163
:10AB30007181882777FD8095982F0E9423CC9B01F7
:10AB4000AC01688179818A819B810E94A7CA0E9499
:10AB5000F0CB97FF07C090958095709561957F4FDA
:10AB60008F4F9F4F64307105810591050CF43CCFE8
:10AB70000E94E5C76B017C0137CFE0E0F9E08491EA
:10AB8000882341F09091C00095FFFCCF8093C600D0
:10AB90003196F5CFE091490584E0E89FF00111245A
:10ABA000E256FD4E408151816281738121E030E0A7
:10ABB0008CEB94E00E94BE23ECEFF8E084918823B4
:10ABC00041F09091C00095FFFCCF8093C600319674
:10ABD000F5CF6091490570E04AE050E08CEB94E0DD
:10ABE0000E94EC22E8EFF8E08491882341F09091F4
:10ABF000C00095FFFCCF8093C6003196F5CFF7FEDD
:10AC000003C0E6EFF8E026C00E94E5C74B015C01F7
:10AC1000C701B601605F784D8F4F9F4F6819790962
:10AC20008A099B09A30192010E9452CFBA01A9018E
:10AC30002AE030E08CEB94E00E9418238091C00061
:10AC400085FFFCCF0EC09091C00095FFFCCF809394
:10AC5000C600319684918111F6CF8091C00085FFA6
:10AC6000FCCF1093C6000E94E5C74B015C0104CFE6
:10AC7000DF91CF911F91FF90EF90DF90CF90BF9029
:10AC8000AF909F908F907F906F905F904F900895BE
:10AC9000CF92DF92EF92FF926B017C0180917F0552
:10ACA000882331F120E030E0A901C701B6010E94FC
:10ACB00081CB8823E9F020E030E040E05FE3C7018A
:10ACC000B6010E9456CE6B017C012BED3FE049E4BA
:10ACD00050E40E9456CEA70196010E9456CE9B01D9
:10ACE000AC0160E070E080E89FE30E9488CB04C084
:10ACF00060E070E080E89FE3FF90EF90DF90CF90FE
:10AD000008956091290270912A0280912B029091FE
:10AD10002C02BEDF609325027093260280932702E7
:10AD2000909328020895CF92DF92EF92FF92CF93F3
:10AD300088EC90E06DDC811144C084E40E94EA2636
:10AD4000882309F43EC00E94AC266B017C01C1E05F
:10AD500020E030E0A9010E9481CB811101C0C0E058
:10AD6000C0937F05CC2339F1E091490584E0E89F49
:10AD7000F0011124E75DFD4FC082D182E282F382AF
:10AD800020E030E0A9016091290270912A028091AF
:10AD90002B0290912C020E9481CB81110CC080E08B
:10ADA00090E0A0E4B0E48093290290932A02A0935B
:10ADB0002B02B0932C02CF91FF90EF90DF90CF90B9
:10ADC000A0CFCF91FF90EF90DF90CF900895CF92DA
:10ADD000DF92EF92FF920F931F93CF93DF93209117
:10ADE0000A0730910B0740E6429FC001439F900D38
:10ADF00011248A579A4F90930F0780930E078091E2
:10AE0000350280FF22C0E7ECFFE08491882341F007
:10AE10009091C00095FFFCCF8093C6003196F5CF8E
:10AE2000E0910E07F0910F078191882339F09091FE
:10AE3000C00095FFFCCF8093C600F6CF8091C00084
:10AE400085FFFCCF8AE08093C60080910E07909129
:10AE50000F07FC01208101962032D9F3F0930F07F0
:10AE6000E0930E072E3461F0C0910E07D0910F07CA
:10AE70006AE270E0CE010E94D7D20097D1F420C0E0
:10AE8000818190ED980F9A3010F08D3269F73296EB
:10AE9000DF0131962C9120532A30D0F3CD01FC01F3
:10AEA000019620812032D9F3F0930F07E0930E072B
:10AEB000DBCFFC0131968291803251F08A3241F031
:10AEC0001881898180538A3008F0C7C39E0102C06F
:10AED0001082F1CFF9012F5F3F4F40814F7DD1F7B5
:10AEE000CF01FC01019620812032D9F3F0930D07A8
:10AEF000E0930C07D0935D05C0935C050E94DD26AE
:10AF00001D3409F44FC0143509F487C3173409F010
:10AF1000A4C38C319105C9F17CF48430910534F4DB
:10AF20008230910554F597FF1EC079C3049709F04C
:10AF300076C30E94E74773C38A35910561F14CF4EB
:10AF40008D31910529F14E9709F069C30E94332D87
:10AF500066C38B35910511F18C35910509F05FC3FE
:10AF60000E94B62D5CC380913602882309F457C332
:10AF70000E94B22A0E94284052C321E0029709F0A1
:10AF800020E0822F0E94BF434AC30E944E2B47C33A
:10AF90000E94384844C31092620541C381E0809307
:10AFA00062053DC38037910509F4AFC10CF09FC025
:10AFB0008032910509F477C10CF055C087319105B5
:10AFC00009F43EC114F58231910509F407C28CF4ED
:10AFD00097FD25C3823091050CF425C1419709F0F6
:10AFE0001EC360E089E89AE00E94F9A90E94024429
:10AFF00016C38531910509F419C10CF01CC14497A1
:10B0000009F00DC30E94062E0AC38B31910509F485
:10B0100032C1ACF48931910509F41DC10CF020C195
:10B020008FE397E00E9470130E94E5C760934E057E
:10B0300070934F058093500590935105F0C28E3167
:10B04000910509F41DC10CF03AC14C9709F0E7C213
:10B0500060910C0770910D0721E040E08FE397E0CD
:10B060000E942017DCC28535910509F4BAC1E4F4C9
:10B070008135910509F494C174F48033910509F484
:10B0800021C18035910509F47EC18A9709F0C7C2B4
:10B090000E942D2FC4C28335910509F49BC10CF089
:10B0A0009DC110928505BBC28A36910509F44FC136
:10B0B0006CF48836910509F408C10CF03DC18C355B
:10B0C000910509F0ACC20E94C637A9C28D36910520
:10B0D00009F43BC18F36910509F414C18B369105F3
:10B0E00009F09DC2109265051092640598C28C3DCE
:10B0F000910509F4FEC10CF046C08139910509F4AF
:10B10000A7C1FCF48737910509F49FC17CF483370C
:10B11000910509F485C08537910509F486C1823708
:10B12000910509F07CC20E94603879C28937910587
:10B1300009F487C10CF481C18C38910509F4E9C088
:10B140006EC28B3C910509F4A3C174F4883C91054F
:10B1500009F481C1893C910509F47FC18E3B9105B9
:10B1600009F05DC2EFD85BC28D3C910509F4AAC11C
:10B170000CF4A5C18E3C910509F051C2C5E1D4E0A3
:10B1800003E715E0A9C18A3921E0920709F41CC23E
:10B1900014F58D32F1E09F0709F4FCC174F4823E8E
:10B1A000910509F4D0C18C32E1E09E0709F4CDC1CC
:10B1B0008D3D910509F033C2ABC18F32F1E09F079D
:10B1C00009F4FFC10CF4E9C18039914009F027C2AC
:10B1D0000E948D9924C2873FF1E09F0709F400C2C5
:10B1E00074F4853FE1E09E0709F4F1C10CF0F5C16C
:10B1F0008C3A914009F013C20E94053C10C2803A7B
:10B20000E3E09E0709F452C0873EF3E09F0709F48C
:10B21000FCC18335934009F002C20E940C3DFFC17E
:10B22000EDEFF7E0FEC00E94FC50F9C18FE397E01C
:10B230000E94A612F4C18FE397E00E946C13EFC145
:10B2400060910C0770910D0721E041E08FE397E0DA
:10B250000E942017E4C18FE397E00E947713DFC1BB
:10B2600080914207882309F4DAC183E50E94EA2627
:10B270008111DFC1D4C18FE397E00E940015CFC1D7
:10B2800080914207882309F4CAC160E08FE397E008
:10B290000E94B11660910C0770910D078FE397E043
:10B2A0000E94DB13BCC10E94CA2EB9C160910C0779
:10B2B00070910D078FE397E00E94281AB0C10E9499
:10B2C000332EADC10E94722FAAC188E690E0A0D9AA
:10B2D0008111A5C18091350283FDA1C183E50E9442
:10B2E000EA26882309F49BC10E94AC26C091490537
:10B2F000D0E0CC0FDD1FC854DD4E0E94F0CB798327
:10B3000068838DC10E9464368AC18EE299E00E94F2
:10B3100020448091350283FD82C183E50E94EA26A4
:10B32000882309F47CC10E94AC260E94F0CB709364
:10B33000B7126093B61273C1DF91CF911F910F9135
:10B34000FF90EF90DF90CF90B2C9C2DA68C183E579
:10B350000E94EA26811103C08FEF90E00FC00E9487
:10B36000DD2697FD09C00E94DD268F3F910509F07B
:10B370009CF70E94DD2602C080E090E09093650576
:10B38000809364054CC1269A2E9881E080930D022B
:10B3900060E086EB98E00E94F9A90E9486AA3FC16E
:10B3A0000E94809F0E94089A109265051092640581
:10B3B00068EE73E080E090E00E9414C8269A2E9A0E
:10B3C00010920D0260E088EA98E00E94F9A90E94BC
:10B3D00086AA25C181E08093850521C10E946F372F
:10B3E0001EC183E50E94EA26882309F418C10E9441
:10B3F000AC2620E030E04AE754E40E9456CE0E949A
:10B40000F5CB609352057093530580935405909348
:10B41000550505C19091C00095FFFCCF8093C600F3
:10B42000319684918111F6CFFAC060E080910C07CB
:10B4300090910D070E94AFA9F2C081E00E94749123
:10B44000EEC080E00E947491EAC00E941F39E7C0FC
:10B450000E94BA36E4C067DCE2C0C5E1D4E009EF7F
:10B460001EE089910E94EA26882349F00E94AC26BA
:10B470000E94F5CBF80160837183828393830C5F14
:10B480001F4FF4E0C931DF0761F70E946F6FC7C03B
:10B49000C5E1D4E009E11FE089910E94EA268823F2
:10B4A00039F00E94AC26F801608371838283938314
:10B4B0000C5F1F4FF4E0C931DF0771F7B0C00E9485
:10B4C000F039ADC00E94693AAAC00C5F1F4FF4E08A
:10B4D000C831DF0709F4A3C089910E94EA268823B6
:10B4E000A1F30E94AC26F801608371838283938369
:10B4F000ECCF83E50E94EA26882309F490C00E94DD
:10B50000AC260E94F0CB7093300260932F0287C06C
:10B5100083E50E94EA26882309F481C00E94AC26B4
:10B520000E94F0CB6B017C018DED90E071D8811110
:10B5300076C0E0914905F0E0EE0FFF1FE35DFD4F9F
:10B54000D182C0826CC002D86AC083E50E94EA261C
:10B55000882321F00E94DD26EC0102C0CEE6D0E077
:10B5600080E50E94EA26882369F00E94D226693885
:10B5700023E172078105910548F068E873E180E0F6
:10B5800090E004C068EE73E080E090E0AE010E94BD
:10B59000F60F45C00E94C63A42C083E50E94EA26E3
:10B5A000882319F00E94AC2603C060E070E0CB0154
:10B5B0006093060270930702809308029093090239
:10B5C0002EC00E94D03B2BC00E940B9A28C00E9424
:10B5D000E71B80E00E94711D22C00E94E71B1FC074
:10B5E00083E50E94EA26882361F00E94AC26C1E030
:10B5F00020E030E0A9010E9481CB8111C0E08C2FB6
:10B6000001C080E00E94711D0AC081E08093360273
:10B610000E9414AA0E94403E02C00E94A63DDF91F3
:10B62000CF911F910F91FF90EF90DF90CF900C94EE
:10B63000203E0E94DD26AC01662757FD6095762FDF
:10B640004093C2095093C3096093C4097093C5091C
:10B650008DE099E00E94C186E2CF0E94182BDFCFD7
:10B66000CF93DF938091060790910707039714F417
:10B670000E945B4460E08FE397E00E94C0158091D8
:10B68000060790910707892B09F463C080913F0753
:10B690008823B1F180910A0790910B0720E6289F3B
:10B6A000E001299FD00D1124CA57DA4F6CE97EE0E2
:10B6B000CE010E9489D2892BB9F060E08FE397E038
:10B6C0000E94B116EAE8FEE08491882341F090914F
:10B6D000C00095FFFCCF8093C6003196F5CF8091D6
:10B6E000C00085FFFCCF1CC0BE018FE397E00E9425
:10B6F0004F1580914007811103C0E7E8FEE009C0C3
:10B7000066DB11C09091C00095FFFCCF8093C6000E
:10B71000319684918111F6CF8091C00085FFFCCFD6
:10B720008AE08093C60080910607909107070197F1
:10B73000909307078093060780910A0790910B0763
:10B74000019664E070E00E943FCF90930B078093D6
:10B750000A070E94E290DF91CF910C94E1478F920B
:10B760009F92AF92BF92CF92DF92EF92FF920F9390
:10B770001F93CF93DF938C0186539E4F0E940A1034
:10B7800068018FE6C80ED11CC114D10421F17801E3
:10B790008BE5E81A8EEFF80AE70157018FE1A81A46
:10B7A000B1088DE2882E84E0982ECC15DD0599F045
:10B7B000FE01EE19FF09EA0DFB1D91828082FE0158
:10B7C00078978081811102C06F97EFCFCE014B97A0
:10B7D0000E94A487F9CFC801805B9F4F0E940A1086
:10B7E000C8018F96DF91CF911F910F91FF90EF903D
:10B7F000DF90CF90BF90AF909F908F900C940A10E5
:10B800008FE397E00C9416108FE397E0A8CF2F9268
:10B810003F924F925F926F927F928F929F92AF92E0
:10B82000BF92CF92DF92EF92FF920F931F93CF932D
:10B83000DF93CDB7DEB768970FB6F894DEBF0FBEC3
:10B84000CDBF1C012A013B0148015901DC01D896FA
:10B850006D917D918D919C91DB970E9421CC6B0124
:10B860007C01A30192010E9456CE0E946ECB0E94E1
:10B87000F5CB69877A878B879C87A5019401C701DF
:10B88000B6010E9456CE0E946ECB0E94F5CB6D870A
:10B890007E878F87988B29853A854B855C852837ED
:10B8A00031054105510540F488E790E0A0E0B0E0A3
:10B8B00089879A87AB87BC872D853E854F855889B8
:10B8C000283731054105510540F488E790E0A0E0B4
:10B8D000B0E08D879E87AF87B88B91012C5B3F4F7F
:10B8E000D9018D919D910D90BC91A02D8D839E834A
:10B8F000AF83B887BC01CD010E9423CC69837A83D2
:10B900008B839C8369857A858B859C850E9421CC5D
:10B91000698B7A8B8B8B9C8B20E030E0A90169814D
:10B920007A818B819C810E9481CB882339F1A70188
:10B930009601C701B6010E9456CE4B015C012989D0
:10B940003A894B895C89CA01B9010E9456CE9B0194
:10B95000AC01C501B4010E94A7CA4B015C01298159
:10B960003A814B815C81CA01B9010E94A8CA9B013E
:10B97000AC01C501B4010E9488CB03C060E070E057
:10B98000CB010E946ECB0E94F0CB2B013C016D815C
:10B990007E818F81988590958095709561957F4F78
:10B9A0008F4F9F4F0E9423CC4B015C016D857E859C
:10B9B0008F8598890E9421CC6D837E838F839887A1
:10B9C00020E030E0A901C501B4010E9481CB8823A9
:10B9D00049F12D813E814F815885CA01B9010E94EC
:10B9E00056CE6D8B7E8B8F8B988FA7019601C701EA
:10B9F000B6010E9456CE9B01AC016D897E898F896C
:10BA0000988D0E94A7CA6B017C01A5019401C50114
:10BA1000B4010E94A8CA9B01AC01C701B6010E94F3
:10BA200088CB03C060E070E0CB010E945ECCF101E6
:10BA300080889188A288B38875016401C418D508EC
:10BA4000E608F7080E94F0CBC61AD70AE80AF90AF6
:10BA5000F7FE6BC020E030E0A90169817A818B811B
:10BA60009C810E9481CB882309F447C029813A81B7
:10BA70004B815C81CA01B9010E94A8CA6B017C019B
:10BA8000C501B4010E9421CC9B01AC01C701B601E4
:10BA90000E9456CE6B017C0129893A894B895C89C9
:10BAA000CA01B9010E9456CE9B01AC01C701B60183
:10BAB0000E94A7CA6B017C012D813E814F81588570
:10BAC000CA01B9010E9456CE9B01AC01C701B60163
:10BAD0000E94A8CA6B017C0120E030E040E850E4FD
:10BAE00069817A818B819C810E9456CE9B01AC0139
:10BAF000C701B6010E9488CB03C060E070E0CB01B3
:10BB00000E946ECB0E94F0CB2B013C0197FF03C03B
:10BB1000412C512C3201481459046A047B0410F062
:10BB200024013501C12CD12C76018FB7F894F10195
:10BB3000E45BFF4F9081911125C0D10154964D9245
:10BB40005D926D927C925797C40CD51CE61CF71C35
:10BB5000F101C08ED18EE28EF38E29853A854B8518
:10BB60005C85DC962D933D934D935C93DF97A05CB1
:10BB7000BF4F2D853E854F8558892D933D934D931D
:10BB80005C9313978FBF68960FB6F894DEBF0FBE15
:10BB9000CDBFDF91CF911F910F91FF90EF90DF907C
:10BBA000CF90BF90AF909F908F907F906F905F905D
:10BBB0004F903F902F9008954F925F926F927F9297
:10BBC000AF92BF92CF92DF92EF92FF920F931F93AB
:10BBD000CF93DF93EB017A01209709F458C0411508
:10BBE000510509F454C0AAA4BBA40CA51DA5950138
:10BBF000A8016EA17FA188A599A50E9481CB882369
:10BC000009F445C08FA981113AC0F70146A057A099
:10BC100060A471A4A3019201B501C8010E9484CD62
:10BC200018166CF5A3019201C301B2010E9456CE11
:10BC30006B017C018AA99BA9ACA9BDA9BC01CD015E
:10BC400090589B01AC010E94A8CA2EA53FA548A907
:10BC500059A90E9456CE9B01AC01C701B6010E94B2
:10BC6000A7CA0E94C3CE6B017C019B01AC01B50148
:10BC7000C8010E9481CB87FD02C056018701A50142
:10BC8000B8014EA35FA368A779A781E08EABDF91CF
:10BC9000CF911F910F91FF90EF90DF90CF90BF90C9
:10BCA000AF907F906F905F904F900895DF92EF92EA
:10BCB000FF920F931F93CF93DF938091F7098FB774
:10BCC000F894E090F6098FBF8091F70990E08E1903
:10BCD00091098F7099270497E4F01091F709135098
:10BCE0001F7040E050E000E0F12C8DE4D82E1E15CE
:10BCF00081F011501F70D19EE0011124C850D64F21
:10BD0000602F7F2DCE0158DF402F5F2D0C2FFD2E91
:10BD1000EECFDF91CF911F910F91FF90EF90DF90C9
:10BD200008954F925F926F927F92AF92BF92CF929F
:10BD3000DF92EF92FF920F931F93CF93DF938C01CB
:10BD4000EB01009709F453C0FC0187A981114FC092
:10BD500046A057A060A471A4AEA0BFA0C8A4D9A457
:10BD60009501A601C301B2010E9481CB87FF3FC0AC
:10BD7000A3019201C301B2010E9456CE2B013C01E6
:10BD8000F80182A993A9A4A9B5A9BC01CD01905835
:10BD90009B01AC010E94A8CAF80126A537A540A9BD
:10BDA00051A90E9456CE9B01AC01C301B2010E9471
:10BDB000A7CA0E94C3CE7B018C019B01AC01B501D7
:10BDC000C6010E9481CB87FF02C0750186019701E1
:10BDD000A801B501C6010E9481CB882341F0A701CB
:10BDE000B8014EA35FA368A779A781E08EABDF916E
:10BDF000CF911F910F91FF90EF90DF90CF90BF9068
:10BE0000AF907F906F905F904F900895EF92FF9268
:10BE10000F931F93CF93DF931091F609F12C00E05D
:10BE200080E090E02DE4E22E2091F709121781F0D6
:10BE3000E19EE0011124C850D64FAE016F2D702F46
:10BE400070DF1F5F1F708F2D902FFC2E0D2FECCFFA
:10BE500040E050E06F2D702FDF91CF911F910F9137
:10BE6000FF90EF905ECF4F925F926F927F928F9292
:10BE70009F92AF92BF92CF92DF92EF92FF920F9379
:10BE80001F93CF93DF939090F609C0E0D0E03DE49C
:10BE9000832E892D992787FD90952091F70930E011
:10BEA00082179307B1F1889E5001899EB00C11242E
:10BEB000C5018850964F5C01209729F18EA9811108
:10BEC00004C0F50186A98823F1F0CAA0DBA0ECA08C
:10BED000FDA0A7019601F50166A177A180A591A516
:10BEE0000E9488CB2B013C01A70196016EA17FA186
:10BEF00088A599A50E9488CBAB01BC019301820162
:10BF0000CE0185DC1EAA9394F92DFF709F2EE501CA
:10BF1000C0CF2097E9F0CAA0DBA0ECA0FDA0A7014C
:10BF200096016DEC7CEC8CE49DE30E9488CB4B0188
:10BF30005C01A70196016EA17FA188A599A50E9429
:10BF400088CBAB01BC0195018401CE0160DC1EAA47
:10BF5000DF91CF911F910F91FF90EF90DF90CF90E5
:10BF6000BF90AF909F908F907F906F905F904F9019
:10BF700008959CDE4BDF77CF1092F6091092F709F7
:10BF800080E1E6EEF9E0DF011D928A95E9F7109273
:10BF9000D6091092D7091092D8091092D909109297
:10BFA000DA091092DB091092DC091092DD09109277
:10BFB000DE091092DF091092E0091092E109109257
:10BFC000E2091092E3091092E4091092E509109237
:10BFD000D2091092D3091092D4091092D50908956C
:10BFE0004F925F926F927F928F929F92AF92BF9289
:10BFF000CF92DF92EF92FF920F931F93CF93DF9335
:10C000008091C80E882309F4E9C000913B02109189
:10C010003C02D0913D02C0913E026091B8127091F5
:10C02000B912882777FD8095982F0E9423CC20E0B5
:10C0300030E040E050E40E94A8CA98014D2F5C2FE8
:10C040000E9481CB87FDCAC05090F609612C712CEB
:10C05000812C912C4DE4442E8091F709581609F457
:10C060004CC0459C50011124C5018850964F5C017D
:10C07000FC0180819181A281B381892B8A2B8B2B3A
:10C0800081F484819581A681B781892B8A2B8B2BA2
:10C0900041F480859185A285B385892B8A2B8B2BD2
:10C0A00039F1F50164857585868597850E9423CCD5
:10C0B0006B017C01F50160897189828993890E94F5
:10C0C00021CC9B01AC01C701B6010E9488CBF501D0
:10C0D00022A133A144A155A10E9456CE6B017C013F
:10C0E0009301A4010E9484CD181614F4360147016F
:10C0F0005394F52DFF705F2EAFCF20913702309112
:10C1000038024091390250913A02B301C4010E94B1
:10C1100056CE9B01AC01B8018D2F9C2F0E94A8CA5E
:10C120006B017C0198014D2F5C2F0E9481CB87FD14
:10C1300014C000913F0210914002D0914102C09181
:10C14000420298014D2F5C2FB601C7010E9484CD99
:10C1500018161CF08601DE2DCF2D8090CD09909011
:10C16000CE09A090CF09B090D00998014D2F5C2F37
:10C17000C501B4010E9484CD1816E4F420E037ED27
:10C1800043EA5CE3B8018D2F9C2F0E9456CE6B01D1
:10C190007C0128E431EE4AE75FE3C501B4010E9467
:10C1A00056CE9B01AC01C701B6010E94A8CA8B0103
:10C1B000D82FC92FC801AD2FBC2F8093CD099093E4
:10C1C000CE09A093CF09B093D009B8018D2F9C2F31
:10C1D0000E94F0CB7093B9126093B812DF91CF91A7
:10C1E0001F910F91FF90EF90DF90CF90BF90AF9095
:10C1F0009F908F907F906F905F904F900895609187
:10C2000064059091F7098091F609981781F0809163
:10C21000F6099DE4899FF0011124E05CF54F6081EF
:10C220009091F709891719F08F5F8F70F9CF70E03F
:10C2300089E00E94A6C8D4CE2F923F924F925F927F
:10C240006F927F928F929F92AF92BF92CF92DF9226
:10C25000EF92FF920F931F93CF93DF93CDB7DEB78B
:10C26000C059D1090FB6F894DEBF0FBECDBF69AF7C
:10C270007AAF8BAF9CAFCE01CD9627969FAF8EAF96
:10C28000279721962CAF3DAF4EAF5FAF21971E0190
:10C2900091E4290E311CD101ED92FD920D931C9376
:10C2A0001397A6968FAEA697AA969FAEAA97AE961C
:10C2B000AFAEAE97E296BFAEE297B091F709BF5F1F
:10C2C000BF70CC57DF4FB883C458D040EB2EFF244B
:10C2D000E7FCF0948091F60990E08E159F0519F423
:10C2E0000E94E147F7CF3F922F922796EFAD279715
:10C2F000EF932696FFAD2697FF93CE01C9969F93A5
:10C300008F932DB73EB7245231090FB6F8943EBF34
:10C310000FBE2DBFADB7BEB7119684E2E3E4F2E0E5
:10C3200001900D928A95E1F70E942BC10FB6F89407
:10C33000DEBF0FBECDBF2091090F30910A0F409193
:10C340000B0F50910C0F69AD7AAD8BAD9CAD0E9477
:10C3500056CE0E9426CE2B013C0169A77AA78BA757
:10C360009CA720910D0F30910E0F40910F0F50910F
:10C37000100F21966CAD7DAD8EAD9FAD21970E94C3
:10C3800056CE0E9426CE4B015C016DA77EA78FA7DB
:10C3900098AB2091110F3091120F4091130F5091D3
:10C3A000140FD1016D917D918D919C910E9456CE7B
:10C3B0000E9426CE2B966CAF7DAF8EAF9FAF2B9792
:10C3C00069AB7AAB8BAB9CAB2091150F3091160FFC
:10C3D0004091170F5091180FF60160817181828191
:10C3E00093810E9456CE0E9426CE6B017C016DABDC
:10C3F0007EAB8FAB98AF8091E6099091E709A09151
:10C40000E809B091E909A3019201281B390B4A0BF5
:10C410005B0BCA01B9010E9423CC2F966CAF7DAF94
:10C420008EAF9FAF2F978091EA099091EB09A09171
:10C43000EC09B091ED09A5019401281B390B4A0BB9
:10C440005B0BCA01B9010E9423CC63966CAF7DAF30
:10C450008EAF9FAF63978091EE099091EF09A09105
:10C46000F009B091F1092B962CAD3DAD4EAD5FAD0D
:10C470002B97281B390B4A0B5B0BCA01B9010E9491
:10C4800023CC6D966CAF7DAF8EAF9FAF6D978091D3
:10C49000350283FF08C0C092F209D092F309E092FE
:10C4A000F409F092F5098091F2099091F309A091B5
:10C4B000F409B091F509A7019601281B390B4A0B25
:10C4C0005B0BCA01B9010E9423CC67966CAF7DAFAC
:10C4D0008EAF9FAF679720E030E0A9010E9481CB2B
:10C4E000882309F4A8C0CA55DF4F4881C65AD040F6
:10C4F00034E0439FF0011124E256FD4E20910602E4
:10C5000030910702409108025091090260817181C7
:10C51000828193810E9481CB87FF2FC0C092F20954
:10C52000D092F309E092F409F092F509E7ECFFE00C
:10C530008491882341F09091C00095FFFCCF8093B7
:10C54000C6003196F5CFE2EFFFE08491882341F0F9
:10C550009091C00095FFFCCF8093C6003196F5CF37
:10C560008091C00085FFFCCF8AE08093C60067966B
:10C570001CAE1DAE1EAE1FAE679767966CAD7DAD4F
:10C580008EAD9FAD67970E94F0CB97FF07C0909547
:10C590008095709561957F4F8F4F9F4F0E9423CC60
:10C5A0006B017C0120E030E04CED53E46091150F0D
:10C5B0007091160F8091170F9091180F0E9456CE10
:10C5C0009B01AC01C701B6010E9484CD18169CF5F1
:10C5D0008DA99EA9AFA9B8AD8093F2099093F309F4
:10C5E000A093F409B093F509E7ECFFE08491882368
:10C5F00041F09091C00095FFFCCF8093C60031962A
:10C60000F5CFE4EDFFE08491882341F09091C000E4
:10C6100095FFFCCF8093C6003196F5CF8091C00086
:10C6200085FFFCCF8AE08093C60067961CAE1DAEE6
:10C630001EAE1FAE67978091F709EDE48E9FD00183
:10C640001124A850B64F2996BFAFAEAF2997FD0170
:10C65000E45BFF4F108263962CAD3DAD4EAD5FADF8
:10C6600063972F966CAD7DAD8EAD9FAD2F970E94D9
:10C67000A8CAA1966CAF7DAF8EAF9FAFA1970E9465
:10C68000F0CB2B013C0197FF08C07094609450944C
:10C690004094411C511C611C711C2996AEADBFAD6C
:10C6A00029974D925D926D927C92139763962CAD73
:10C6B0003DAD4EAD5FAD63972F966CAD7DAD8EAD4C
:10C6C0009FAD2F970E94A7CAEB966CAF7DAF8EAF40
:10C6D0009FAFEB970E94F0CB4B015C0197FF08C026
:10C6E000B094A09490948094811C911CA11CB11CC6
:10C6F0002996EEADFFAD299784829582A682B782F6
:10C700006D966CAD7DAD8EAD9FAD6D970E94F0CBFB
:10C710006B017C0197FF08C0F094E094D094C09422
:10C72000C11CD11CE11CF11C2996AEADBFAD2997EF
:10C730001896CD92DD92ED92FC921B97CA55DF4F71
:10C74000F881C65AD040EF2FF0E0A396FFAFEEAFCE
:10C75000A39767966CAD7DAD8EAD9FAD67970E9438
:10C76000F0CB97FF07C090958095709561957F4FAE
:10C770008F4F9F4F0E9423CCA3962EAD3FADA39722
:10C78000220F331F220F331FE7963FAF2EAFE797DD
:10C79000F901EB5DFD4F20813181428153810E947F
:10C7A00056CE0E94F0CB9B01AC01A396EEADFFAD3F
:10C7B000A397EE0FFF1FE35DFD4FA081B1810E94A3
:10C7C000A0CF24E630E040E050E00E9474CF2996EC
:10C7D000AEADBFAD29971C962D933D934D935C93C1
:10C7E0001F97F82DE92D7A2D6B2D8C149D04AE0426
:10C7F000BF0424F4FC2DED2D7E2D6F2D8F2F9E2F49
:10C80000A72FB62F82179307A407B50714F4DA01F0
:10C81000C901B301A201481659066A067B0614F441
:10C82000AC01BD012996EEADFFAD2997408B518B30
:10C83000628B738B463051056105710510F40C94C1
:10C840009D6DE85BFF4F8091640590916505AA2777
:10C8500097FDA095BA2F80839183A283B38320E0B4
:10C8600030E0A9012F966CAD7DAD8EAD9FAD2F97B9
:10C870000E9481CB182F111F1127111F1295107FB5
:10C8800020E030E0A90163966CAD7DAD8EAD9FAD2B
:10C8900063970E9481CB87FD106220E030E0A90100
:10C8A0006D966CAD7DAD8EAD9FAD6D970E9481CBC9
:10C8B00087FD146020E030E0A901A1966CAD7DAD4C
:10C8C0008EAD9FADA1970E9481CB87FD116020E0C6
:10C8D00030E0A901EB966CAD7DAD8EAD9FADEB97D1
:10C8E0000E9481CB87FD126020E030E0A9016796AD
:10C8F0006CAD7DAD8EAD9FAD67970E9481CB87FDFE
:10C9000018602996AEADBFAD299790961C9390976D
:10C91000CA55DF4FE881C65AD0409196EC9345281E
:10C920004628472821F489288A288B2811F05F9807
:10C930008A982996EEADFFAD299780859185A285CD
:10C94000B385892B8A2B8B2B41F09FB7F89480916C
:10C9500008018E7F809308019FBF2996EEADFFAD41
:10C96000299784859585A685B785892B8A2B8B2B5E
:10C9700091F08091D109882319F081508093D109D9
:10C98000CA55DF4FF881C65AD040F11104C0129841
:10C9900080E28093D1092996AEADBFAD29971C9650
:10C9A0002D913D914D915C911F97C458DF4F288385
:10C9B00039834A835B83CC57D040232B242B252BF0
:10C9C00039F12090F50E3090F60E0091F70E10918F
:10C9D000F80E9101A801A6966FADA697AA967FAD15
:10C9E000AA97AE968FADAE97E2969FADE2970E9462
:10C9F00081CB87FD16C0A6962FACA697AA963FAC12
:10CA0000AA97AE960FADAE97E2961FADE29709C01A
:10CA10002090D90E3090DA0E0091DB0E1091DC0ED2
:10CA2000D8CF4090090F50900A0F60900B0F709074
:10CA30000C0FA30192012F966CAD7DAD8EAD9FAD15
:10CA40002F970E9488CB2F966CAF7DAF8EAF9FAF94
:10CA50002F97698B7A8B8B8B9C8B80900D0F90908E
:10CA60000E0FA0900F0FB090100FA50194016396C8
:10CA70006CAD7DAD8EAD9FAD63970E9488CB639604
:10CA80006CAF7DAF8EAF9FAF63976D8B7E8B8F8BBF
:10CA9000988F2091110F3091120F4091130F5091E8
:10CAA000140F6D966CAD7DAD8EAD9FAD6D970E94F0
:10CAB00088CB6B017C0169877A878B879C87A30170
:10CAC0009201A1966CAD7DAD8EAD9FADA1970E94F8
:10CAD00088CB69837A838B839C83A5019401EB9631
:10CAE0006CAD7DAD8EAD9FADEB970E9488CB6D8315
:10CAF0007E838F8398872091150F3091160F409178
:10CB0000170F5091180F67966CAD7DAD8EAD9FAD30
:10CB100067970E9488CBE796EEADFFADE797EB5D98
:10CB2000FD4F20813181428153810E9456CE4B01BD
:10CB30005C01A396EEADFFADA397EE0FFF1FE35D83
:10CB4000FD4F60817181882777FD8095982F0E9425
:10CB500023CC9B01AC01C501B4010E9456CE20E05C
:10CB600030E048EC52E40E9488CB6D877E878F8747
:10CB7000988B2996AEADBFAD29972D913D914D91E2
:10CB80005C911397C058DF4F288339834A835B83B6
:10CB9000C058D040263031054105510534F5149672
:10CBA0008D909D90AD90BC901797B6E08B16910438
:10CBB000A104B104D4F42996EEADFFAD2997808489
:10CBC0009184A284B384F6E08F169104A104B10489
:10CBD00064F4DC01CB01BF772996EEADFFAD299758
:10CBE00086A797A7A0ABB1AB30C02F966CAD7DAD3B
:10CBF0008EAD9FAD2F970E9401CF4B015C016396D4
:10CC00006CAD7DAD8EAD9FAD63970E9401CF9B0152
:10CC1000AC01C501B4010E94A8CA4B015C01C70167
:10CC2000B6010E9401CF9B01AC01C501B4010E9475
:10CC3000A8CA0E94C3CE2996AEADBFAD29979E96D5
:10CC40006D937D938D939C93D1972996AEADBFAD97
:10CC500029979E962D913D914D915C91D197EB96A0
:10CC60002CAF3DAF4EAF5FAFEB9760E070E080E878
:10CC70009FE30E9488CB9B01AC01B101C8010E94D7
:10CC800056CE6B017C011091F7098091F609181BB3
:10CC90001F70E12FF0E0CB57DF4FF983E883C558D1
:10CCA000D040A701960160E074E284E799E40E9415
:10CCB00088CB0E9426CE4B015C01CB57DF4F888189
:10CCC0009981C558D0400297069798F58091290F11
:10CCD00090912A0FA0912B0FB0912C0F88169906D6
:10CCE000AA06BB0630F5BC01CD01681979098A098D
:10CCF0009B09660F771F881F991F212F30E040E0A6
:10CD000050E00E9452CFCA01B9010E9421CC0E947A
:10CD100026CE680D791D8A1D9B1D0E9421CC9B018A
:10CD2000AC0160E074E284E799E40E9488CB6B0177
:10CD30007C01A7019601EB966CAD7DAD8EAD9FADEC
:10CD4000EB970E9456CE6D966CAF7DAF8EAF9FAFC6
:10CD50006D972996AEADBFAD299792966D937D9351
:10CD60008D939C93959750966D917D918D919C910B
:10CD700053970E9421CC67966CAF7DAF8EAF9FAF6B
:10CD80006797A70196010E9456CE0E946ECB0E9423
:10CD9000F5CBA1966CAF7DAF8EAF9FAFA1972996D3
:10CDA000EEADFFAD299760AF71AF82AF93AF9E013B
:10CDB0002F5F3F4F69963FAF2EAF699749E15FE024
:10CDC000A7965FAF4EAFA797CE01419627969FAF2C
:10CDD0008EAF2797DE015996A396BFAFAEAFA3974C
:10CDE000212C312CB0E82C96BFAF2C97EFE3609646
:10CDF000EFAF60976996AEADBFAD69976D917D91CC
:10CE00008D919D916996BFAFAEAF6997A7019601CD
:10CE10000E9456CEA396EEADFFADA397619371939A
:10CE200081939193A396FFAFEEAFA3972B013C01A3
:10CE3000E89477F8A796AEADBFADA7978D909D907B
:10CE4000AD90BD90A796BFAFAEAFA797A5019401D7
:10CE5000C301B2010E9484CD18160CF5A301920102
:10CE6000C501B4010E9488CB162F072FB82EA92E1A
:10CE7000262F372F482F592FB1012C968FAD2C9785
:10CE800060969FAD60970E9481CB87FD08C0212EE0
:10CE9000302E2C96BFAE2C976096AFAE60976996F9
:10CEA000EEADFFAD699727962EAD3FAD2797E21700
:10CEB000F30709F09FCF20E030E040E85FE3B101E5
:10CEC0002C968FAD2C9760969FAD60970E9481CB7A
:10CED00087FF52C07E0139E2E30EF11C8E01075E2E
:10CEE0001F4F91012C964FAD2C9760965FAD6097C8
:10CEF000D8016D917D918D919C910E9456CEF80143
:10CF000061937193819391938F01EE15FF0549F71A
:10CF100091012C964FAD2C9760965FAD60976D9602
:10CF20006CAD7DAD8EAD9FAD6D970E9456CE2996AE
:10CF3000AEADBFAD299792966D937D938D939C93E3
:10CF40009597A1966CAD7DAD8EAD9FADA1970E94DA
:10CF500021CC91012C964FAD2C9760965FAD6097D8
:10CF60000E9456CE0E94F5CB2996EEADFFAD2997D3
:10CF700060AF71AF82AF93AFEB962CAD3DAD4EADD0
:10CF80005FADEB9767966CAD7DAD8EAD9FAD67974E
:10CF90000E9488CB6B017C012996AEADBFAD29976D
:10CFA00014968D909D90AD90BC90179718962D91EA
:10CFB0003D914D915C911B97C757DF4F2883398373
:10CFC0004A835B83C958D040C058DF4F28813981DC
:10CFD0004A815B81C058D040232B242B252B31F56F
:10CFE00081149104A104B10409F5C757DF4F88816A
:10CFF0009981AA81BB81C958D040892B8A2B8B2B60
:10D00000A9F42091ED0E3091EE0E4091EF0E50916B
:10D01000F00EC701B6010E9456CE0E946ECB299633
:10D020000EAD1FAD29970C5B1F4F20C029960EAD8A
:10D030001FAD29970C5B1F4FC458DF4F28813981E2
:10D040004A815B81CC57D040232B242B252BB9F46C
:10D050002091E90E3091EA0E4091EB0E5091EC0ECA
:10D06000C701B6010E9456CE0E946ECB0E94F5CB3E
:10D07000D8016D937D938D939C93139715C0209148
:10D08000F10E3091F20E4091F30E5091F40EC70163
:10D09000B6010E9456CE0E946ECB0E94F5CBF801DD
:10D0A00060837183828393832996EEADFFAD2997C8
:10D0B000EC5BFF4F2081C357DF4F2883CD58D04012
:10D0C0003181C257DF4F3883CE58D0404281C1579B
:10D0D000DF4F4883CF58D0405381C057DF4F58832C
:10D0E000C059D0408091C90E2C968FAF2C9790914B
:10D0F000CA0E60969FAF6097A091CB0E6896AFAFB7
:10D100006897B091CC0E6A96BFAF6A97E091CD0E4A
:10D110006E96EFAF6E97F091CE0EA296FFAFA297EC
:10D120002091CF0EA6962FAFA6973091D00EAA963B
:10D130003FAFAA974091D10EAE964FAFAE975091A8
:10D14000D20EE2965FAFE2978091D30EE6968FAF54
:10D15000E6979091D40EEC969FAFEC973090D50E59
:10D160002090D60E0091D70E1091D80EC357DF4FE6
:10D170006881CD58D040C257DF4F7881CE58D0401B
:10D18000C157DF4F8881CF58D040C057DF4F9881BB
:10D19000C059D0400E9421CC2B013C01C058DF4F28
:10D1A000688179818A819B81C058D0400E9423CCBC
:10D1B0009B01AC01C301B2010E9456CE67962CAD13
:10D1C0003DAD4EAD5FAD67970E9488CB2B013C0112
:10D1D0002C966FAD2C9760967FAD609768968FAD5B
:10D1E00068976A969FAD6A970E9421CC9B01AC011B
:10D1F000C301B2010E9484CD181604F1C357DF4F5A
:10D20000A881CD58D0402C96AFAF2C97C257DF4F96
:10D21000B881CE58D0406096BFAF6097C157DF4FFE
:10D22000E881CF58D0406896EFAF6897C057DF4F7E
:10D23000F881C059D0406A96FFAF6A972C966FADBF
:10D240002C9760967FAD609768968FAD68976A96C9
:10D250009FAD6A970E9421CC2B013C01C501B4010E
:10D260000E9423CC9B01AC01C301B2010E9456CEA7
:10D2700067962CAD3DAD4EAD5FAD67970E9488CBF4
:10D280004B015C016E966FAD6E97A2967FADA29733
:10D29000A6968FADA697AA969FADAA970E9421CC7D
:10D2A0009B01AC01C501B4010E9484CD1816C4F0E5
:10D2B0002C962FAD2C976E962FAF6E9760963FAD44
:10D2C0006097A2963FAFA29768964FAD6897A696D3
:10D2D0004FAFA6976A965FAD6A97AA965FAFAA9777
:10D2E0006E966FAD6E97A2967FADA297A6968FAD04
:10D2F000A697AA969FADAA970E9421CC4B015C01EC
:10D30000C757DF4F688179818A819B81C958D04096
:10D310000E9423CC9B01AC01C501B4010E9456CEF2
:10D3200067962CAD3DAD4EAD5FAD67970E9488CB43
:10D330004B015C01AE966FADAE97E2967FADE29782
:10D34000E6968FADE697EC969FADEC970E9421CCC8
:10D350009B01AC01C501B4010E9484CD1816C4F034
:10D360006E968FAD6E97AE968FAFAE97A2969FAD2D
:10D37000A297E2969FAFE297A696AFADA697E696E4
:10D38000AFAFE697AA96BFADAA97EC96BFAFEC9762
:10D39000AE966FADAE97E2967FADE297E6968FAD13
:10D3A000E697EC969FADEC970E9421CC4B015C0177
:10D3B000C458DF4F688179818A819B81CC57D040E6
:10D3C0000E9423CC9B01AC01C501B4010E9456CE42
:10D3D00067962CAD3DAD4EAD5FAD67970E9488CB93
:10D3E0004B015C01632D722DC8010E9421CC9B0171
:10D3F000AC01C501B4010E9484CD181664F0AE964C
:10D400003FACAE97E2962FACE297E6960FADE6976B
:10D41000EC961FADEC972996EEADFFAD2997EC5B2E
:10D42000FF4F3082218202831383632D722DC80146
:10D430000E9421CC4B015C01A70196010E9488CB80
:10D44000C757DF4F688379838A839B83C958D0404D
:10D450002996EEADFFAD299762AB73AB84AB95AB6C
:10D4600020E030E040E85BE4C501B4010E9456CE04
:10D4700020E034E244EF59E40E9488CB0E94F0CBD4
:10D480002996AEADBFAD29975C966D937D938D9334
:10D490009C935F972091E50E3091E60E4091E70E48
:10D4A0005091E80EA5962CAF3DAF4EAF5FAFA5975C
:10D4B00020E030E040E05FE3A5966CAD7DAD8EAD41
:10D4C0009FADA5970E9456CE64966FAF6497272EA6
:10D4D0002C968FAF2C97392E8091E10E9091E20E11
:10D4E000A091E30EB091E40EA9968CAF9DAFAEAFC4
:10D4F000BFAFA99720E030E040E05FE3BC01CD0181
:10D500000E9456CE162F072FF82EE92E2091DD0E01
:10D510003091DE0E4091DF0E5091E00EAD962CAFB3
:10D520003DAF4EAF5FAFAD9720E030E040E05FE34E
:10D53000AD966CAD7DAD8EAD9FADAD970E9456CED4
:10D54000D62EC72EB82EA92E89A19AA1ABA1BCA117
:10D55000E1968CAF9DAFAEAFBFAFE1972DA13EA1DD
:10D560004FA158A5E5962CAF3DAF4EAF5FAFE59705
:10D57000BC01CD019F77212F302F4F2D5E2D0E94B2
:10D5800084CD1816C4F4212F302F4F2D5E2D6496B4
:10D590006FAD6497722D2C968FAD2C97932D0E94B2
:10D5A00081CB87FD08C064961FAF6497202E2C9610
:10D5B000FFAE2C973E2C2D2D3C2D4B2D5A2DE59654
:10D5C0006CAD7DAD8EAD9FADE5979F770E9484CD0C
:10D5D0001816C4F42D2D3C2D4B2D5A2D64966FAD8D
:10D5E0006497722D2C968FAD2C97932D0E9481CB32
:10D5F00087FD08C06496DFAE64972C2C2C96BFAED6
:10D600002C973A2C2996AEADBFAD29979296BC9136
:10D610006096BFAF60972996EEADFFAD2997F3A155
:10D620006896FFAF68972996AEADBFAD29979496DF
:10D63000BC916A96BFAF6A972996EEADFFAD299768
:10D64000F5A16E96FFAF6E9760962FAD60976896C6
:10D650003FAD68974B2F5F2F64966FAD6497722D27
:10D660002C968FAD2C97932D0E9481CB87FD12C0F5
:10D6700060962FAD609764962FAF649768962FAC35
:10D6800068976A963FAD6A972C963FAF2C976E9637
:10D690003FAC6E97CB57DF4F48815981C558D0407A
:10D6A000423051050CF434C15091D209E6965FAF77
:10D6B000E6978091D309EC968FAFEC979091D409BF
:10D6C000ED969FAFED97A091D509C058DF4FA88385
:10D6D000C058D04027E137EB41ED58E3E6966FADF7
:10D6E000E697782F892F9A2F0E9484CD18160CF078
:10D6F0000FC12091D6093091D7094091D809509196
:10D70000D909698D7A8D8B8D9C8D0E94A7CA2B01BA
:10D710003C012091DA093091DB094091DC095091FC
:10D72000DD096D8D7E8D8F8D98A10E94A7CA4B015A
:10D730005C012091DE093091DF094091E0095091B0
:10D74000E109E1966CAD7DAD8EAD9FADE1970E9494
:10D75000A7CA6B017C01E894F7F82091E2093091A7
:10D76000E3094091E4095091E509E5966CAD7DAD82
:10D770008EAD9FADE5970E94A7CA9B01AC015F7774
:10D78000CB57DF4F288339834A835B83C558D0400A
:10D79000A3019201C301B2010E9456CE2B013C01AC
:10D7A000A5019401C501B4010E9456CE9B01AC01B4
:10D7B000C301B2010E94A8CA0E94C3CE4B015C0102
:10D7C000A5962CAD3DAD4EAD5FADA5970E9484CD25
:10D7D00018166CF4A5019401A5966CAD7DAD8EADC7
:10D7E0009FADA5970E9488CB4B015C0106C0812CA0
:10D7F000912C50E8A52E6FE3B62EA9962CAD3DAD29
:10D800004EAD5FADA997C701B6010E9484CD181631
:10D81000E4F4A7019601A9966CAD7DAD8EAD9FADE8
:10D82000A9970E9488CB162F072FF82EE92E262FB6
:10D83000372F482F592FB401C5010E9481CB87FD96
:10D8400004C0812E902EAF2CBE2CAD962CAD3DADDC
:10D850004EAD5FADAD97CB57DF4F688179818A813F
:10D860009B81C558D0400E9484CD1816E4F4CB5754
:10D87000DF4F288139814A815B81C558D040AD9600
:10D880006CAD7DAD8EAD9FADAD970E9488CB7B0119
:10D890008C019B01AC01B401C5010E9481CB87FDC5
:10D8A00002C0470158019401A50160966FAD6097D1
:10D8B00068967FAD68976A968FAD6A976E969FADB2
:10D8C0006E970E9456CE7B018C019B01AC01E696BF
:10D8D0006FADE697EC967FADEC97ED968FADED973B
:10D8E000C058DF4F9881C058D0400E9481CB87FF3D
:10D8F00017C0E696EFACE697EC96FFACEC97ED968A
:10D900000FADED97C058DF4F1881C058D04008C008
:10D910006496EFAC6497F22C2C960FAD2C97132DD8
:10D92000C701D8012996EEADFFAD299782A793A72D
:10D93000A4A7B5A7C757DF4F688179818A819B81EA
:10D94000C958D04090589B01AC010E94A8CAEB96E0
:10D950002CAD3DAD4EAD5FADEB970E9456CE9B0119
:10D96000AC016BE077ED83E29BE30E94A7CA0E94C3
:10D97000C3CE5B016C019B01AC01B701C8010E94E1
:10D9800081CB87FF02C0902E03C075019C2C1D2DFA
:10D99000C701A92DB12F2996EEADFFAD299786A31A
:10D9A00097A3A0A7B1A701E09501A60160966FAD6E
:10D9B000609768967FAD68976A968FAD6A976E9606
:10D9C0009FAD6E970E9481CB18160CF400E029964B
:10D9D000AEADBFAD2997D7960C93D79781E0D69679
:10D9E0008C93898D9A8DAB8DBC8D8093D609909345
:10D9F000D709A093D809B093D9098D8D9E8DAF8D8D
:10DA0000B8A18093DA099093DB09A093DC09B09365
:10DA1000DD09E1962CAD3DAD4EAD5FADE1972093B4
:10DA2000DE093093DF094093E0095093E109E59660
:10DA30008CAD9DADAEADBFADE5978093E2099093FF
:10DA4000E309A093E409B093E50960968FAD609770
:10DA500068969FAD68976A96AFAD6A976E96BFADB0
:10DA60006E978093D2099093D309A093D409B09371
:10DA7000D5099C01AD0164966FAD6497722D2C960B
:10DA80008FAD2C97932D0E9488CB2B013C01609683
:10DA90002FAD609768963FAD68976A964FAD6A97CD
:10DAA0006E965FAD6E97B701892D912F0E9488CB3E
:10DAB000AB01BC019301820129968EAD9FAD2997E0
:10DAC0000E94075CCC57DF4F9881C458D040909398
:10DAD000F70989A59AA5ABA5BCA58093E609909303
:10DAE000E709A093E809B093E9098DA59EA5AFA524
:10DAF000B8A98093EA099093EB09A093EC09B0933D
:10DB0000ED0989A99AA9ABA9BCA98093EE099093C4
:10DB1000EF09A093F009B093F1098DA99EA9AFA9CF
:10DB2000B8AD8093F2099093F309A093F409B093F0
:10DB3000F5090E94B95F0E94BB92C057DF4F0FB634
:10DB4000F894DEBF0FBECDBFDF91CF911F910F9133
:10DB5000FF90EF90DF90CF90BF90AF909F908F900D
:10DB60007F906F905F904F903F902F9008956F92AD
:10DB70007F928F929F92AF92BF92CF92DF92EF925D
:10DB8000FF920F931F93CF93DF93CDB7DEB7A49788
:10DB90000FB6F894DEBF0FBECDBF3C0182E090E02F
:10DBA0000E94F2996B017C0181E090E00E94F29961
:10DBB0004B015C0180E090E00E94F299AB01BC0156
:10DBC00095018401C3010E9450BF8DB79EB7849711
:10DBD0000FB6F8949EBF0FBE8DBFADB7BEB71196FE
:10DBE00084E2E3E4F2E001900D928A95E1F7CE0140
:10DBF00001960E9433C38DB79EB784960FB6F894F2
:10DC0000DEBF0FBECDBF84970FB6F8949EBF0FBE88
:10DC10008DBFADB7BEB7119684E2FE01319601907B
:10DC20000D928A95E1F7C3010E94E6BF0FB6F89402
:10DC3000DEBF0FBECDBFC301A4960FB6F894DEBF02
:10DC40000FBECDBFDF91CF911F910F91FF90EF904D
:10DC5000DF90CF90BF90AF909F908F907F906F900C
:10DC600008954F925F926F927F928F929F92AF92A0
:10DC7000BF92CF92DF92EF92FF920F931F93CF93B9
:10DC8000DF93CDB7DEB76C970FB6F894DEBF0FBE4B
:10DC9000CDBF698B7A8B8B8B9C8B2D8B3E8B4F8B67
:10DCA000588FE98EFA8E0B8F1C8F8601CE01499614
:10DCB0009F938F9304979F938F9304979F938F9332
:10DCC0008DB79EB784970FB6F8949EBF0FBE8DBFD9
:10DCD000ADB7BEB7119684E2E3E4F2E001900D9295
:10DCE0008A95E1F70E942BC10FB6F894DEBF0FBEF4
:10DCF000CDBF2091090F30910A0F40910B0F509129
:10DD00000C0F69897A898B899C890E9456CE0E9462
:10DD100026CE4B015C016093E6097093E70980937E
:10DD2000E8099093E90920910D0F30910E0F409171
:10DD30000F0F5091100F6D897E898F89988D0E94E9
:10DD400056CE0E9426CE2B013C016093EA097093C7
:10DD5000EB098093EC099093ED092091110F30911C
:10DD6000120F4091130F5091140F698D7A8D8B8D86
:10DD70009C8D0E9456CE0E9426CE6B017C01609342
:10DD8000EE097093EF098093F0099093F1092091C7
:10DD9000150F3091160F4091170F5091180FF80181
:10DDA00060817181828193810E9456CE0E9426CE2D
:10DDB0006093F2097093F3098093F4099093F50945
:10DDC0000E9423CC0E94F0CB69837A838B839C834F
:10DDD000C701B6010E9423CC0E94F0CB6D837E83E5
:10DDE0008F839887C301B2010E9423CC0E94F0CB9D
:10DDF00069877A878B879C87C501B4010E9423CCF1
:10DE00000E94F0CB6D877E878F87988B9E012F5F56
:10DE10003F4FAE014B5F5F4FBE01675F7F4FCE014B
:10DE20000D960E9497991092D2091092D3091092E0
:10DE3000D4091092D5091092D6091092D7091092E0
:10DE4000D8091092D9091092DA091092DB091092C0
:10DE5000DC091092DD091092DE091092DF091092A0
:10DE6000E0091092E1091092E2091092E309109280
:10DE7000E4091092E5096C960FB6F894DEBF0FBE68
:10DE8000CDBFDF91CF911F910F91FF90EF90DF9069
:10DE9000CF90BF90AF909F908F907F906F905F904A
:10DEA0004F9008952091150F3091160F4091170F44
:10DEB0005091180FFC0160817181828193810E94D1
:10DEC00056CE0E9426CE6093F2097093F309809398
:10DED000F4099093F50982EF99E00C94D399CF92CD
:10DEE000DF92EF92FF920F931F93CF93DF9300D0B7
:10DEF0001F92CDB7DEB709EFC02E0EE0D02E89E01D
:10DF0000E82E8FE0F82E09EC1EE0F6016191719188
:10DF1000819191916F01F70121913191419151913D
:10DF20007F0129833A834B835C830E9421CC298122
:10DF30003A814B815C810E9456CE0E94F5CBF8015C
:10DF400061937193819391938F01F9E0CF16FFE074
:10DF5000DF06D9F60F900F900F900F90DF91CF91C1
:10DF60001F910F91FF90EF90DF90CF9008954F9207
:10DF70005F926F927F92AF92BF92CF92DF92EF92B9
:10DF8000FF920F931F93CF93DF93EC018B017A01E4
:10DF900063E070E00E943FCF5C01F801D70120E010
:10DFA00030E028173907A4F44081518162817381E0
:10DFB0004D905D906D907C9013974192519261923B
:10DFC00071924D935D936D937D932F5F3F4FE9CF9A
:10DFD000DC01AA0FBB1FAA0FBB1FF801EA0FFB1F32
:10DFE000AE0DBF1DAC16BD060CF040C04081518186
:10DFF000628173810D911D912D913C911397008346
:10E000001183228333834D935D936D937C93139798
:10E01000448155816681778114960D911D912D91D2
:10E020003C911797048315832683378314964D9369
:10E030005D936D937C9317970085118522853385B9
:10E040001896CD90DD90ED90FC901B97C086D18600
:10E05000E286F38618960D931D932D933C931B97A0
:10E0600083E0A80EB11C3C961C96BCCFDF91CF91EB
:10E070001F910F91FF90EF90DF90CF90BF90AF90E6
:10E080007F906F905F904F9008952F923F924F92A4
:10E090005F926F927F928F929F92AF92BF92CF9238
:10E0A000DF92EF92FF920F931F93CF93DF9300D0F5
:10E0B00000D0CDB7DEB75C017C836B838A01FA01A7
:10E0C000C080D180E280F38020E030E0A901C70168
:10E0D000B6010E9481CB87FF04C0F7FAF094F7F8ED
:10E0E000F0949501220F331F220F331F3A832983A7
:10E0F0001E821D828D819E81EB81FC818E179F0780
:10E10000B4F5812C912C212C312C2A143B042CF5B4
:10E11000F801E80DF91D408051806280738020E095
:10E1200030E0A901C301B2010E9481CB87FF04C086
:10E1300077FA709477F87094A3019201C701B60141
:10E140000E9481CB87FF02C0730162013FEF231A57
:10E15000330A84E0880E911CD8CFED81FE81319680
:10E16000FE83ED8329813A81020F131FC3CFC701BC
:10E17000B60126960FB6F894DEBF0FBECDBFDF9175
:10E18000CF911F910F91FF90EF90DF90CF90BF90B4
:10E19000AF909F908F907F906F905F904F903F9047
:10E1A0002F9008952F923F924F925F926F927F929D
:10E1B0008F929F92AF92BF92CF92DF92EF92FF9297
:10E1C0000F931F93CF93DF937B01EE0CFF1CEE0C9C
:10E1D000FF1CE0E0F0E000E010E0041715073CF55C
:10E1E000A0E0B0E0212C312C5901AE0EBF1E4C0135
:10E1F0008E0E9F1E26163706ACF46501CA0EDB1E76
:10E20000E601488059806A807B806401CA0EDB1E6B
:10E21000E601488259826A827B82DFEF2D1A3D0A2D
:10E220001496E8CF0F5F1F4FEE0DFF1DD6CFDF9185
:10E23000CF911F910F91FF90EF90DF90CF90BF9003
:10E24000AF909F908F907F906F905F904F903F9096
:10E250002F9008952F923F924F925F926F927F92EC
:10E260008F929F92AF92BF92CF92DF92EF92FF92E6
:10E270000F931F93CF93DF9300D000D0CDB7DEB7BD
:10E280009E838D834A015B013901181619060CF033
:10E2900028C120E030E0A901C501B4010E9481CB72
:10E2A000882309F41EC10130110529F421E0C216AA
:10E2B000D10489F473C017FF0EC021E030E04D8116
:10E2C0005E81241B350B209FC001219F900D309F44
:10E2D000900D112402C080E090E0D7FE0EC021E036
:10E2E00030E0ED81FE812E1B3F0B2C9DA0012D9D6A
:10E2F000500D3C9D500D112402C040E050E09601AD
:10E30000220F331F220F331F3C832B83F801EE0FA4
:10E31000FF1FEE0FFF1FFA83E9838A01000F111F11
:10E32000000F111F0E0D1F1D7C01EE0CFF1CEE0CCB
:10E33000FF1CE60CF71C612C712CC12CD12C412C3C
:10E34000512C18012C0C3D1CF701E60DF71D208106
:10E35000318142815381C501B4010E9456CE9B0197
:10E36000AC01F10160817181828193810E94A8CA10
:10E37000F1016083718382839383FFEF4F1A5F0AF9
:10E380002B813C81C20ED31E49815A81640E751EB9
:10E390008D819E8148165906A1F6A3C0CD80DE80EE
:10E3A00093E0C922DD2413018701412C512C4C1428
:10E3B0005D04ECF4F10121913191419151911F01E2
:10E3C000C501B4010E9456CE9B01AC01F8016081E9
:10E3D0007181828193810E94A8CAF801619371932F
:10E3E000819391938F01FFEF4F1A5F0AE0CFC6012F
:10E3F000880F991F880F991F8701080F191F7C012B
:10E4000024E0E20EF11CE60CF71C4D815E81C4167F
:10E41000D5060CF066C0F701349720813181428126
:10E420005381C501B4010E9456CE9B01AC01F80195
:10E4300060817181828193810E94A8CAF801608302
:10E44000718382839383F7012081318142815381DB
:10E45000C501B4010E9456CE9B01AC01F801648154
:10E460007581868197810E94A8CAF80164837583AB
:10E4700086839783F7012481358146815781C501C1
:10E48000B4010E9456CE9B01AC01F80160857185F4
:10E49000828593850E94A8CAF80160877187828768
:10E4A0009387F7012085318542855385C501B401E5
:10E4B0000E9456CE9B01AC01F80164857585868566
:10E4C00097850E94A8CAF801648775878687978711
:10E4D000F4E0CF0ED11C005F1F4F20E1E20EF11CD3
:10E4E00094CF26960FB6F894DEBF0FBECDBFDF9156
:10E4F000CF911F910F91FF90EF90DF90CF90BF9041
:10E50000AF909F908F907F906F905F904F903F90D3
:10E510002F9008952F923F924F925F926F927F9229
:10E520008F929F92AF92BF92CF92DF92EF92FF9223
:10E530000F931F93CF93DF9300D01F92CDB7DEB719
:10E540007C015B016901181619060CF01DC14130F0
:10E55000510521F40130110579F46AC057FF0CC050
:10E5600081E090E08E199F09849F2001859F500CC7
:10E57000949F500C112402C0412C512C17FF0CC049
:10E5800021E030E02E193F09209FC001219F900D0E
:10E59000309F900D112402C080E090E01A01220CFF
:10E5A000331C220C331C9801220F331F220F331F00
:10E5B0003A832983440C551C440C551C4A0C5B1CA3
:10E5C0005C01AA0CBB1CAA0CBB1CAC0CBD1C00E063
:10E5D00010E0C12CD12C612C712C812C912C1C822F
:10E5E0001B82F201EC0DFD1DD501A00FB11F2D9175
:10E5F0003D914D915C9160817181828193810E94F6
:10E6000056CE9B01AC01B301C4010E94A8CA3B01D4
:10E610004C018B819C8101969C838B83C20CD31C03
:10E62000E981FA810E0F1F1F8E159F05D1F6B0C02C
:10E6300065E070E00E943FCF9C838B832C01BA82FF
:10E64000A9821901612C712C812C912C00E010E021
:10E650002B813C8102171307DCF4E981FA81619177
:10E66000719181919191FA83E983F1012191319125
:10E67000419151911F010E9456CE9B01AC01B30103
:10E68000C4010E94A8CA3B014C010F5F1F4FE0CF9D
:10E69000C901880F991F880F991F8501080F191F3D
:10E6A0001C012C0C3D1C4E145F040CF071C0F101D8
:10E6B0002081318142815381F801608171818281A1
:10E6C00093810E9456CE5B016C01F101248135815A
:10E6D00046815781F80164817581868197810E9406
:10E6E00056CE9B01AC01C601B5010E94A8CA5B01D0
:10E6F0006C01F1012085318542855385F8016085E3
:10E700007185828593850E9456CE9B01AC01C6011E
:10E71000B5010E94A8CA5B016C01F1012485358511
:10E7200046855785F80164857585868597850E949D
:10E7300056CE9B01AC01C601B5010E94A8CA5B017F
:10E740006C01F1012089318942895389F80160897E
:10E750007189828993890E9456CE9B01AC01C601C2
:10E76000B5010E94A8CA9B01AC01B301C4010E947B
:10E77000A8CA3B014C01F5E04F0E511C0C5E1F4F27
:10E7800024E1220E311C8FCF612C712C812C912C15
:10E79000B301C4010F900F900F900F90DF91CF91B4
:10E7A0001F910F91FF90EF90DF90CF90BF90AF90AF
:10E7B0009F908F907F906F905F904F903F902F90A1
:10E7C00008952F923F924F925F926F927F928F9215
:10E7D0009F92AF92BF92CF92DF92EF92FF920F93F0
:10E7E0001F93CF93DF9300D01F92CDB7DEB79C83EA
:10E7F0008B83181619060CF09AC0141615060CF027
:10E8000096C0019799F4FB01C080D180E280F3802B
:10E8100020E030E0A901C701B6010E9481CB87FF4B
:10E8200089C0F7FAF094F7F8F09484C0CA01880F11
:10E83000991F880F991F9A8389838B01212C312C72
:10E84000812C912CA0E8AA2EAFE3BA2E412C512C9A
:10E85000612C712CF801C080D180E280F38020E02F
:10E8600030E0A901C701B6010E9481CB882309F4D9
:10E8700044C020E030E0A901C701B6010E9481CB6D
:10E8800087FF04C0F7FAF094F7F8F094A701960117
:10E89000B201C3010E9481CB87FF1DC0A701960171
:10E8A000B201C3010E9488CB2B013C019B01AC014A
:10E8B000C501B4010E9456CEA30192010E9456CE1A
:10E8C00020E030E040E85FE30E94A8CA4B015C0111
:10E8D0002601370112C09201A301C701B6010E94AF
:10E8E00088CB9B01AC010E9456CE9B01AC01C501B7
:10E8F000B4010E94A8CA4B015C01FFEF2F1A3F0A26
:10E9000089819A81080F191FEB81FC812E163F0621
:10E9100009F0A0CFC501B4010E94C3CE9B01AC0198
:10E92000B201C3010E9456CE6B017C0103C0C12C11
:10E93000D12C7601C701B6010F900F900F900F9068
:10E94000DF91CF911F910F91FF90EF90DF90CF90CB
:10E95000BF90AF909F908F907F906F905F904F90FF
:10E960003F902F9008952F923F924F925F926F9217
:10E970007F928F929F92AF92BF92CF92DF92EF924F
:10E98000FF920F931F93CF93DF93CDB7DEB7E4973A
:10E990000FB6F894DEBF0FBECDBF9C878B877A87FA
:10E9A0006987588B4F8729011CA30BA315019C8EE7
:10E9B0008B8E6096EEADFFAD6097CF01815F984D75
:10E9C00021E030E08F319E4410F420E030E0CF01B0
:10E9D00060E177E20E943FCF61E070E07E8B6D8B5B
:10E9E000892B11F41E8A1D8ACF0168EE73E00E9404
:10E9F0003FCF8D599F4FA1E0B0E0BAA3A9A3873CB8
:10EA0000910510F41AA219A2CF0164E670E00E94E9
:10EA10003FCF099641E050E05E8F4D8F439710F451
:10EA20001E8E1D8ECF016AE070E00E943FCF61E034
:10EA300070E078A36F8F892B11F418A21F8E6F845A
:10EA4000788871E0671A7108461457040CF4320193
:10EA50006114710409F062C0232B51F0F701808129
:10EA60009181A281B381F60180839183A283B383D4
:10EA70002D893E89232B51F0F70180819181A2815C
:10EA8000B381F10180839183A283B3832F8D38A159
:10EA9000232B69F0F70180819181A281B3812E96A9
:10EAA000EEADFFAD2E9780839183A283B38329A11E
:10EAB0003AA1232BF9F0AB85BC858D909D90AD904C
:10EAC000BC9020E030E0A901C501B4010E9481CBD7
:10EAD000882391F0A5019401F70160817181828101
:10EAE00093810E9488CBAB8DBC8D6D937D938D936C
:10EAF0009C9313971D8202C0B1E0BD831D86ED8DEE
:10EB0000FE8DEF2B09F40BC42C96AEADBFAD2C9748
:10EB10001D921D921D921C92139701C4211531055F
:10EB200029F4ED89FE89EF2BB9F413C0F701D60162
:10EB300081E090E04F8558894817590794F3419137
:10EB40005191619171914D935D936D937D93019678
:10EB5000F1CF232BA1F46DC0F701D10181E090E04A
:10EB60006F85788968177907A4F341915191619174
:10EB700071914D935D936D937D930196F1CFA9852E
:10EB8000BA85A095B095AA0FBB1FAA0FBB1FBE8365
:10EB9000AD839301220F331F220F331FEBA1FCA182
:10EBA000E20FF31FFAABE9AB49855A854F5F5F4F20
:10EBB000C3010197849F5001859FB00C949FB00CB6
:10EBC0001124AA0CBB1CAA0CBB1C4B855C85A40E93
:10EBD000B51EB601620F731FA985BA858A9F4001D1
:10EBE0008B9F900C9A9F900C1124860C971C880C7C
:10EBF000991C880C991C840E951E18A61FA21EA293
:10EC00001DA21E861D86E1E0F0E0FA83E9836450D0
:10EC100071097CA76BA7F4E08F1A91082F853889BA
:10EC2000261937093CAB2BABA981BA816A167B0642
:10EC300034F48D899E89892B09F07CC09CC0E9A998
:10EC4000FAA94D855E85E40FF51F3497C080D18009
:10EC5000E280F38020E030E0A901C701B6010E9404
:10EC600081CB882309F44CC06DA17EA16A0D7B1D68
:10EC70007AA769A7DB018D919D910D90BC91A02D84
:10EC80008DA79EA7AFA7B8ABFB01C082D182E2825D
:10EC9000F38201E010E02BA53CA54D855E85240F95
:10ECA000351F3A8B298B41E050E06FA178A5680DA4
:10ECB000791D78876F838BA99CA9A981BA818A0F56
:10ECC0009B1F9C838B8326DC9058A70196010E9492
:10ECD00088CBAB01BC01CC24C394D12CE988FA8841
:10ECE0002F8138858B819C81B5DA2DA53EA54FA556
:10ECF00058A9A9A5BAA52D933D934D935C9313975D
:10ED0000E981FA813196FA83E9832D853E85245085
:10ED100031093E872D874DA15EA16D817E81460F11
:10ED2000571F5EA34DA38FA198A5860F971F98A785
:10ED30008FA37ACF2BA13CA138872F83A984BA84D3
:10ED40003FEFA31AB30AAA0CBB1CAA0CBB1C4B8531
:10ED50005C855A8349836F8578897E836D833E867F
:10ED60002D864A0181E090E09C838B838B819C817E
:10ED70006816790634F4E9A1FAA1EF2B09F06DC009
:10ED800060C0AF81B885CD90DD90ED90FD90B887E3
:10ED9000AF8320E030E0A901C701B6010E9481CB1A
:10EDA0008823A9F1A981BA812D913D914D915C9162
:10EDB0001397298B3A8B4B8B5C8BFD01C082D182E0
:10EDC000E282F38201E010E02D853E8541E050E0D3
:10EDD000B4018D819E819EDB9058A70196010E940F
:10EDE00088CBAB01BC01CC24C394D12CED84FE8430
:10EDF00094018D819E812EDA29893A894B895C891B
:10EE0000A981BA812D933D934D935C931397EB8128
:10EE1000FC813196FC83EB8329813A812A0D3B1DCD
:10EE20003A8329834D815E81415051095E834D8330
:10EE30008A0C9B1C6D857E856C5F7F4F7E876D87FE
:10EE400095CFAF8DB8A1AB2B91F1B1012E964EAD00
:10EE50005FAD2E9721E030E017C0B1014B8D5C8D86
:10EE600021E030E04216530664F3FB018191919159
:10EE7000A191B191BF01FA0181939193A193B193B3
:10EE8000AF012F5F3F4FEECF421653060CF441C047
:10EE9000FB0181919191A191B191BF01FA018193FF
:10EEA0009193A193B193AF012F5F3F4FEDCFED8DC4
:10EEB000FE8DEF2BC1F12F85388942165306E4F5FC
:10EEC0009201B201660F771F660F771FA101460FEF
:10EED000571F2C968EAD9FAD2C97680F791F80E041
:10EEE00090E02F5F3F4FAF85B889A217B3070CF4AE
:10EEF000F2C1FA01E80FF91FC080D180E280F380EF
:10EF0000FB01E80FF91FC082D182E282F3820496EE
:10EF1000E8CF2D8D3E8D232B71F6EF85F8894E16A7
:10EF20005F060CF4DDC1A9A1BAA1AB2BA1F462C0AC
:10EF30008D8D9E8D892BB9F32C96EEADFFAD2C9760
:10EF400081E090E04816590674F3119211921192E3
:10EF500011920196F7CFF201EE0FFF1FEE0FFF1F88
:10EF60002B8D3C8D2E0F3F1F3A8329832CEF498533
:10EF70005A852403B001259F700D11247AA369A33B
:10EF800040955095440F551F440F551F5E8B4D8B78
:10EF900029853A852F5F3F4FC2010197829F40012B
:10EFA000839F900C929F900C1124880C991C880CC4
:10EFB000991CAB85BC858A0E9B1EE985FA858E9FC0
:10EFC00050018F9FB00C9E9FB00C1124AA0CBB1C4B
:10EFD000AA0CBB1CAA0EBB1E12011A8A198A18861B
:10EFE0001F8221E030E03C832B83EB81FC814E16B5
:10EFF0005F061CF41D821D865CC0A2016B817C81B2
:10F00000461B570B5EA34DA32D823D86E989FA89E5
:10F01000E80DF91DC080D180E280F38020E030E06F
:10F02000A901C701B6010E9481CB882309F441C020
:10F03000A7019601A981BA819E918E917E916E91D0
:10F04000BA83A9830E9488CBE981FA8160837183A6
:10F0500082839383F1E02F16310489F0AB01BC0168
:10F060007058CC24C394D12CEB8CFC8C01E010E0C4
:10F070002F8138852A0D3B1D8DA19EA1EBD82B81B8
:10F080003C812F5F3F4F3C832B8331E0231A3108B3
:10F090004F81588569A17AA1460F571F58874F8322
:10F0A00089899A89AD89BE898A0F9B1F9A8B898B22
:10F0B0009CCF2D8D3E8D232B29F44F8D58A1452BB0
:10F0C00009F42DC169857A8560957095660F771F63
:10F0D000660F771F7A83698389859A8501969301E4
:10F0E00021503109289F1001299F300C389F300C86
:10F0F0001124220C331C220C331C8B859C85280E7A
:10F10000391EC301880F991F880F991FABA1BCA19D
:10F11000A80FB91FBCA3ABA32C96EEADFFAD2C97E7
:10F12000E80FF91FF88FEF8B49855A85249F20013E
:10F13000259F500C349F500C1124460C571C440C36
:10F14000551C440C551C6B857C85460E571E2E960F
:10F15000AEADBFAD2E97A80FB91F1C821B821C86B7
:10F160001B86E1E0F0E0FA87E9871497BA8FA98F50
:10F17000F4E04F1A51082F85388926193709388B42
:10F180002F874F89588D44505109588F4F8B89854F
:10F190009A85681679060CF4C2C0EBA1FCA16B85B8
:10F1A0007C85E60FF71F3497C080D180E280F38022
:10F1B00020E030E0A901C701B6010E9481CB88237D
:10F1C00009F473C0D1018D919D910D90BC91A02D3A
:10F1D000898B9A8BAB8BBC8BF101C082D182E2828E
:10F1E000F3822D8D3E8D232B49F101E010E04F89F4
:10F1F000588D6B857C85460F571F58874F839A0122
:10F2000041E050E08B809C80840C951CB401AF845D
:10F21000B88889859A85A80EB91EC5017BD99058F2
:10F22000A70196010E9488CBAB01BC01CC24C394FA
:10F23000D12CEF80F8849401C5010CD8AF8DB8A112
:10F24000AB2B49F101E010E0E98CFA8CEB85FC85F1
:10F25000EE0EFF1E970141E050E08B809C80840CF5
:10F26000951CB401AF84B88889859A85A80EB91E0B
:10F27000C50150D99058D1012D913D914D915C918E
:10F280000E9488CBAB01BC01CC24C394D12C940147
:10F29000C5010E942A7129893A894B895C89D1016B
:10F2A0002D933D934D935C931397E985FA853196A1
:10F2B000FA87E9872B853C85245031093C872B87C9
:10F2C00049815A81240E351E6B817C81640F751F24
:10F2D0007C836B835CCFAF8DB8A1AB2B09F42CCEB4
:10F2E000C201A201440F551F440F551F2E962EAD8B
:10F2F0003FAD2E97420F531F20E030E001966F85FF
:10F300007889681779070CF413CEFA01E20FF31F1E
:10F3100010821182128213822C5F3F4FEFCF8D81BA
:10F320009D85E4960FB6F894DEBF0FBECDBFDF918A
:10F33000CF911F910F91FF90EF90DF90CF90BF90F2
:10F34000AF909F908F907F906F905F904F903F9085
:10F350002F9008952F923F924F925F926F927F92DB
:10F360008F929F92AF92BF92CF92DF92EF92FF92D5
:10F370000F931F93CF93DF931F921F92CDB7DEB7EA
:10F380003A8329833801260165011401011511050D
:10F3900091F01F922EE62F93DF92AF92DF92AF9201
:10F3A0004201088D198D9301DEDA0F900F900F90B6
:10F3B0000F900F900F90F10180E090E029813A8149
:10F3C000821793074CF420813181319521953109C1
:10F3D000219331930196F2CF9301220F331F220F15
:10F3E000331F240D351D80E090E0A981BA816A1693
:10F3F0007B0664F4F901E80FF91F10821182128272
:10F4000013824FEF641A740A0496EFCF3201B101F0
:10F4100041E050E0E981FA81E417F507E4F1FB01EE
:10F42000208131811216130674F13195219531092D
:10F43000318320832417350731F1D3018D909D90BE
:10F44000AD90BC901397F901E150F04CEE0FFF1F07
:10F45000EE0FFF1FE40DF51DC080D180E280F38028
:10F46000CD92DD92ED92FC92139780829182A282DE
:10F47000B382F901E150F048EE0FFF1FE20DF31DDA
:10F4800020813181D2CF4F5F5F4F6E5F7F4FB4E0FD
:10F490006B0E711CBFCF0F900F90DF91CF911F911A
:10F4A0000F91FF90EF90DF90CF90BF90AF909F9023
:10F4B0008F907F906F905F904F903F902F90089526
:10F4C0002F923F924F925F926F927F928F929F9274
:10F4D000AF92BF92CF92DF92EF92FF920F931F9362
:10F4E000CF93DF934C016A017B013901181619068D
:10F4F0000CF0A3C00130110509F069C065E070E0AF
:10F500000E943FCFEC012C01590100E010E00C17E4
:10F510001D0794F4A7019601F50160817181828134
:10F5200093810E9456CEF5016193719381939193DB
:10F530005F010F5F1F4FEBCFCC0FDD1FCC0FDD1F27
:10F54000C60DD71D481459040CF077C0A7019601C9
:10F55000688179818A819B810E9456CE68837983F4
:10F560008A839B83A70196016C817D818E819F8117
:10F570000E9456CE6C837D838E839F83A701960164
:10F58000688579858A859B850E9456CE68877987AC
:10F590008A879B87A70196016C857D858E859F85CF
:10F5A0000E9456CE6C877D878E879F87A701960124
:10F5B000688979898A899B890E9456CE688B798B64
:10F5C0008A8B9B8BF5E04F0E511C6496BBCF17FFC7
:10F5D0000CC081E090E088199909809F2001819FEB
:10F5E000500C909F500C112402C0412C512C18013A
:10F5F000220C331C220C331C440C551C440C551C8F
:10F60000460C571C00E010E0C0E0D0E05201A00E14
:10F61000B11EA7019601F5016081718182819381FC
:10F620000E9456CEF5016083718382839383219675
:10F63000020D131DC815D90549F7DF91CF911F9110
:10F640000F91FF90EF90DF90CF90BF90AF909F9081
:10F650008F907F906F905F904F903F902F90089584
:10F660002F923F924F925F926F927F928F929F92D2
:10F67000AF92BF92CF92DF92EF92FF920F931F93C0
:10F68000CF93DF93CDB7DEB7E6970FB6F894DEBF22
:10F690000FBECDBF9E838D837E8B6D8B1A013A8BFF
:10F6A000298B18A70FA3FC8EEB8EDAA6C9A6AB2870
:10F6B00009F4C8C087017C0166246394712CCC24B2
:10F6C000C394D12C29893A892C153D050CF44AC0E4
:10F6D000D8018D919C9197FF05C0222733272C19C3
:10F6E0003D0901C09601F8013183208318161906DF
:10F6F00084F5C614D704D1F0C30101972D893E8942
:10F70000829FB001839F700D929F700D1124660F30
:10F71000771F660F771F4D815E81640F751F12146E
:10F72000130424F4A701C1010E94B76FF301E15053
:10F73000F048EE0FFF1F8B8D9C8DE80FF91F808125
:10F740009181D8018D939C93D182C082BFEF6B1AB7
:10F750007B0AEFEFCE1ADE0A0E5F1F4FF4E0EF0ECA
:10F76000F11CB0CF4901880C991C4B8D5C8D840E27
:10F77000951E2CEF4D895E8924036001259FD00CD6
:10F78000112489899A890197849F8001859F100D92
:10F79000949F100D1124000F111F000F111F8D8158
:10F7A0009E81080F191F49885A887201A12CB12C1B
:10F7B0001E141F040CF04BC0D4019E918E914D017C
:10F7C00097FF3AC09195819591098D939C93E4148C
:10F7D000F50479F1A501400F511FC2010197ED8990
:10F7E000FE898E9FB0018F9F700D9E9F700D11241A
:10F7F000660F771F660F771F2D813E81620F731F83
:10F80000121413041CF4C1010E94B76FF201E150FD
:10F81000F048EE0FFF1F4B8D5C8DE40FF51F8081CC
:10F820009181D4012D913C911197318320838D9347
:10F830009C93B1E04B1A5108E1E0EE1AF108AC0CD0
:10F84000BD1CB6CF412C512C66246394712C2D899C
:10F850003E89220F331F220F331F388F2F8BCD800D
:10F86000DE80C21AD30A9301215031094D895E8985
:10F87000249FC001259F900D349F900D1124880F67
:10F88000991F880F991FC80ED91E4301880C991C17
:10F89000880C991CAFA0B8A4A80CB91C930100E077
:10F8A00010E0E12CF12C8F89988DE80EF91E0C5F89
:10F8B0001F4F42165306BCF041E050E0B6016E0DFA
:10F8C0007F1DC1012CAB3DAB0E94E173F501E00F40
:10F8D000F11F389760837183828393832CA93DA99C
:10F8E0002F5F3F4FE0CFA9A5BAA58A0E9B1E9301BB
:10F8F00080E090E00496421653069CF0F501E80F74
:10F90000F91F38974081518162817381F401E80FBA
:10F91000F91F389740835183628373832F5F3F4F72
:10F92000E9CFE989FA89F8ABEFA72E163F0614F460
:10F9300038AA2FA62F89388D2C5F3F4F3AAB29ABC1
:10F940004FA158A55A8F498F89A59AA59AA389A333
:10F95000D1011197B8A3AF8FED81FE81FEA3EDA376
:10F96000F88BEF87FC8BEB8B21E030E03A83298327
:10F97000A981BA81EFA5F8A9EA17FB070CF461C2C7
:10F9800049815A81461557050CF49EC0441555050A
:10F990000CF09AC05E8F4D8F8A01E12CF12C1D86F0
:10F9A000812CA12CB12CC98CDA8C54E0C50ED11C51
:10F9B000F601EE0DFF1D349780818B8391819F832B
:10F9C0009280A381A9879C01492D5A2F6D85782D9E
:10F9D000C5010E9481CB87FD06C0BD85BB838F8298
:10F9E0009A2CB98602C01E8F0D8F0F5F1F4FE4E067
:10F9F000EE0EF11C4016510634F0FB81FD878F801E
:10FA0000A92CB984D5CF2D8D3E8D49815A812417DB
:10FA1000350709F459C0C9010197AD89BE898A9F8C
:10FA2000A0018B9F500D9A9F500D1124440F551F1C
:10FA3000440F551FED81FE814E0F5F1F12141304FA
:10FA40002CF46DA17EA1C1010E94B76F8D8D9E8D9A
:10FA50008150904C880F991F880F991FA98DBA8DDE
:10FA60004D915D916D917C91EFA1F8A5E80FF91F83
:10FA70004083518362837383E9A1FAA1408151815C
:10FA800062817381E9A5FAA5E80FF91F40835183CC
:10FA9000628373834D8D5E8D41505048440F551FD6
:10FAA0002B8D3C8D420F531FDA018D919C91119744
:10FAB000E981FA81EE0FFF1FE20FF31F32912291CD
:10FAC0002D933C9391838083E98DFA8D119211924D
:10FAD00011921192FA8FE98F29813A81221533050B
:10FAE00009F488C14F8D58A14F5F5F4F5CA34BA3B2
:10FAF00041E050E06B897C898BA19CA10E94E1735D
:10FB000069877A878B879C8720E030E0A9010E9473
:10FB100081CB882309F46EC1AF85B889CD90DD9083
:10FB2000ED90FC9020E030E0A901C701B6010E94F1
:10FB300081CB8823E1F020E030E0A901C701B601C4
:10FB40000E9481CB87FF05C020E030E040E85FEBFA
:10FB500004C020E030E040E85FE369857A858B856A
:10FB60009C850E9456CE69877A878B879C872985DA
:10FB70003A854B855C8560E070E080E89FE30E94F9
:10FB800088CBAB01BC0101E010E02B893C898BA143
:10FB90009CA196DC20E030E040E85FE3EF85F88947
:10FBA00060817181828193810E94A8CAAF85B889E2
:10FBB0006D937D938D939C931397E981FA81319690
:10FBC000F887EF832B893C894F89588D240F351F87
:10FBD0003C832B8389A19AA104969E8F8D8FA98D3A
:10FBE000BA8DBE87AD872F81388549895A894217DA
:10FBF00053070CF4E5C001E010E02B813C8141E0AB
:10FC000050E06B897C898BA19CA10E948A729058DC
:10FC1000EF85F88920813181428153810E9488CB10
:10FC2000AB01BC01CC24C394D12CEB80FC802B898C
:10FC30003C898BA19CA10E942A712F8138852615B1
:10FC400037050CF4A3C0421653060CF49FC0AD85D3
:10FC5000BE85CD90DD90ED90FC9020E030E0A901D4
:10FC6000C701B6010E9481CB882309F48FC0EB81C4
:10FC7000FC8180809180A280B38020E030E0A901E7
:10FC8000C501B4010E9481CB87FF04C0C501B40146
:10FC9000905802C0C501B401A70196010E9488CB0B
:10FCA0009B01AC010E9456CE9B01AC0160E070E06C
:10FCB00080E89FE30E94A7CA8B015C0120E030E04E
:10FCC000A9010E9484CD18161CF4AEAABBAA04C0D8
:10FCD00000E010E01EAA1BAAAD8DBE8D2D913D91B6
:10FCE0004D915C91C701B6010E9488CB4B015C012C
:10FCF0002DEC3CEC4CE45DE3B8018EA99BA90E947D
:10FD000056CE6BA77CA78DA79EA7A5019401C50120
:10FD1000B4010E9456CE9B01AC016BA57CA58DA5BC
:10FD20009EA50E9456CE20E030E040E85FE30E94AE
:10FD3000A8CA20E030E040E85FE30E9481CB88233E
:10FD400071F0B8018EA99BA90E94C3CE9B01AC01A2
:10FD5000C701B6010E9456CEED85FE8513C041E075
:10FD600050E06B817C816C5F7F4F8F8D98A10E94EA
:10FD7000E173AD85BE856D937D938D939C931397B1
:10FD8000ED8DFE8D60837183828393832F8138850F
:10FD90002F5F3F4F38872F834D855E854C5F5F4FC8
:10FDA0005E874D878D8D9E8D04969E8F8D8FAB8146
:10FDB000BC81EF89F88DAE0FBF1FBC83AB8313CF1F
:10FDC000EF85F88980819181A281B381298D3A8D57
:10FDD00024503109F90180839183A283B3838985FB
:10FDE0009A85AB85BC85B058EF85F889808391836F
:10FDF000A283B38329813A812F5F3F4F3A832983BE
:10FE00004B895C8989A99AA9480F591F5C8B4B8B38
:10FE1000AF85B889A80FB91FB88BAF87E9A1FAA140
:10FE20003496FAA3E9A32DA13EA14F89588D240F42
:10FE3000351F3EA32DA38F8D98A1019798A38F8F77
:10FE400097CDE6960FB6F894DEBF0FBECDBFDF911B
:10FE5000CF911F910F91FF90EF90DF90CF90BF90C7
:10FE6000AF909F908F907F906F905F904F903F905A
:10FE70002F9008952F923F924F925F926F927F92B0
:10FE80008F929F92AF92BF92CF92DF92EF92FF92AA
:10FE90000F931F93CF93DF93CDB7DEB72C970FB699
:10FEA000F894DEBF0FBECDBF9C838B837E836D83B2
:10FEB0005A8349833901E986FA860B871C87D886DD
:10FEC000CF82750184014DB65EB6C901880F991FB6
:10FED000880F991F2DB73EB7281B390B0FB6F89422
:10FEE0003EBF0FBE2DBF8DB79EB701966C01F501C9
:10FEF00080E090E08615970524F411921192019606
:10FF0000F9CFAA24A394B12C930149815A816D8120
:10FF10007E818B819C81A4DBEF81F8851182108228
:10FF2000130129813A81261537050CF419010D8139
:10FF30001E810F5F1F4F000F111F000F111F8B81BC
:10FF40009C819A838983612C712C621473040CF058
:10FF500040C0E981FA8180809180A280B38020E056
:10FF600030E0A901C501B4010E9481CB87FF04C024
:10FF7000B7FAB094B7F8B094EB81FC81C080D1801F
:10FF8000E280F38020E030E0A901C701B6010E94C1
:10FF900081CBA701960187FD505889819A81800FF6
:10FFA000911F9A83898369857A858B859C850E94B8
:10FFB00056CE9B01AC01C501B4010E9481CB18163D
:10FFC00044F49FEF691A790AEF81F88571826082A3
:10FFD000BCCF0FB6F8945EBE0FBE4DBE0FB6F89400
:10FFE0005EBE0FBE4DBE2C960FB6F894DEBF0FBEA0
:10FFF000CDBFDF91CF911F910F91FF90EF90DF90D8
:020000021000EC
:10000000CF90BF90AF909F908F907F906F905F90B8
:100010004F903F902F9008952F923F924F925F9272
:100020006F927F928F929F92AF92BF92CF92DF9208
:10003000EF92FF920F931F93CF93DF93CDB7DEB76D
:100040002A970FB6F894DEBF0FBECDBF9A8389837F
:100050002B011A013901DC82CB82B886AF829A86E5
:1000600089868CA18D839DA19E838EA19FA16417FB
:10007000750754F11216130654F51816190654F59F
:10008000019739F48D809E80AAA0BBA089819A81B6
:10009000F1DEEB81FC8100811181FE81FF938D8176
:1000A0008F938AA09BA0A8A0B9A0C984DA84EF800E
:1000B000F8849301A101B20189819A814BD90F90F3
:1000C0000F9080E090E008C08FEF9FEF05C08EEFAB
:1000D0009FEF02C08DEF9FEF2A960FB6F894DEBF18
:1000E0000FBECDBFDF91CF911F910F91FF90EF9089
:1000F000DF90CF90BF90AF909F908F907F906F9048
:100100005F904F903F902F9008952F923F924F9283
:100110005F926F927F928F929F92AF92BF92CF9297
:10012000DF92EF92FF920F931F93CF93DF9300D054
:100130001F92CDB7DEB74C013B012A014DB75EB728
:100140005C834B83469EC001479E900D569E900D4A
:100150001124880F991F880F991F481B590B0FB640
:10016000F8945EBF0FBE4DBF8DB79EB701961C01C0
:10017000C201880F991F880F991F481B590B0FB692
:10018000F8945EBF0FBE4DBF8DB79EB701966C0150
:10019000C301880F991F880F991F481B590B0FB671
:1001A000F8945EBF0FBE4DBF8DB79EB701967C0120
:1001B000C201880F991F481B590B0FB6F8945EBFF8
:1001C0000FBE4DBF8DB79EB701965C01A201B30172
:1001D000C1010E94D270A101B201C3010E94457009
:1001E0009B01AC0160E070E080E895E20E9488CB62
:1001F0001F9221E02F93DF92CF92BF92AF92FF9296
:10020000EF9258019E012F5F3F4F69017B018C01E6
:100210009201A301B301C101FFDE4DB75EB7485F94
:100220005F4F0FB6F8945EBF0FBE4DBF8B819C81B0
:100230000FB6F8949EBF0FBE8DBF0F900F900F901A
:100240000F90DF91CF911F910F91FF90EF90DF9072
:10025000CF90BF90AF909F908F907F906F905F9066
:100260004F903F902F9008958FEF8EBD0DB407FEF5
:10027000FDCF8EB508958EBD0DB407FEFDCF089558
:1002800061E0FC0180810C94F5C9FC012281322FD0
:10029000306A36953CBD20FD06C031E0263009F4B9
:1002A00030E0232F01C020E02DBD60E0FC01808103
:1002B0000C94F5C9CF92DF92EF92FF920F931F93A8
:1002C000CF93DF93EC018B017A010E94E5C76B01AC
:1002D000CBDF8B838F3F49F40E94E5C76C197D0902
:1002E0006D327140A8F381E103C08E3F31F08FE0A1
:1002F0008983CE01C5DF80E024C0E114F104E1F080
:1003000081E0E81AF1088FEF8EBDF8012FEFCF01E1
:10031000801B910B8E159F0538F40DB407FEFDCFA1
:100320008EB581932EBDF3CF0DB407FEFDCF8EB5F4
:10033000F801EE0DFF1D808397DF96DFCE01A0DF71
:1003400081E0DF91CF911F910F91FF90EF90DF90AF
:10035000CF9008950F931F93CF93DF93EB010E94EB
:10036000E5C78B0181DF8F3F49F00E94E5C7601B25
:10037000710B6C177D07B0F380E001C081E0DF9165
:10038000CF911F910F910895CF92DF92FF920F931B
:100390001F93CF93DF9300D01F92CDB7DEB76C01D0
:1003A000F62E29833A834B835C836FDF6CE271E026
:1003B000C601D0DF8F2D80645EDF08E110E05C8134
:1003C0004B813A812981DA01C901002E04C0B6951A
:1003D000A795979587950A94D2F729833A834B83FB
:1003E0005C8349DF0850110929813A814B815C8186
:1003F000083F8FEF180739F7FF2029F0E8E0FE16D5
:1004000021F08FEF03C085E901C087E834DFFCE00D
:10041000FF1201C029DF10E027DFF601838387FF89
:1004200004C01F3F11F01F5FF7CF0F900F900F9088
:100430000F90DF91CF911F910F91FF90DF90CF90A0
:100440000895BF92CF92DF92EF92FF920F931F9386
:10045000CF93DF93EC01B62E1C82198248830E9451
:10046000E5C78B0161E088810E94BCC9CE0108DF2D
:1004700060E082E30E94BCC961E083E30E94BCC9E2
:1004800061E084E30E94BCC961E085E30E94BCC9CD
:1004900061E085E30E94F5C985E08A8382E58CBD31
:1004A0001DBC2AE0F22E8FEFE6DEFA94E1F720E0A1
:1004B00030E0A90160E0CE0167DFF82E8B8381E098
:1004C000F81649F00E94E5C7601B710B613D77404B
:1004D00070F381E046C02AEA31E040E050E068E095
:1004E000CE0152DF82FF02C0FC820CC094E0F92EE4
:1004F000BBDE8B83FA94E1F78A3A11F082E031C0D7
:1005000082E08C838C81823031F4C12CD12CE12C9F
:1005100080E4F82E03C0C12CD12C760120E030E01D
:10052000A90167E3CE0130DFA701960169E2CE01A0
:100530002BDF8B83882349F00E94E5C7601B710B7A
:10054000613D774058F38AE00CC08C818230B1F471
:1005500020E030E0A9016AE3CE0116DF882329F00C
:1005600088E08983CE018CDE14C07EDE807C803CF6
:1005700011F483E08C8378DE77DE76DECE0180DED8
:1005800086E08B1518F488E1898303C0BA8281E084
:1005900001C080E0DF91CF911F910F91FF90EF900C
:1005A000DF90CF90BF9008950F931F93CF93DF9369
:1005B000EC0189018C81833039F039E0440F551FFB
:1005C000661F771F3A95D1F79A01AB0161E1CE0121
:1005D000DBDE811109C040E052E0B801CE01DF91BD
:1005E000CF911F910F9166CE84E08983CE0148DEC2
:1005F00080E0DF91CF911F910F910895CF93DF930A
:10060000EC016EBD20E030E00DB407FEFDCFFA0135
:10061000E20FF31F80818EBD0DB407FEFDCF8181F7
:100620008EBD2E5F3F4F211582E0380769F70DB46C
:1006300007FEFDCF8FEF1FDE8FEF1DDE15DE8B83F4
:100640008F71853031F083E18983CE0119DE80E03E
:1006500001C081E0DF91CF9108950F931F93CF9355
:10066000DF93EC0189018C81833039F089E0440FFC
:10067000551F661F771F8A95D1F79A01AB0168E174
:10068000CE0182DE882311F086E01EC0A8016EEF45
:10069000CE01B4DF8823C9F068E572E0CE015ADEEE
:1006A000182F811102C087E10FC020E030E0A901BE
:1006B0006DE0CE0169DE811106C0D6DD811103C077
:1006C000CE01DEDD05C086E18983CE01D9DD10E0F3
:1006D000812FDF91CF911F910F910895CF93DF93D9
:1006E000EC019C012C5F3F4F41E050E060E070E086
:1006F000898D9A8D0E94458E882399F04D895E8957
:100700006F89788D452B462B472B59F44C815D81A1
:100710006E817F814D8B5E8B6F8B788F9981906816
:100720009983DF91CF910895CF92DF92EF92FF925C
:100730000F931F93CF93DF93EC0189899A89AB893B
:10074000BC89803E9F4FAF41B10510F080E06AC088
:10075000CE01C4DF8823D1F30E94598C182F88233F
:10076000A9F3E98DFA8DCC80DD80EE80FF8032E048
:10077000C31AD108E108F108058404C0CC0CDD1CC3
:10078000EE1CFF1C0A94D2F786859785A089B18953
:10079000C80ED91EEA1EFB1E81E08093330FC09263
:1007A0003611D0923711E0923811F092391180E071
:1007B00092E0E6E3FFE0DF019C011D922150304012
:1007C000E1F701E0E98DFA8D8481081788F426E3CA
:1007D0003FE0B701A601400F511D611D711D8091C1
:1007E000340F9091350F39DF8823E1F00F5FEACFA6
:1007F000C12C82E0D82EE12CF12C058404C0CC0C55
:10080000DD1CEE1CFF1C0A94D2F749895A896B89BA
:100810007C894C0D5D1D6E1D7F1D498B5A8B6B8B2A
:100820007C8B812FDF91CF911F910F91FF90EF90E3
:10083000DF90CF900895CF93DF93EC0141E06111F9
:1008400001C040E06C857D858E859F850E94998CD6
:10085000882341F0888920E2829FC00111248A5CAC
:10086000904F02C080E090E0DF91CF91089530E09A
:1008700020E04EE2DC015C91503271F0383029F416
:10088000FB01E20FF11D40832F5FFB01E20FF11D21
:10089000DC015C9150832F5F3F5F01963B3051F745
:1008A000FB01E20FF11D10820895CF93DF93EB015E
:1008B000FC012381211102C080E00EC022502230B1
:1008C00020F48FE28883198206C060E0B4DF0097CD
:1008D00099F3BE01CCDF81E0DF91CF910895FB0158
:1008E0002BE030E231932150E9F7DC0190E027E082
:1008F0003A2FEB2F8D9181110AC0DA013C931196AA
:10090000EC9381E0FB019081903239F525C08F3264
:10091000A1F38E3219F0ECE0F0E108C02A30E1F0EA
:1009200098E02AE0E5CF31963817B1F034913111D3
:10093000FACF291788F03FED380F3E3568F431E0E3
:10094000390FFB01E90FF11D9FE9980F9A3108F467
:1009500080528083932FCCCF80E008950F931F9314
:10096000CF93DF93EC018B018B81882311F080E022
:1009700042C0FB018789803139F18032C1F783E0C1
:100980008B83F801428D538D648D758D4D8B5E8BFD
:100990006F8B788F9E012F5E3F4FC8010E94508D54
:1009A000882329F31A8F098F81E089831C821D8295
:1009B0001E821F82188619861A861B861C861D8633
:1009C0001E861F86188A17C082E08B831D8A1E8AA6
:1009D0001F8A188EFB01408D518D60E070E095E01C
:1009E000440F551F661F771F9A95D1F7498B5A8B75
:1009F0006B8B7C8BD7CFDF91CF911F910F91089597
:100A00002F923F924F925F926F927F928F929F921E
:100A1000AF92BF92CF92DF92EF92FF920F931F930C
:100A2000CF93DF93EC015B016A018B81811103C0DD
:100A30008FEF9FEFC6C0898180FFFACF49895A891D
:100A40006B897C8988859985AA85BB852601612C5F
:100A5000712C8A019B01081B190B2A0B3B0B4016BA
:100A600051066206730618F06A01C81AD90A76019F
:100A70003E0124E0620E711CE114F10409F476C019
:100A8000488559856A857B854A0181E098222B81BA
:100A90001A012B01E9E05694479437942794EA957C
:100AA000D1F7898D9A8DFC01223049F4628D738DC6
:100AB000848D958D620D731D841D951D3CC0148120
:100AC0001150122181149104C1F4111116C0452B4B
:100AD000462B472B49F48D899E89AF89B88D8C832D
:100AE0009D83AE83BF8309C04C815D816E817F8110
:100AF000930157D7882309F49BCFE98DFA8D6C8138
:100B00007D818E819F8162507109810991090584DF
:100B100004C0660F771F881F991F0A94D2F7268595
:100B2000378540895189620F731F841F951F610F9C
:100B3000711D811D911D20E032E0281939098701BE
:100B40002E153F0508F489010115F2E01F0761F534
:100B5000209136113091371140913811509139114F
:100B6000621773078407950719F41EC0C60129C0D0
:100B70009501AB01BC018091340F9091350F14DDCC
:100B8000882309F455CFA00EB11E88859985AA85C2
:100B9000BB85800F911FA11DB11D88879987AA87EA
:100BA000BB87E01AF10A68CF40E0C3D6882309F476
:100BB0003FCFB4016A5C704FA801C5010E94B0D25A
:100BC000E2CFDF91CF911F910F91FF90EF90DF90D7
:100BD000CF90BF90AF909F908F907F906F905F90DD
:100BE0004F903F902F900895CF93DF931F92CDB7F2
:100BF000DEB741E050E0BE016F5F7F4F01DF01973C
:100C000019F4898190E002C08FEF9FEF0F90DF9180
:100C1000CF910895AF92BF92CF92DF92EF92FF9261
:100C20000F931F93CF93DF936C01EB017A01DC01EB
:100C300013968C911397823070F018960D911D9138
:100C40002D913C911B970F71112722273327012BE0
:100C5000022B032B11F08FEF58C04115510511F0F5
:100C6000F70110821DE040E250E0BE01C601C8DE7F
:100C70009C018032910531F081E0232B09F480E062
:100C8000819543C088818823C1F1853E61F38E320E
:100C900051F3E114F10461F19B859F739F3041F59D
:100CA0004A8D5B8D452B21F58F719FEF980F923008
:100CB000F8F490E00197189F9001199F300D1124CE
:100CC000FE0180E090E05701A20EB31E8530B8F41B
:100CD0006181A501480F591FDA016C930196329684
:100CE0008D30910599F7888186FF02C0F501158640
:100CF0008B8583FDB8CF822F08C080E006C08B3083
:100D000010F46481E6CF6681E4CFDF91CF911F912B
:100D10000F91FF90EF90DF90CF90BF90AF9008952C
:100D20001F93CF93DF93EC018B81823018F480E026
:100D300090E023C0488559856A857B85A5E0769536
:100D4000679557954795AA95D1F7142F1F70CE0137
:100D50004BDF97FDECCF488559856A857B85415EE1
:100D60005F4F6F4F7F4F488759876A877B8720E2A5
:100D7000129FC00111248A5C904FDF91CF911F9187
:100D800008954F925F926F927F92AF92BF92CF92EF
:100D9000DF92EF92FF920F931F93CF93DF93EC01BB
:100DA0006A017B012B81222349F089899A89AB89C9
:100DB000BC8984179507A607B70710F480E06BC0BD
:100DC000223009F463C0C114D104E104F10449F4F0
:100DD0001C821D821E821F82188619861A861B8617
:100DE00059C088859985AA85BB85E98DFA8DE585E9
:100DF000F0E03996AC01BD0141505109610971091A
:100E00000E2E04C076956795579547950A94D2F7AC
:100E100097018601015011092109310904C0369555
:100E2000279517950795EA95D2F704171507260712
:100E3000370720F0892B8A2B8B2B49F48D899E89CB
:100E4000AF89B88D8C839D83AE83BF8304C0041BA0
:100E5000150B260B370B280139015E0184E0A80E23
:100E6000B11C411451046104710481F04C815D8115
:100E70006E817F819501898D9A8D93D591E0491A74
:100E80005108610871088111ECCF05C0C886D98668
:100E9000EA86FB8681E0DF91CF911F910F91FF9051
:100EA000EF90DF90CF90BF90AF907F906F905F906A
:100EB0004F9008950F931F93CF93DF93EC018B8195
:100EC0008823D1F1898187FF32C061E0CE01B3DC94
:100ED0008C01009789F1FC018081853E69F18B814D
:100EE000823040F449895A896B897C89448F558FB7
:100EF000668F778F4D895E896F89788DF801538F62
:100F0000428F758B648BE0912D0FF0912E0F3097EF
:100F100059F0B8016A5E7F4FC80148961995F801EB
:100F2000808D918D938B828B89818F778983DF91DF
:100F3000CF911F910F91BDC481E0888380E0DF9144
:100F4000CF911F910F910895CF93DF93EC01B2DF02
:100F50001B82DF91CF910895FC0123812111F4CFF1
:100F600008954F925F926F927F92AF92BF92CF920D
:100F7000DF92EF92FF920F931F93CF93DF9300D0F6
:100F80001F92CDB7DEB75C016A017B01FC01838152
:100F90008130E9F4818181FF1AC0F501818992894C
:100FA000A389B48984179507A607B70780F0892B12
:100FB0008A2B8B2B09F472C0F50140845184628422
:100FC0007384B701A601C501DCDE811102C080E097
:100FD00066C0F501818D928DC114D104E104F10444
:100FE00069F4458956896789708D58D7882379F3C4
:100FF000F501158A168A178A108E37C0F5014481CB
:101000005581668177819E012F5F3F4FCAD4882327
:10101000F1F249815A816B817C81F501818D928D3C
:10102000FC012789203139F4483FFFEF5F07610554
:101030007105D8F407C0483F2FEF520762072FE031
:10104000720798F42BD7882309F4C1CFF5014481A6
:101050005581668177810FEF1FEF2FEF3FE0818D84
:10106000928D84D5882309F4B2CFF501C18AD28A42
:10107000E38AF48A818180688183C5011BDF88232C
:1010800009F4A5CFB701A6014C145D046E047F04DA
:1010900010F4B301A201C50174DE01C081E00F901C
:1010A0000F900F900F90DF91CF911F910F91FF90B4
:1010B000EF90DF90CF90BF90AF907F906F905F9058
:1010C0004F900895FF920F931F93CF93DF93EC01FE
:1010D000F42E80E2689FF0011124EA5CF04F8385D2
:1010E000817121F0842F827109F04EC080913611F8
:1010F00090913711A0913811B09139118C879D874B
:10110000AE87BF87688B4489558960E070E0BA017B
:1011100055274427028D138D20E030E0402B512BC2
:10112000622B732B4D8B5E8B6F8B788F83858871D1
:1011300051F4048D158D268D378D098B1A8B2B8BD1
:101140003C8B81E00BC08031F9F49E012F5E3F4F54
:10115000898D9A8DA5D48823B9F084E08B838F2D57
:101160008F7089831C821D821E821F8218861986B9
:101170001A861B86F4FE0BC040E050E0BA01CE0197
:10118000F0DE811104C011C01B8280E00EC0F5FEAC
:101190000BC049895A896B897C89CE01DF91CF9137
:1011A0001F910F91FF90EDCD81E0DF91CF911F91C5
:1011B0000F91FF900895AF92BF92CF92DF92EF927E
:1011C000FF920F931F93CF93DF937C01EB016A0192
:1011D000B22E898D9A8DF701928F818F40E050E079
:1011E000BA01CE01CEDDA12C088519852A853B8563
:1011F00089899A89AB89BC89081719072A073B078F
:10120000A0F585E036952795179507958A95D1F72E
:101210000F70CE0185DD009709F481C0FC012081AB
:10122000222311F0253EB9F4A1100EC040913611D1
:10123000509137116091381170913911F70144873D
:10124000558766877787008BFC018081AA24A39449
:101250008111CACF0AC04BE050E0BC01C6010E9418
:10126000A3D2892B09F0C0CF58C08B2D8274823451
:1012700009F055C0AA2049F0F701008961E0C701D3
:10128000DADAEC01009769F44AC08B81823009F404
:1012900046C0CE0149DA882309F441C0C6E3DFE045
:1012A00000E080E2FE0111928A95E9F78BE0F601F9
:1012B000DE0101900D928A95E1F7E0912D0FF091FA
:1012C0002E0F309739F0BE01625F7F4FCE014096FE
:1012D000199508C081E298E2998B888B80E098E0AC
:1012E0009F878E87888999899B8B8A8B998F888F16
:1012F0008E859F859F8B8E8BDCD2882381F04B2D32
:10130000602FC701DF91CF911F910F91FF90EF9058
:10131000DF90CF90BF90AF90D5CEB7FEF0CF80E0FA
:10132000DF91CF911F910F91FF90EF90DF90CF90C1
:10133000BF90AF9008953F924F925F926F927F92CD
:101340008F929F92AF92BF92CF92DF92EF92FF92D5
:101350000F931F93CF93DF93CDB7DEB7C354D1095B
:101360000FB6F894DEBF0FBECDBF5C016B012496B3
:101370005FAF4EAF2497522E1C8E1F8E19821C8297
:101380006115710511F410E073C0FC0183818111B6
:10139000FACF2496EEADFFAD249780818F3211F005
:1013A00076011DC02496EEADFFAD249780818F326B
:1013B00031F431962496FFAFEEAF2497F3CFF601C8
:1013C00083818250823060F3F601618D728DCE018F
:1013D0000196C4DA8823B9F2CE0101967C018E0110
:1013E000045E1F4F3801FE0131964F01402E312E11
:1013F00019C08823A9F121E0AE01495C5F4FB70114
:10140000C801D9DE882309F4BECFEC14FD0411F025
:10141000C7019ADD0615170501F1942D832D78017A
:10142000092F182FAE014E5B5F4FBE01695C7F4FE5
:1014300024968EAD9FAD249752DA882309F4A3CF6A
:101440002496EEADFFAD249780818F3291F63196D0
:101450002496FFAFEEAF2497F3CF982D892DDFCFE1
:10146000252DAE01495C5F4FB701C501A4DE182FE1
:10147000CE01019671DDCE014C966EDD812FCD5BE4
:10148000DF4F0FB6F894DEBF0FBECDBFDF91CF9117
:101490001F910F91FF90EF90DF90CF90BF90AF9092
:1014A0009F908F907F906F905F904F903F900895A6
:1014B000CF93DF93EC0140E050E0BA0152DD882386
:1014C00061F061E0CE01B7D9009739F025EEFC015B
:1014D00020831B82DF91CF91ECC180E0DF91CF911F
:1014E00008951F93CF93DF93CDB7DEB76B970FB6F9
:1014F000F894DEBF0FBECDBFAB0119821C8222E083
:10150000BC01CE01019617DF182F882321F0CE01F0
:101510000196CEDF182FCE0101961EDD812F6B962E
:101520000FB6F894DEBF0FBECDBFDF91CF911F91F4
:1015300008952F923F924F925F926F927F928F9277
:101540009F92AF92BF92CF92DF92EF92FF920F9352
:101550001F93CF93DF9300D01F921F92CDB7DEB7BA
:101560008C015B013A01DC0113968C911397813059
:10157000C1F411968C9181FF14C082FF18C0F8014C
:10158000418952896389748980859185A285B38553
:1015900084179507A607B70751F0C801F2DB811140
:1015A00006C081E0F80180838FEF9FEF37C16301B0
:1015B00083C0D80159968D919C915A97FC01F48172
:1015C000F1501A012B0169E05694479437942794FF
:1015D0006A95D1F7F221FD834A0121E09222FF238F
:1015E00009F476C080E092E08819990976018C159B
:1015F0009D0508F47C01D8015996ED91FC915A970C
:1016000014962D903D904D905C901797B2E02B1A58
:10161000310841085108058404C0220C331C441CC5
:10162000551C0A94D2F786859785A089B189280E22
:10163000391E4A1E5B1EED812E0E311C411C511CB1
:10164000E114F2E0FF0609F089C080913611909113
:101650003711A0913811B091391182159305A40565
:10166000B50569F41092330F8FEF9FEFDC01809383
:10167000361190933711A0933811B0933911950119
:10168000B201A1018091340F9091350F0E942D83FA
:10169000882309F486CFF80180859185A285B385DA
:1016A0008E0D9F1DA11DB11D80879187A287B387D5
:1016B000AE0CBF1CCE18DF08D80118964D915D9175
:1016C0006D917C911B97C114D10409F072CF7AC03F
:1016D0008114910409F086CF14964D915D916D911E
:1016E0007C911797411551056105710559F455967F
:1016F0008D919D910D90BC91A02D0097A105B105F4
:1017000039F520C09E012F5F3F4F4BD1882309F44C
:1017100048CF89819A81AB81BC81F801218D328DBE
:10172000F9012789203139F4883FFFEF9F07A10590
:10173000B10540F40DC0883F2FEF9207A2072FE0BC
:10174000B20730F0C8010E946E8381114BCF29CFC0
:10175000F80184839583A683B78344CF81149104D1
:1017600011F5D80118964D915D916D917C911B9763
:1017700051968D919D910D90BC91A02D48175907C0
:101780006A077B0780F095D0882309F40ACF81E0AF
:101790008093330F209236113092371140923811D6
:1017A0005092391107C041E0C201B101C2D0882373
:1017B00009F4F7CEA701B501C4018A5C904F0E94DD
:1017C000B0D269CF51968D919D910D90BC91A02D75
:1017D000F801218184179507A607B70738F4418BD4
:1017E000528B638B748B206821830CC080912D0FEA
:1017F00090912E0F892B31F06114710419F020683B
:10180000F8012183D80111968C9183FD02C0C30198
:1018100005C0C8014FDB8111FACFC3CE0F900F90E6
:101820000F900F900F90DF91CF911F910F91FF902C
:10183000EF90DF90CF90BF90AF909F908F907F9070
:101840006F905F904F903F902F900895CF93DF93CC
:101850001F92CDB7DEB72091EA133091EB13CE0182
:1018600001962115310519F0821B930B02C0805F90
:1018700093410F90DF91CF910895CF93DF931F9203
:10188000CDB7DEB7698341E050E0BE016F5F7F4FA7
:1018900004964FDE0F90DF91CF910895FB010190E8
:1018A0000020E9F7AF0141505109461B570B049640
:1018B00040CECF938091330F8823B9F140913611F8
:1018C00050913711609138117091391126E33FE042
:1018D0008091340F9091350F0E942D83C82F811174
:1018E00002C0C0E023C040912F0F5091300F609193
:1018F000310F7091320F411551056105710591F05D
:1019000026E33FE08091340F9091350F0E942D83A4
:10191000882339F310922F0F1092300F1092310F4D
:101920001092320F1092330F01C0C1E08C2FCF9173
:101930000895CF92DF92EF92FF92CF936B017C01DB
:10194000C42F8091361190913711A0913811B09128
:1019500039118C159D05AE05BF05C9F0AADF8111AF
:1019600002C080E018C026E33FE0B701A6018091E5
:10197000340F9091350F0E94D482882391F3C09246
:101980003611D0923711E0923811F092391181E07E
:10199000C1118093330FCF91FF90EF90DF90CF90E4
:1019A00008958F929F92AF92BF92CF92DF92EF9263
:1019B000FF920F931F93CF93DF93EC016A017B019A
:1019C000890189859A85AB85BC850196A11DB11DCC
:1019D00084179507A607B70710F480E054C08F89D5
:1019E000803129F49927872F762F652F0BC08032FD
:1019F000A1F7CB01BA0127E0969587957795679572
:101A00002A95D1F78B889C88AD88BE88680D791D92
:101A10008A1D9B1D8090361190903711A09038112F
:101A2000B0903911681579058A059B0581F48F8975
:101A3000803191F4DD24EE24FF24F601EE0FFF1F28
:101A4000EA5CF04F80819181A0E0B0E016C040E0F8
:101A500070DF8111ECCFC1CFE894C7F8DD24EE240C
:101A6000FF24F601EE0FFF1FEE0FFF1FEA5CF04FA1
:101A700080819181A281B381BF70F80180839183BD
:101A8000A283B38381E0DF91CF911F910F91FF90EB
:101A9000EF90DF90CF90BF90AF909F908F90089580
:101AA0004F925F926F927F92AF92BF92CF92DF92EE
:101AB000EF92FF920F931F93CF93DF9300D01F926B
:101AC000CDB7DEB78C0149835A836B837C83590180
:101AD000C12CD12C7601412C42E0542E612C712C6A
:101AE00049815A816B817C819E012F5F3F4FC801E4
:101AF00058DF882341F1D301C201F801058404C0F5
:101B0000880F991FAA1FBB1F0A94D2F7C80ED91EAF
:101B1000EA1EFB1E49815A816B817C818789803155
:101B200039F481E0483F5F4F6105710538F4D8CF43
:101B300081E0483F5F4F6F4F7F4090F2F501C082D8
:101B4000D182E282F3820F900F900F900F90DF917D
:101B5000CF911F910F91FF90EF90DF90CF90BF90AA
:101B6000AF907F906F905F904F9008954F925F92EB
:101B70006F927F928F929F92AF92BF92CF92DF929D
:101B8000EF92FF920F931F93CF93DF93EC014A01E3
:101B90005B0128013901423051056105710508F4E6
:101BA00062C049855A856B857C854F5F5F4F6F4F5B
:101BB0007F4F481559056A057B0508F454C08F8985
:101BC000803129F4FF24EB2CDA2CC92C0CC0803294
:101BD00009F049C07501640177E0F694E794D79461
:101BE000C7947A95D1F74B895C896D897E89C40E3B
:101BF000D51EE61EF71E41E0C701B6019ADE882316
:101C000091F19F89903159F49924AA24BB24F401BD
